Archive member included to satisfy reference by file (symbol)

.\CortexM3\ARM_GCC_541\Debug\VCNL4030X01.a(I2C_1.o)
                              .\CortexM3\ARM_GCC_541\Debug\main.o (I2C_1_Start)
.\CortexM3\ARM_GCC_541\Debug\VCNL4030X01.a(I2C_1_INT.o)
                              .\CortexM3\ARM_GCC_541\Debug\VCNL4030X01.a(I2C_1.o) (I2C_1_ISR)
.\CortexM3\ARM_GCC_541\Debug\VCNL4030X01.a(I2C_1_PM.o)
                              .\CortexM3\ARM_GCC_541\Debug\VCNL4030X01.a(I2C_1.o) (I2C_1_backup)
.\CortexM3\ARM_GCC_541\Debug\VCNL4030X01.a(I2C_1_MASTER.o)
                              .\CortexM3\ARM_GCC_541\Debug\VCNL4030X01.a(I2C_1.o) (I2C_1_mstrStatus)
.\CortexM3\ARM_GCC_541\Debug\VCNL4030X01.a(CDC.o)
                              .\CortexM3\ARM_GCC_541\Debug\main.o (CDC_Start)
.\CortexM3\ARM_GCC_541\Debug\VCNL4030X01.a(CDC_cdc.o)
                              .\CortexM3\ARM_GCC_541\Debug\main.o (CDC_CDC_Init)
.\CortexM3\ARM_GCC_541\Debug\VCNL4030X01.a(CDC_drv.o)
                              .\CortexM3\ARM_GCC_541\Debug\VCNL4030X01.a(CDC.o) (CDC_lastPacketSize)
.\CortexM3\ARM_GCC_541\Debug\VCNL4030X01.a(CDC_episr.o)
                              .\CortexM3\ARM_GCC_541\Debug\VCNL4030X01.a(CDC.o) (CDC_EP_1_ISR)
.\CortexM3\ARM_GCC_541\Debug\VCNL4030X01.a(CDC_pm.o)
                              .\CortexM3\ARM_GCC_541\Debug\VCNL4030X01.a(CDC.o) (CDC_DP_ISR)
.\CortexM3\ARM_GCC_541\Debug\VCNL4030X01.a(CDC_std.o)
                              .\CortexM3\ARM_GCC_541\Debug\VCNL4030X01.a(CDC_pm.o) (CDC_ConfigReg)
.\CortexM3\ARM_GCC_541\Debug\VCNL4030X01.a(CDC_vnd.o)
                              .\CortexM3\ARM_GCC_541\Debug\VCNL4030X01.a(CDC_drv.o) (CDC_HandleVendorRqst)
.\CortexM3\ARM_GCC_541\Debug\VCNL4030X01.a(CDC_Dp.o)
                              .\CortexM3\ARM_GCC_541\Debug\VCNL4030X01.a(CDC.o) (CDC_Dp_ClearInterrupt)
.\CortexM3\ARM_GCC_541\Debug\VCNL4030X01.a(CyLib.o)
                              .\CortexM3\ARM_GCC_541\Debug\Cm3Start.o (CyHalt)
.\CortexM3\ARM_GCC_541\Debug\VCNL4030X01.a(cyPm.o)
                              .\CortexM3\ARM_GCC_541\Debug\VCNL4030X01.a(CyLib.o) (CyPmReadStatus)
.\CortexM3\ARM_GCC_541\Debug\VCNL4030X01.a(CyBootAsmGnu.o)
                              .\CortexM3\ARM_GCC_541\Debug\cyfitter_cfg.o (CyDelayCycles)
.\CortexM3\ARM_GCC_541\Debug\VCNL4030X01.a(CDC_cls.o)
                              .\CortexM3\ARM_GCC_541\Debug\VCNL4030X01.a(CDC_drv.o) (CDC_DispatchClassRqst)
.\CortexM3\ARM_GCC_541\Debug\VCNL4030X01.a(CDC_descr.o)
                              .\CortexM3\ARM_GCC_541\Debug\VCNL4030X01.a(CDC_std.o) (CDC_idSerialNumberStringDescriptor)
.\CortexM3\ARM_GCC_541\Debug\VCNL4030X01.a(CyFlash.o)
                              .\CortexM3\ARM_GCC_541\Debug\VCNL4030X01.a(cyPm.o) (CyFlash_SetWaitCycles)
.\CortexM3\ARM_GCC_541\Debug\VCNL4030X01.a(CySpc.o)
                              .\CortexM3\ARM_GCC_541\Debug\VCNL4030X01.a(CyFlash.o) (CySpcStart)
c:/program files (x86)/cypress/psoc creator/4.3/psoc creator/import/gnu/arm/5.4.1/bin/../lib/gcc/arm-none-eabi/5.4.1/../../../../arm-none-eabi/lib/armv7-m\libm.a(lib_a-w_pow.o)
                              .\CortexM3\ARM_GCC_541\Debug\VCNL4030X01_Application_Library.o (pow)
c:/program files (x86)/cypress/psoc creator/4.3/psoc creator/import/gnu/arm/5.4.1/bin/../lib/gcc/arm-none-eabi/5.4.1/../../../../arm-none-eabi/lib/armv7-m\libm.a(lib_a-e_pow.o)
                              c:/program files (x86)/cypress/psoc creator/4.3/psoc creator/import/gnu/arm/5.4.1/bin/../lib/gcc/arm-none-eabi/5.4.1/../../../../arm-none-eabi/lib/armv7-m\libm.a(lib_a-w_pow.o) (__ieee754_pow)
c:/program files (x86)/cypress/psoc creator/4.3/psoc creator/import/gnu/arm/5.4.1/bin/../lib/gcc/arm-none-eabi/5.4.1/../../../../arm-none-eabi/lib/armv7-m\libm.a(lib_a-e_sqrt.o)
                              c:/program files (x86)/cypress/psoc creator/4.3/psoc creator/import/gnu/arm/5.4.1/bin/../lib/gcc/arm-none-eabi/5.4.1/../../../../arm-none-eabi/lib/armv7-m\libm.a(lib_a-e_pow.o) (__ieee754_sqrt)
c:/program files (x86)/cypress/psoc creator/4.3/psoc creator/import/gnu/arm/5.4.1/bin/../lib/gcc/arm-none-eabi/5.4.1/../../../../arm-none-eabi/lib/armv7-m\libm.a(lib_a-s_fabs.o)
                              c:/program files (x86)/cypress/psoc creator/4.3/psoc creator/import/gnu/arm/5.4.1/bin/../lib/gcc/arm-none-eabi/5.4.1/../../../../arm-none-eabi/lib/armv7-m\libm.a(lib_a-e_pow.o) (fabs)
c:/program files (x86)/cypress/psoc creator/4.3/psoc creator/import/gnu/arm/5.4.1/bin/../lib/gcc/arm-none-eabi/5.4.1/../../../../arm-none-eabi/lib/armv7-m\libm.a(lib_a-s_finite.o)
                              c:/program files (x86)/cypress/psoc creator/4.3/psoc creator/import/gnu/arm/5.4.1/bin/../lib/gcc/arm-none-eabi/5.4.1/../../../../arm-none-eabi/lib/armv7-m\libm.a(lib_a-w_pow.o) (finite)
c:/program files (x86)/cypress/psoc creator/4.3/psoc creator/import/gnu/arm/5.4.1/bin/../lib/gcc/arm-none-eabi/5.4.1/../../../../arm-none-eabi/lib/armv7-m\libm.a(lib_a-s_lib_ver.o)
                              c:/program files (x86)/cypress/psoc creator/4.3/psoc creator/import/gnu/arm/5.4.1/bin/../lib/gcc/arm-none-eabi/5.4.1/../../../../arm-none-eabi/lib/armv7-m\libm.a(lib_a-w_pow.o) (__fdlib_version)
c:/program files (x86)/cypress/psoc creator/4.3/psoc creator/import/gnu/arm/5.4.1/bin/../lib/gcc/arm-none-eabi/5.4.1/../../../../arm-none-eabi/lib/armv7-m\libm.a(lib_a-s_matherr.o)
                              c:/program files (x86)/cypress/psoc creator/4.3/psoc creator/import/gnu/arm/5.4.1/bin/../lib/gcc/arm-none-eabi/5.4.1/../../../../arm-none-eabi/lib/armv7-m\libm.a(lib_a-w_pow.o) (matherr)
c:/program files (x86)/cypress/psoc creator/4.3/psoc creator/import/gnu/arm/5.4.1/bin/../lib/gcc/arm-none-eabi/5.4.1/../../../../arm-none-eabi/lib/armv7-m\libm.a(lib_a-s_nan.o)
                              c:/program files (x86)/cypress/psoc creator/4.3/psoc creator/import/gnu/arm/5.4.1/bin/../lib/gcc/arm-none-eabi/5.4.1/../../../../arm-none-eabi/lib/armv7-m\libm.a(lib_a-e_pow.o) (nan)
c:/program files (x86)/cypress/psoc creator/4.3/psoc creator/import/gnu/arm/5.4.1/bin/../lib/gcc/arm-none-eabi/5.4.1/../../../../arm-none-eabi/lib/armv7-m\libm.a(lib_a-s_rint.o)
                              c:/program files (x86)/cypress/psoc creator/4.3/psoc creator/import/gnu/arm/5.4.1/bin/../lib/gcc/arm-none-eabi/5.4.1/../../../../arm-none-eabi/lib/armv7-m\libm.a(lib_a-w_pow.o) (rint)
c:/program files (x86)/cypress/psoc creator/4.3/psoc creator/import/gnu/arm/5.4.1/bin/../lib/gcc/arm-none-eabi/5.4.1/../../../../arm-none-eabi/lib/armv7-m\libm.a(lib_a-s_scalbn.o)
                              c:/program files (x86)/cypress/psoc creator/4.3/psoc creator/import/gnu/arm/5.4.1/bin/../lib/gcc/arm-none-eabi/5.4.1/../../../../arm-none-eabi/lib/armv7-m\libm.a(lib_a-e_pow.o) (scalbn)
c:/program files (x86)/cypress/psoc creator/4.3/psoc creator/import/gnu/arm/5.4.1/bin/../lib/gcc/arm-none-eabi/5.4.1/../../../../arm-none-eabi/lib/armv7-m\libm.a(lib_a-s_copysign.o)
                              c:/program files (x86)/cypress/psoc creator/4.3/psoc creator/import/gnu/arm/5.4.1/bin/../lib/gcc/arm-none-eabi/5.4.1/../../../../arm-none-eabi/lib/armv7-m\libm.a(lib_a-s_scalbn.o) (copysign)
c:/program files (x86)/cypress/psoc creator/4.3/psoc creator/import/gnu/arm/5.4.1/bin/../lib/gcc/arm-none-eabi/5.4.1/armv7-m\libgcc.a(_arm_addsubdf3.o)
                              c:/program files (x86)/cypress/psoc creator/4.3/psoc creator/import/gnu/arm/5.4.1/bin/../lib/gcc/arm-none-eabi/5.4.1/../../../../arm-none-eabi/lib/armv7-m\libm.a(lib_a-e_pow.o) (__aeabi_dsub)
c:/program files (x86)/cypress/psoc creator/4.3/psoc creator/import/gnu/arm/5.4.1/bin/../lib/gcc/arm-none-eabi/5.4.1/armv7-m\libgcc.a(_arm_muldivdf3.o)
                              .\CortexM3\ARM_GCC_541\Debug\VCNL4030X01_Application_Library.o (__aeabi_dmul)
c:/program files (x86)/cypress/psoc creator/4.3/psoc creator/import/gnu/arm/5.4.1/bin/../lib/gcc/arm-none-eabi/5.4.1/armv7-m\libgcc.a(_arm_cmpdf2.o)
                              c:/program files (x86)/cypress/psoc creator/4.3/psoc creator/import/gnu/arm/5.4.1/bin/../lib/gcc/arm-none-eabi/5.4.1/../../../../arm-none-eabi/lib/armv7-m\libm.a(lib_a-w_pow.o) (__aeabi_dcmpeq)
c:/program files (x86)/cypress/psoc creator/4.3/psoc creator/import/gnu/arm/5.4.1/bin/../lib/gcc/arm-none-eabi/5.4.1/armv7-m\libgcc.a(_arm_unorddf2.o)
                              c:/program files (x86)/cypress/psoc creator/4.3/psoc creator/import/gnu/arm/5.4.1/bin/../lib/gcc/arm-none-eabi/5.4.1/../../../../arm-none-eabi/lib/armv7-m\libm.a(lib_a-w_pow.o) (__aeabi_dcmpun)
c:/program files (x86)/cypress/psoc creator/4.3/psoc creator/import/gnu/arm/5.4.1/bin/../lib/gcc/arm-none-eabi/5.4.1/armv7-m\libgcc.a(_arm_truncdfsf2.o)
                              .\CortexM3\ARM_GCC_541\Debug\VCNL4030X01_Application_Library.o (__aeabi_d2f)
c:/program files (x86)/cypress/psoc creator/4.3/psoc creator/import/gnu/arm/5.4.1/bin/../lib/gcc/arm-none-eabi/5.4.1/armv7-m\libgcc.a(_arm_addsubsf3.o)
                              .\CortexM3\ARM_GCC_541\Debug\VCNL4030X01_Application_Library.o (__aeabi_fsub)
c:/program files (x86)/cypress/psoc creator/4.3/psoc creator/import/gnu/arm/5.4.1/bin/../lib/gcc/arm-none-eabi/5.4.1/armv7-m\libgcc.a(_arm_muldivsf3.o)
                              .\CortexM3\ARM_GCC_541\Debug\VCNL4030X01_Application_Library.o (__aeabi_fmul)
c:/program files (x86)/cypress/psoc creator/4.3/psoc creator/import/gnu/arm/5.4.1/bin/../lib/gcc/arm-none-eabi/5.4.1/armv7-m\libgcc.a(_arm_fixsfsi.o)
                              .\CortexM3\ARM_GCC_541\Debug\VCNL4030X01_Application_Library.o (__aeabi_f2iz)
c:/program files (x86)/cypress/psoc creator/4.3/psoc creator/import/gnu/arm/5.4.1/bin/../lib/gcc/arm-none-eabi/5.4.1/../../../../arm-none-eabi/lib/armv7-m\libg_nano.a(lib_a-errno.o)
                              .\CortexM3\ARM_GCC_541\Debug\Cm3Start.o (__errno)
c:/program files (x86)/cypress/psoc creator/4.3/psoc creator/import/gnu/arm/5.4.1/bin/../lib/gcc/arm-none-eabi/5.4.1/../../../../arm-none-eabi/lib/armv7-m\libg_nano.a(lib_a-exit.o)
                              c:/program files (x86)/cypress/psoc creator/4.3/psoc creator/import/gnu/arm/5.4.1/bin/../lib/gcc/arm-none-eabi/5.4.1/../../../../arm-none-eabi/lib/armv7-m/crt0.o (exit)
c:/program files (x86)/cypress/psoc creator/4.3/psoc creator/import/gnu/arm/5.4.1/bin/../lib/gcc/arm-none-eabi/5.4.1/../../../../arm-none-eabi/lib/armv7-m\libg_nano.a(lib_a-impure.o)
                              c:/program files (x86)/cypress/psoc creator/4.3/psoc creator/import/gnu/arm/5.4.1/bin/../lib/gcc/arm-none-eabi/5.4.1/../../../../arm-none-eabi/lib/armv7-m\libg_nano.a(lib_a-exit.o) (_global_impure_ptr)
c:/program files (x86)/cypress/psoc creator/4.3/psoc creator/import/gnu/arm/5.4.1/bin/../lib/gcc/arm-none-eabi/5.4.1/../../../../arm-none-eabi/lib/armv7-m\libg_nano.a(lib_a-init.o)
                              c:/program files (x86)/cypress/psoc creator/4.3/psoc creator/import/gnu/arm/5.4.1/bin/../lib/gcc/arm-none-eabi/5.4.1/../../../../arm-none-eabi/lib/armv7-m/crt0.o (__libc_init_array)
c:/program files (x86)/cypress/psoc creator/4.3/psoc creator/import/gnu/arm/5.4.1/bin/../lib/gcc/arm-none-eabi/5.4.1/../../../../arm-none-eabi/lib/armv7-m\libg_nano.a(lib_a-memcpy-stub.o)
                              .\CortexM3\ARM_GCC_541\Debug\cyfitter_cfg.o (memcpy)
c:/program files (x86)/cypress/psoc creator/4.3/psoc creator/import/gnu/arm/5.4.1/bin/../lib/gcc/arm-none-eabi/5.4.1/../../../../arm-none-eabi/lib/armv7-m\libg_nano.a(lib_a-memset.o)
                              c:/program files (x86)/cypress/psoc creator/4.3/psoc creator/import/gnu/arm/5.4.1/bin/../lib/gcc/arm-none-eabi/5.4.1/../../../../arm-none-eabi/lib/armv7-m/crt0.o (memset)
c:/program files (x86)/cypress/psoc creator/4.3/psoc creator/import/gnu/arm/5.4.1/bin/../lib/gcc/arm-none-eabi/5.4.1/../../../../arm-none-eabi/lib/armv7-m\libg_nano.a(lib_a-sprintf.o)
                              .\CortexM3\ARM_GCC_541\Debug\VCNL4030X01_Application_Library.o (sprintf)
c:/program files (x86)/cypress/psoc creator/4.3/psoc creator/import/gnu/arm/5.4.1/bin/../lib/gcc/arm-none-eabi/5.4.1/../../../../arm-none-eabi/lib/armv7-m\libg_nano.a(lib_a-nano-svfprintf.o)
                              c:/program files (x86)/cypress/psoc creator/4.3/psoc creator/import/gnu/arm/5.4.1/bin/../lib/gcc/arm-none-eabi/5.4.1/../../../../arm-none-eabi/lib/armv7-m\libg_nano.a(lib_a-sprintf.o) (_svfprintf_r)
c:/program files (x86)/cypress/psoc creator/4.3/psoc creator/import/gnu/arm/5.4.1/bin/../lib/gcc/arm-none-eabi/5.4.1/../../../../arm-none-eabi/lib/armv7-m\libg_nano.a(lib_a-nano-vfprintf_i.o)
                              c:/program files (x86)/cypress/psoc creator/4.3/psoc creator/import/gnu/arm/5.4.1/bin/../lib/gcc/arm-none-eabi/5.4.1/../../../../arm-none-eabi/lib/armv7-m\libg_nano.a(lib_a-nano-svfprintf.o) (_printf_i)
c:/program files (x86)/cypress/psoc creator/4.3/psoc creator/import/gnu/arm/5.4.1/bin/../lib/gcc/arm-none-eabi/5.4.1/../../../../arm-none-eabi/lib/armv7-m\libg_nano.a(lib_a-memchr-stub.o)
                              c:/program files (x86)/cypress/psoc creator/4.3/psoc creator/import/gnu/arm/5.4.1/bin/../lib/gcc/arm-none-eabi/5.4.1/../../../../arm-none-eabi/lib/armv7-m\libg_nano.a(lib_a-nano-svfprintf.o) (memchr)
c:/program files (x86)/cypress/psoc creator/4.3/psoc creator/import/gnu/arm/5.4.1/bin/../lib/gcc/arm-none-eabi/5.4.1/../../../../arm-none-eabi/lib/armv7-m\libg_nano.a(lib_a-memmove.o)
                              c:/program files (x86)/cypress/psoc creator/4.3/psoc creator/import/gnu/arm/5.4.1/bin/../lib/gcc/arm-none-eabi/5.4.1/../../../../arm-none-eabi/lib/armv7-m\libg_nano.a(lib_a-nano-svfprintf.o) (memmove)
c:/program files (x86)/cypress/psoc creator/4.3/psoc creator/import/gnu/arm/5.4.1/bin/../lib/gcc/arm-none-eabi/5.4.1/../../../../arm-none-eabi/lib/armv7-m\libg_nano.a(lib_a-nano-freer.o)
                              c:/program files (x86)/cypress/psoc creator/4.3/psoc creator/import/gnu/arm/5.4.1/bin/../lib/gcc/arm-none-eabi/5.4.1/../../../../arm-none-eabi/lib/armv7-m\libg_nano.a(lib_a-nano-svfprintf.o) (_free_r)
c:/program files (x86)/cypress/psoc creator/4.3/psoc creator/import/gnu/arm/5.4.1/bin/../lib/gcc/arm-none-eabi/5.4.1/../../../../arm-none-eabi/lib/armv7-m\libg_nano.a(lib_a-nano-mallocr.o)
                              c:/program files (x86)/cypress/psoc creator/4.3/psoc creator/import/gnu/arm/5.4.1/bin/../lib/gcc/arm-none-eabi/5.4.1/../../../../arm-none-eabi/lib/armv7-m\libg_nano.a(lib_a-nano-svfprintf.o) (_malloc_r)
c:/program files (x86)/cypress/psoc creator/4.3/psoc creator/import/gnu/arm/5.4.1/bin/../lib/gcc/arm-none-eabi/5.4.1/../../../../arm-none-eabi/lib/armv7-m\libg_nano.a(lib_a-nano-reallocr.o)
                              c:/program files (x86)/cypress/psoc creator/4.3/psoc creator/import/gnu/arm/5.4.1/bin/../lib/gcc/arm-none-eabi/5.4.1/../../../../arm-none-eabi/lib/armv7-m\libg_nano.a(lib_a-nano-svfprintf.o) (_realloc_r)
c:/program files (x86)/cypress/psoc creator/4.3/psoc creator/import/gnu/arm/5.4.1/bin/../lib/gcc/arm-none-eabi/5.4.1/../../../../arm-none-eabi/lib/armv7-m\libg_nano.a(lib_a-sbrkr.o)
                              c:/program files (x86)/cypress/psoc creator/4.3/psoc creator/import/gnu/arm/5.4.1/bin/../lib/gcc/arm-none-eabi/5.4.1/../../../../arm-none-eabi/lib/armv7-m\libg_nano.a(lib_a-nano-mallocr.o) (_sbrk_r)
c:/program files (x86)/cypress/psoc creator/4.3/psoc creator/import/gnu/arm/5.4.1/bin/../lib/gcc/arm-none-eabi/5.4.1/../../../../arm-none-eabi/lib/armv7-m\libg_nano.a(lib_a-mlock.o)
                              c:/program files (x86)/cypress/psoc creator/4.3/psoc creator/import/gnu/arm/5.4.1/bin/../lib/gcc/arm-none-eabi/5.4.1/../../../../arm-none-eabi/lib/armv7-m\libg_nano.a(lib_a-nano-freer.o) (__malloc_lock)
c:/program files (x86)/cypress/psoc creator/4.3/psoc creator/import/gnu/arm/5.4.1/bin/../lib/gcc/arm-none-eabi/5.4.1/../../../../arm-none-eabi/lib/armv7-m\libg_nano.a(lib_a-nano-msizer.o)
                              c:/program files (x86)/cypress/psoc creator/4.3/psoc creator/import/gnu/arm/5.4.1/bin/../lib/gcc/arm-none-eabi/5.4.1/../../../../arm-none-eabi/lib/armv7-m\libg_nano.a(lib_a-nano-reallocr.o) (_malloc_usable_size_r)
c:/program files (x86)/cypress/psoc creator/4.3/psoc creator/import/gnu/arm/5.4.1/bin/../lib/gcc/arm-none-eabi/5.4.1/../../../../arm-none-eabi/lib/armv7-m\libg_nano.a(lib_a-reent.o)
                              c:/program files (x86)/cypress/psoc creator/4.3/psoc creator/import/gnu/arm/5.4.1/bin/../lib/gcc/arm-none-eabi/5.4.1/../../../../arm-none-eabi/lib/armv7-m\libg_nano.a(lib_a-sbrkr.o) (errno)

Allocating common symbols
Common symbol       size              file

CDC_linesControlBitmap
                    0x4               .\CortexM3\ARM_GCC_541\Debug\VCNL4030X01.a(CDC_cdc.o)
CDC_idSerialNumberStringDescriptor
                    0x22              .\CortexM3\ARM_GCC_541\Debug\VCNL4030X01.a(CDC_descr.o)
CDC_device          0x1               .\CortexM3\ARM_GCC_541\Debug\VCNL4030X01.a(CDC_drv.o)
CDC_interfaceSettingLast
                    0x2               .\CortexM3\ARM_GCC_541\Debug\VCNL4030X01.a(CDC_drv.o)
CDC_EP              0x6c              .\CortexM3\ARM_GCC_541\Debug\VCNL4030X01.a(CDC_drv.o)
CDC_transferState   0x1               .\CortexM3\ARM_GCC_541\Debug\VCNL4030X01.a(CDC_drv.o)
errno               0x4               c:/program files (x86)/cypress/psoc creator/4.3/psoc creator/import/gnu/arm/5.4.1/bin/../lib/gcc/arm-none-eabi/5.4.1/../../../../arm-none-eabi/lib/armv7-m\libg_nano.a(lib_a-reent.o)
CDC_ep0Toggle       0x1               .\CortexM3\ARM_GCC_541\Debug\VCNL4030X01.a(CDC_drv.o)
CDC_cdcDataOutEp    0x2               .\CortexM3\ARM_GCC_541\Debug\VCNL4030X01.a(CDC_cdc.o)
I2C_1_mstrWrBufIndex
                    0x1               .\CortexM3\ARM_GCC_541\Debug\VCNL4030X01.a(I2C_1_MASTER.o)
CDC_configurationChanged
                    0x1               .\CortexM3\ARM_GCC_541\Debug\VCNL4030X01.a(CDC_drv.o)
CDC_ep0Count        0x1               .\CortexM3\ARM_GCC_541\Debug\VCNL4030X01.a(CDC_drv.o)
I2C_1_mstrControl   0x1               .\CortexM3\ARM_GCC_541\Debug\VCNL4030X01.a(I2C_1_MASTER.o)
CDC_linesChanged    0x2               .\CortexM3\ARM_GCC_541\Debug\VCNL4030X01.a(CDC_cdc.o)
CDC_deviceStatus    0x1               .\CortexM3\ARM_GCC_541\Debug\VCNL4030X01.a(CDC_drv.o)
CDC_configuration   0x1               .\CortexM3\ARM_GCC_541\Debug\VCNL4030X01.a(CDC_drv.o)
CDC_cdcCommInInterruptEp
                    0x2               .\CortexM3\ARM_GCC_541\Debug\VCNL4030X01.a(CDC_cdc.o)
CDC_interfaceClass  0x4               .\CortexM3\ARM_GCC_541\Debug\VCNL4030X01.a(CDC_drv.o)
CDC_ep0Mode         0x1               .\CortexM3\ARM_GCC_541\Debug\VCNL4030X01.a(CDC_drv.o)
CDC_interfaceStatus
                    0x2               .\CortexM3\ARM_GCC_541\Debug\VCNL4030X01.a(CDC_drv.o)
I2C_1_mstrStatus    0x1               .\CortexM3\ARM_GCC_541\Debug\VCNL4030X01.a(I2C_1_MASTER.o)
I2C_1_mstrWrBufSize
                    0x1               .\CortexM3\ARM_GCC_541\Debug\VCNL4030X01.a(I2C_1_MASTER.o)
CDC_transferByteCount
                    0x2               .\CortexM3\ARM_GCC_541\Debug\VCNL4030X01.a(CDC_drv.o)
CDC_currentTD       0xc               .\CortexM3\ARM_GCC_541\Debug\VCNL4030X01.a(CDC_drv.o)
CDC_deviceAddress   0x1               .\CortexM3\ARM_GCC_541\Debug\VCNL4030X01.a(CDC_drv.o)
I2C_1_mstrRdBufIndex
                    0x1               .\CortexM3\ARM_GCC_541\Debug\VCNL4030X01.a(I2C_1_MASTER.o)
CDC_interfaceNumber
                    0x1               .\CortexM3\ARM_GCC_541\Debug\VCNL4030X01.a(CDC_drv.o)
CDC_cdcDataInEp     0x2               .\CortexM3\ARM_GCC_541\Debug\VCNL4030X01.a(CDC_cdc.o)
CDC_interfaceSetting
                    0x2               .\CortexM3\ARM_GCC_541\Debug\VCNL4030X01.a(CDC_drv.o)
I2C_1_state         0x1               .\CortexM3\ARM_GCC_541\Debug\VCNL4030X01.a(I2C_1.o)
I2C_1_mstrWrBufPtr  0x4               .\CortexM3\ARM_GCC_541\Debug\VCNL4030X01.a(I2C_1_MASTER.o)
dieTemperature      0x2               .\CortexM3\ARM_GCC_541\Debug\VCNL4030X01.a(CyFlash.o)
I2C_1_mstrRdBufPtr  0x4               .\CortexM3\ARM_GCC_541\Debug\VCNL4030X01.a(I2C_1_MASTER.o)
CDC_lastPacketSize  0x1               .\CortexM3\ARM_GCC_541\Debug\VCNL4030X01.a(CDC_drv.o)
I2C_1_mstrRdBufSize
                    0x1               .\CortexM3\ARM_GCC_541\Debug\VCNL4030X01.a(I2C_1_MASTER.o)
CDC_serialStateBitmap
                    0x4               .\CortexM3\ARM_GCC_541\Debug\VCNL4030X01.a(CDC_cdc.o)

Discarded input sections

 .text          0x00000000        0x0 c:/program files (x86)/cypress/psoc creator/4.3/psoc creator/import/gnu/arm/5.4.1/bin/../lib/gcc/arm-none-eabi/5.4.1/armv7-m/crti.o
 .data          0x00000000        0x0 c:/program files (x86)/cypress/psoc creator/4.3/psoc creator/import/gnu/arm/5.4.1/bin/../lib/gcc/arm-none-eabi/5.4.1/armv7-m/crti.o
 .bss           0x00000000        0x0 c:/program files (x86)/cypress/psoc creator/4.3/psoc creator/import/gnu/arm/5.4.1/bin/../lib/gcc/arm-none-eabi/5.4.1/armv7-m/crti.o
 .data          0x00000000        0x4 c:/program files (x86)/cypress/psoc creator/4.3/psoc creator/import/gnu/arm/5.4.1/bin/../lib/gcc/arm-none-eabi/5.4.1/armv7-m/crtbegin.o
 .text          0x00000000       0x74 c:/program files (x86)/cypress/psoc creator/4.3/psoc creator/import/gnu/arm/5.4.1/bin/../lib/gcc/arm-none-eabi/5.4.1/../../../../arm-none-eabi/lib/armv7-m/crt0.o
 .data          0x00000000        0x0 c:/program files (x86)/cypress/psoc creator/4.3/psoc creator/import/gnu/arm/5.4.1/bin/../lib/gcc/arm-none-eabi/5.4.1/../../../../arm-none-eabi/lib/armv7-m/crt0.o
 .bss           0x00000000        0x0 c:/program files (x86)/cypress/psoc creator/4.3/psoc creator/import/gnu/arm/5.4.1/bin/../lib/gcc/arm-none-eabi/5.4.1/../../../../arm-none-eabi/lib/armv7-m/crt0.o
 .ARM.extab     0x00000000        0x0 c:/program files (x86)/cypress/psoc creator/4.3/psoc creator/import/gnu/arm/5.4.1/bin/../lib/gcc/arm-none-eabi/5.4.1/../../../../arm-none-eabi/lib/armv7-m/crt0.o
 .ARM.exidx     0x00000000        0x8 c:/program files (x86)/cypress/psoc creator/4.3/psoc creator/import/gnu/arm/5.4.1/bin/../lib/gcc/arm-none-eabi/5.4.1/../../../../arm-none-eabi/lib/armv7-m/crt0.o
 .text          0x00000000        0x0 .\CortexM3\ARM_GCC_541\Debug\main.o
 .bss           0x00000000        0x4 .\CortexM3\ARM_GCC_541\Debug\main.o
 .text.White_Mode
                0x00000000       0x34 .\CortexM3\ARM_GCC_541\Debug\main.o
 .text.ALS_Mode
                0x00000000       0x58 .\CortexM3\ARM_GCC_541\Debug\main.o
 .text.Low_Power_Mode
                0x00000000       0xd8 .\CortexM3\ARM_GCC_541\Debug\main.o
 .text.AF_Mode  0x00000000       0xe0 .\CortexM3\ARM_GCC_541\Debug\main.o
 .text.Auto_Mode
                0x00000000       0xd8 .\CortexM3\ARM_GCC_541\Debug\main.o
 .text          0x00000000        0x0 .\CortexM3\ARM_GCC_541\Debug\I2C_Functions.o
 .data          0x00000000        0x0 .\CortexM3\ARM_GCC_541\Debug\I2C_Functions.o
 .bss           0x00000000        0x0 .\CortexM3\ARM_GCC_541\Debug\I2C_Functions.o
 .text          0x00000000        0x0 .\CortexM3\ARM_GCC_541\Debug\VCNL4030X01_PS.o
 .data          0x00000000        0x0 .\CortexM3\ARM_GCC_541\Debug\VCNL4030X01_PS.o
 .bss           0x00000000        0x0 .\CortexM3\ARM_GCC_541\Debug\VCNL4030X01_PS.o
 .text.VCNL4030X01_SET_PS_DUTY
                0x00000000       0x44 .\CortexM3\ARM_GCC_541\Debug\VCNL4030X01_PS.o
 .text.VCNL4030X01_SET_PS_PERS
                0x00000000       0x44 .\CortexM3\ARM_GCC_541\Debug\VCNL4030X01_PS.o
 .text.VCNL4030X01_SET_PS_Gain
                0x00000000       0x44 .\CortexM3\ARM_GCC_541\Debug\VCNL4030X01_PS.o
 .text.VCNL4030X01_SET_PS_NS
                0x00000000       0x44 .\CortexM3\ARM_GCC_541\Debug\VCNL4030X01_PS.o
 .text.VCNL4030X01_SET_PS_INT
                0x00000000       0x44 .\CortexM3\ARM_GCC_541\Debug\VCNL4030X01_PS.o
 .text.VCNL4030X01_SET_PS_LED_I_LOW
                0x00000000       0x44 .\CortexM3\ARM_GCC_541\Debug\VCNL4030X01_PS.o
 .text.VCNL4030X01_SET_PS_SMART_PERS
                0x00000000       0x44 .\CortexM3\ARM_GCC_541\Debug\VCNL4030X01_PS.o
 .text.VCNL4030X01_SET_PS_MS
                0x00000000       0x44 .\CortexM3\ARM_GCC_541\Debug\VCNL4030X01_PS.o
 .text.VCNL4030X01_SET_PS_SC_CUR
                0x00000000       0x44 .\CortexM3\ARM_GCC_541\Debug\VCNL4030X01_PS.o
 .text.VCNL4030X01_SET_PS_SP
                0x00000000       0x44 .\CortexM3\ARM_GCC_541\Debug\VCNL4030X01_PS.o
 .text.VCNL4030X01_SET_PS_SPO
                0x00000000       0x44 .\CortexM3\ARM_GCC_541\Debug\VCNL4030X01_PS.o
 .text.VCNL4030X01_SET_PS_CANC
                0x00000000       0x34 .\CortexM3\ARM_GCC_541\Debug\VCNL4030X01_PS.o
 .text.VCNL4030X01_SET_PS_LowThreshold
                0x00000000       0x34 .\CortexM3\ARM_GCC_541\Debug\VCNL4030X01_PS.o
 .text.VCNL4030X01_SET_PS_HighThreshold
                0x00000000       0x34 .\CortexM3\ARM_GCC_541\Debug\VCNL4030X01_PS.o
 .text.VCNL4030X01_GET_PS_Data
                0x00000000       0x34 .\CortexM3\ARM_GCC_541\Debug\VCNL4030X01_PS.o
 .text.VCNL4030X01_GET_ID
                0x00000000       0x34 .\CortexM3\ARM_GCC_541\Debug\VCNL4030X01_PS.o
 .text          0x00000000        0x0 .\CortexM3\ARM_GCC_541\Debug\VCNL4030X01_ALS.o
 .data          0x00000000        0x0 .\CortexM3\ARM_GCC_541\Debug\VCNL4030X01_ALS.o
 .bss           0x00000000        0x0 .\CortexM3\ARM_GCC_541\Debug\VCNL4030X01_ALS.o
 .text.VCNL4030X01_SET_ALS_SD
                0x00000000       0x44 .\CortexM3\ARM_GCC_541\Debug\VCNL4030X01_ALS.o
 .text.VCNL4030X01_SET_ALS_IT
                0x00000000       0x44 .\CortexM3\ARM_GCC_541\Debug\VCNL4030X01_ALS.o
 .text.VCNL4030X01_SET_ALS_HD
                0x00000000       0x44 .\CortexM3\ARM_GCC_541\Debug\VCNL4030X01_ALS.o
 .text.VCNL4030X01_SET_ALS_PERS
                0x00000000       0x44 .\CortexM3\ARM_GCC_541\Debug\VCNL4030X01_ALS.o
 .text.VCNL4030X01_SET_ALS_Interrupt
                0x00000000       0x44 .\CortexM3\ARM_GCC_541\Debug\VCNL4030X01_ALS.o
 .text.VCNL4030X01_SET_ALS_NS
                0x00000000       0x44 .\CortexM3\ARM_GCC_541\Debug\VCNL4030X01_ALS.o
 .text.VCNL4030X01_SET_WHITE_SD
                0x00000000       0x44 .\CortexM3\ARM_GCC_541\Debug\VCNL4030X01_ALS.o
 .text.VCNL4030X01_SET_ALS_LowThreshold
                0x00000000       0x34 .\CortexM3\ARM_GCC_541\Debug\VCNL4030X01_ALS.o
 .text.VCNL4030X01_SET_ALS_HighThreshold
                0x00000000       0x34 .\CortexM3\ARM_GCC_541\Debug\VCNL4030X01_ALS.o
 .text          0x00000000        0x0 .\CortexM3\ARM_GCC_541\Debug\VCNL4030X01_Application_Library.o
 .data          0x00000000        0x0 .\CortexM3\ARM_GCC_541\Debug\VCNL4030X01_Application_Library.o
 .bss           0x00000000        0x0 .\CortexM3\ARM_GCC_541\Debug\VCNL4030X01_Application_Library.o
 .text.Print_Variable_DEC
                0x00000000       0x94 .\CortexM3\ARM_GCC_541\Debug\VCNL4030X01_Application_Library.o
 .text.Print_Variable_HEX
                0x00000000       0x94 .\CortexM3\ARM_GCC_541\Debug\VCNL4030X01_Application_Library.o
 .text.Print_All
                0x00000000      0x59c .\CortexM3\ARM_GCC_541\Debug\VCNL4030X01_Application_Library.o
 .text          0x00000000        0x0 .\CortexM3\ARM_GCC_541\Debug\cyfitter_cfg.o
 .data          0x00000000        0x0 .\CortexM3\ARM_GCC_541\Debug\cyfitter_cfg.o
 .bss           0x00000000        0x0 .\CortexM3\ARM_GCC_541\Debug\cyfitter_cfg.o
 .text.SetAnalogRoutingPumps
                0x00000000       0x10 .\CortexM3\ARM_GCC_541\Debug\cyfitter_cfg.o
 .text          0x00000000        0x0 .\CortexM3\ARM_GCC_541\Debug\cymetadata.o
 .data          0x00000000        0x0 .\CortexM3\ARM_GCC_541\Debug\cymetadata.o
 .bss           0x00000000        0x0 .\CortexM3\ARM_GCC_541\Debug\cymetadata.o
 .text          0x00000000        0x0 .\CortexM3\ARM_GCC_541\Debug\Cm3Start.o
 .bss           0x00000000        0x0 .\CortexM3\ARM_GCC_541\Debug\Cm3Start.o
 .text._exit    0x00000000        0xc .\CortexM3\ARM_GCC_541\Debug\Cm3Start.o
 .text          0x00000000        0x0 .\CortexM3\ARM_GCC_541\Debug\VCNL4030X01.a(I2C_1.o)
 .data          0x00000000        0x0 .\CortexM3\ARM_GCC_541\Debug\VCNL4030X01.a(I2C_1.o)
 .text.I2C_1_Stop
                0x00000000       0xb4 .\CortexM3\ARM_GCC_541\Debug\VCNL4030X01.a(I2C_1.o)
 .text          0x00000000        0x0 .\CortexM3\ARM_GCC_541\Debug\VCNL4030X01.a(I2C_1_INT.o)
 .data          0x00000000        0x0 .\CortexM3\ARM_GCC_541\Debug\VCNL4030X01.a(I2C_1_INT.o)
 .bss           0x00000000        0x0 .\CortexM3\ARM_GCC_541\Debug\VCNL4030X01.a(I2C_1_INT.o)
 .text          0x00000000        0x0 .\CortexM3\ARM_GCC_541\Debug\VCNL4030X01.a(I2C_1_PM.o)
 .data          0x00000000        0x6 .\CortexM3\ARM_GCC_541\Debug\VCNL4030X01.a(I2C_1_PM.o)
 .bss           0x00000000        0x0 .\CortexM3\ARM_GCC_541\Debug\VCNL4030X01.a(I2C_1_PM.o)
 .text.I2C_1_SaveConfig
                0x00000000       0x3c .\CortexM3\ARM_GCC_541\Debug\VCNL4030X01.a(I2C_1_PM.o)
 .text.I2C_1_Sleep
                0x00000000       0x24 .\CortexM3\ARM_GCC_541\Debug\VCNL4030X01.a(I2C_1_PM.o)
 .text.I2C_1_RestoreConfig
                0x00000000       0x60 .\CortexM3\ARM_GCC_541\Debug\VCNL4030X01.a(I2C_1_PM.o)
 .text.I2C_1_Wakeup
                0x00000000       0x24 .\CortexM3\ARM_GCC_541\Debug\VCNL4030X01.a(I2C_1_PM.o)
 .text          0x00000000        0x0 .\CortexM3\ARM_GCC_541\Debug\VCNL4030X01.a(I2C_1_MASTER.o)
 .data          0x00000000        0x0 .\CortexM3\ARM_GCC_541\Debug\VCNL4030X01.a(I2C_1_MASTER.o)
 .bss           0x00000000        0x0 .\CortexM3\ARM_GCC_541\Debug\VCNL4030X01.a(I2C_1_MASTER.o)
 .text.I2C_1_MasterWriteBuf
                0x00000000       0xcc .\CortexM3\ARM_GCC_541\Debug\VCNL4030X01.a(I2C_1_MASTER.o)
 .text.I2C_1_MasterReadBuf
                0x00000000       0xd0 .\CortexM3\ARM_GCC_541\Debug\VCNL4030X01.a(I2C_1_MASTER.o)
 .text.I2C_1_MasterClearStatus
                0x00000000       0x24 .\CortexM3\ARM_GCC_541\Debug\VCNL4030X01.a(I2C_1_MASTER.o)
 .text.I2C_1_MasterGetReadBufSize
                0x00000000        0xc .\CortexM3\ARM_GCC_541\Debug\VCNL4030X01.a(I2C_1_MASTER.o)
 .text.I2C_1_MasterGetWriteBufSize
                0x00000000        0xc .\CortexM3\ARM_GCC_541\Debug\VCNL4030X01.a(I2C_1_MASTER.o)
 .text          0x00000000        0x0 .\CortexM3\ARM_GCC_541\Debug\VCNL4030X01.a(CDC.o)
 .data          0x00000000        0x0 .\CortexM3\ARM_GCC_541\Debug\VCNL4030X01.a(CDC.o)
 .text.CDC_Stop
                0x00000000       0xb8 .\CortexM3\ARM_GCC_541\Debug\VCNL4030X01.a(CDC.o)
 .text.CDC_CheckActivity
                0x00000000       0x20 .\CortexM3\ARM_GCC_541\Debug\VCNL4030X01.a(CDC.o)
 .text.CDC_GetConfiguration
                0x00000000        0xc .\CortexM3\ARM_GCC_541\Debug\VCNL4030X01.a(CDC.o)
 .text.CDC_IsConfigurationChanged
                0x00000000       0x20 .\CortexM3\ARM_GCC_541\Debug\VCNL4030X01.a(CDC.o)
 .text.CDC_GetInterfaceSetting
                0x00000000        0xc .\CortexM3\ARM_GCC_541\Debug\VCNL4030X01.a(CDC.o)
 .text.CDC_GetEPCount
                0x00000000       0x28 .\CortexM3\ARM_GCC_541\Debug\VCNL4030X01.a(CDC.o)
 .text.CDC_ReadOutEP
                0x00000000       0x50 .\CortexM3\ARM_GCC_541\Debug\VCNL4030X01.a(CDC.o)
 .text.CDC_DisableOutEP
                0x00000000       0x18 .\CortexM3\ARM_GCC_541\Debug\VCNL4030X01.a(CDC.o)
 .text.CDC_Force
                0x00000000        0xc .\CortexM3\ARM_GCC_541\Debug\VCNL4030X01.a(CDC.o)
 .text.CDC_GetEPAckState
                0x00000000       0x20 .\CortexM3\ARM_GCC_541\Debug\VCNL4030X01.a(CDC.o)
 .text.CDC_SetPowerStatus
                0x00000000       0x20 .\CortexM3\ARM_GCC_541\Debug\VCNL4030X01.a(CDC.o)
 .text.CDC_RWUEnabled
                0x00000000       0x18 .\CortexM3\ARM_GCC_541\Debug\VCNL4030X01.a(CDC.o)
 .text.CDC_GetDeviceAddress
                0x00000000       0x10 .\CortexM3\ARM_GCC_541\Debug\VCNL4030X01.a(CDC.o)
 .text.CDC_EnableSofInt
                0x00000000       0x10 .\CortexM3\ARM_GCC_541\Debug\VCNL4030X01.a(CDC.o)
 .text.CDC_DisableSofInt
                0x00000000       0x10 .\CortexM3\ARM_GCC_541\Debug\VCNL4030X01.a(CDC.o)
 .text          0x00000000        0x0 .\CortexM3\ARM_GCC_541\Debug\VCNL4030X01.a(CDC_cdc.o)
 .text.CDC_PutData
                0x00000000       0x50 .\CortexM3\ARM_GCC_541\Debug\VCNL4030X01.a(CDC_cdc.o)
 .text.CDC_PutChar
                0x00000000       0x28 .\CortexM3\ARM_GCC_541\Debug\VCNL4030X01.a(CDC_cdc.o)
 .text.CDC_PutCRLF
                0x00000000       0x30 .\CortexM3\ARM_GCC_541\Debug\VCNL4030X01.a(CDC_cdc.o)
 .text.CDC_GetCount
                0x00000000       0x34 .\CortexM3\ARM_GCC_541\Debug\VCNL4030X01.a(CDC_cdc.o)
 .text.CDC_DataIsReady
                0x00000000       0x18 .\CortexM3\ARM_GCC_541\Debug\VCNL4030X01.a(CDC_cdc.o)
 .text.CDC_GetData
                0x00000000       0x20 .\CortexM3\ARM_GCC_541\Debug\VCNL4030X01.a(CDC_cdc.o)
 .text.CDC_GetAll
                0x00000000       0x30 .\CortexM3\ARM_GCC_541\Debug\VCNL4030X01.a(CDC_cdc.o)
 .text.CDC_GetChar
                0x00000000       0x28 .\CortexM3\ARM_GCC_541\Debug\VCNL4030X01.a(CDC_cdc.o)
 .text.CDC_IsLineChanged
                0x00000000       0x38 .\CortexM3\ARM_GCC_541\Debug\VCNL4030X01.a(CDC_cdc.o)
 .text.CDC_GetDTERate
                0x00000000       0x30 .\CortexM3\ARM_GCC_541\Debug\VCNL4030X01.a(CDC_cdc.o)
 .text.CDC_GetCharFormat
                0x00000000       0x18 .\CortexM3\ARM_GCC_541\Debug\VCNL4030X01.a(CDC_cdc.o)
 .text.CDC_GetParityType
                0x00000000       0x18 .\CortexM3\ARM_GCC_541\Debug\VCNL4030X01.a(CDC_cdc.o)
 .text.CDC_GetDataBits
                0x00000000       0x18 .\CortexM3\ARM_GCC_541\Debug\VCNL4030X01.a(CDC_cdc.o)
 .text.CDC_GetLineControl
                0x00000000       0x18 .\CortexM3\ARM_GCC_541\Debug\VCNL4030X01.a(CDC_cdc.o)
 .text.CDC_SendSerialState
                0x00000000       0x64 .\CortexM3\ARM_GCC_541\Debug\VCNL4030X01.a(CDC_cdc.o)
 .text.CDC_GetSerialState
                0x00000000       0x18 .\CortexM3\ARM_GCC_541\Debug\VCNL4030X01.a(CDC_cdc.o)
 .text.CDC_NotificationIsReady
                0x00000000       0x24 .\CortexM3\ARM_GCC_541\Debug\VCNL4030X01.a(CDC_cdc.o)
 .text.CDC_SetComPort
                0x00000000       0x18 .\CortexM3\ARM_GCC_541\Debug\VCNL4030X01.a(CDC_cdc.o)
 .text.CDC_GetComPort
                0x00000000        0xc .\CortexM3\ARM_GCC_541\Debug\VCNL4030X01.a(CDC_cdc.o)
 .rodata        0x00000000        0x2 .\CortexM3\ARM_GCC_541\Debug\VCNL4030X01.a(CDC_cdc.o)
 .text          0x00000000        0x0 .\CortexM3\ARM_GCC_541\Debug\VCNL4030X01.a(CDC_drv.o)
 .data          0x00000000        0x0 .\CortexM3\ARM_GCC_541\Debug\VCNL4030X01.a(CDC_drv.o)
 .bss           0x00000000        0x0 .\CortexM3\ARM_GCC_541\Debug\VCNL4030X01.a(CDC_drv.o)
 .text          0x00000000        0x0 .\CortexM3\ARM_GCC_541\Debug\VCNL4030X01.a(CDC_episr.o)
 .data          0x00000000        0x0 .\CortexM3\ARM_GCC_541\Debug\VCNL4030X01.a(CDC_episr.o)
 .bss           0x00000000        0x0 .\CortexM3\ARM_GCC_541\Debug\VCNL4030X01.a(CDC_episr.o)
 .text          0x00000000        0x0 .\CortexM3\ARM_GCC_541\Debug\VCNL4030X01.a(CDC_pm.o)
 .data          0x00000000        0x0 .\CortexM3\ARM_GCC_541\Debug\VCNL4030X01.a(CDC_pm.o)
 .bss           0x00000000        0x2 .\CortexM3\ARM_GCC_541\Debug\VCNL4030X01.a(CDC_pm.o)
 .text.CDC_SaveConfig
                0x00000000        0x4 .\CortexM3\ARM_GCC_541\Debug\VCNL4030X01.a(CDC_pm.o)
 .text.CDC_RestoreConfig
                0x00000000       0x1c .\CortexM3\ARM_GCC_541\Debug\VCNL4030X01.a(CDC_pm.o)
 .text.CDC_Suspend
                0x00000000       0xc8 .\CortexM3\ARM_GCC_541\Debug\VCNL4030X01.a(CDC_pm.o)
 .text.CDC_Resume
                0x00000000       0xbc .\CortexM3\ARM_GCC_541\Debug\VCNL4030X01.a(CDC_pm.o)
 .text          0x00000000        0x0 .\CortexM3\ARM_GCC_541\Debug\VCNL4030X01.a(CDC_std.o)
 .data          0x00000000        0x0 .\CortexM3\ARM_GCC_541\Debug\VCNL4030X01.a(CDC_std.o)
 .text.CDC_EpStateInit
                0x00000000       0x44 .\CortexM3\ARM_GCC_541\Debug\VCNL4030X01.a(CDC_std.o)
 .text.CDC_TerminateEP
                0x00000000       0x4c .\CortexM3\ARM_GCC_541\Debug\VCNL4030X01.a(CDC_std.o)
 .text          0x00000000        0x0 .\CortexM3\ARM_GCC_541\Debug\VCNL4030X01.a(CDC_vnd.o)
 .data          0x00000000        0x0 .\CortexM3\ARM_GCC_541\Debug\VCNL4030X01.a(CDC_vnd.o)
 .bss           0x00000000        0x0 .\CortexM3\ARM_GCC_541\Debug\VCNL4030X01.a(CDC_vnd.o)
 .text          0x00000000        0x0 .\CortexM3\ARM_GCC_541\Debug\VCNL4030X01.a(CDC_Dp.o)
 .data          0x00000000        0x0 .\CortexM3\ARM_GCC_541\Debug\VCNL4030X01.a(CDC_Dp.o)
 .bss           0x00000000        0x0 .\CortexM3\ARM_GCC_541\Debug\VCNL4030X01.a(CDC_Dp.o)
 .text.CDC_Dp_Write
                0x00000000       0x18 .\CortexM3\ARM_GCC_541\Debug\VCNL4030X01.a(CDC_Dp.o)
 .text.CDC_Dp_SetDriveMode
                0x00000000       0x18 .\CortexM3\ARM_GCC_541\Debug\VCNL4030X01.a(CDC_Dp.o)
 .text.CDC_Dp_Read
                0x00000000       0x10 .\CortexM3\ARM_GCC_541\Debug\VCNL4030X01.a(CDC_Dp.o)
 .text.CDC_Dp_ReadDataReg
                0x00000000       0x10 .\CortexM3\ARM_GCC_541\Debug\VCNL4030X01.a(CDC_Dp.o)
 .text.CDC_Dp_SetInterruptMode
                0x00000000       0x14 .\CortexM3\ARM_GCC_541\Debug\VCNL4030X01.a(CDC_Dp.o)
 .text          0x00000000        0x0 .\CortexM3\ARM_GCC_541\Debug\VCNL4030X01.a(CyLib.o)
 .bss           0x00000000       0x1c .\CortexM3\ARM_GCC_541\Debug\VCNL4030X01.a(CyLib.o)
 .text.CyUSB_PowerOnCheck
                0x00000000       0x48 .\CortexM3\ARM_GCC_541\Debug\VCNL4030X01.a(CyLib.o)
 .text.CyBusClk_Internal_SetDivider
                0x00000000       0x48 .\CortexM3\ARM_GCC_541\Debug\VCNL4030X01.a(CyLib.o)
 .text.CyPLL_OUT_Stop
                0x00000000       0x10 .\CortexM3\ARM_GCC_541\Debug\VCNL4030X01.a(CyLib.o)
 .text.CyIMO_Stop
                0x00000000       0x1c .\CortexM3\ARM_GCC_541\Debug\VCNL4030X01.a(CyLib.o)
 .text.CyIMO_EnableDoubler
                0x00000000       0x10 .\CortexM3\ARM_GCC_541\Debug\VCNL4030X01.a(CyLib.o)
 .text.CyIMO_DisableDoubler
                0x00000000       0x10 .\CortexM3\ARM_GCC_541\Debug\VCNL4030X01.a(CyLib.o)
 .text.CyMasterClk_SetSource
                0x00000000       0x18 .\CortexM3\ARM_GCC_541\Debug\VCNL4030X01.a(CyLib.o)
 .text.CyMasterClk_SetDivider
                0x00000000        0xc .\CortexM3\ARM_GCC_541\Debug\VCNL4030X01.a(CyLib.o)
 .text.CyBusClk_SetDivider
                0x00000000       0x70 .\CortexM3\ARM_GCC_541\Debug\VCNL4030X01.a(CyLib.o)
 .text.CyUsbClk_SetSource
                0x00000000       0x18 .\CortexM3\ARM_GCC_541\Debug\VCNL4030X01.a(CyLib.o)
 .text.CyILO_Start1K
                0x00000000       0x10 .\CortexM3\ARM_GCC_541\Debug\VCNL4030X01.a(CyLib.o)
 .text.CyILO_Stop1K
                0x00000000       0x10 .\CortexM3\ARM_GCC_541\Debug\VCNL4030X01.a(CyLib.o)
 .text.CyILO_Start100K
                0x00000000       0x10 .\CortexM3\ARM_GCC_541\Debug\VCNL4030X01.a(CyLib.o)
 .text.CyILO_Stop100K
                0x00000000       0x10 .\CortexM3\ARM_GCC_541\Debug\VCNL4030X01.a(CyLib.o)
 .text.CyPLL_OUT_Start
                0x00000000       0x78 .\CortexM3\ARM_GCC_541\Debug\VCNL4030X01.a(CyLib.o)
 .text.CyIMO_Start
                0x00000000       0x60 .\CortexM3\ARM_GCC_541\Debug\VCNL4030X01.a(CyLib.o)
 .text.CyILO_Enable33K
                0x00000000       0x10 .\CortexM3\ARM_GCC_541\Debug\VCNL4030X01.a(CyLib.o)
 .text.CyILO_Disable33K
                0x00000000       0x10 .\CortexM3\ARM_GCC_541\Debug\VCNL4030X01.a(CyLib.o)
 .text.CyILO_SetSource
                0x00000000       0x18 .\CortexM3\ARM_GCC_541\Debug\VCNL4030X01.a(CyLib.o)
 .text.CyILO_SetPowerMode
                0x00000000       0x24 .\CortexM3\ARM_GCC_541\Debug\VCNL4030X01.a(CyLib.o)
 .text.CyXTAL_32KHZ_Stop
                0x00000000       0x30 .\CortexM3\ARM_GCC_541\Debug\VCNL4030X01.a(CyLib.o)
 .text.CyXTAL_32KHZ_ReadStatus
                0x00000000       0x10 .\CortexM3\ARM_GCC_541\Debug\VCNL4030X01.a(CyLib.o)
 .text.CyXTAL_Start
                0x00000000       0xac .\CortexM3\ARM_GCC_541\Debug\VCNL4030X01.a(CyLib.o)
 .text.CyXTAL_Stop
                0x00000000       0x10 .\CortexM3\ARM_GCC_541\Debug\VCNL4030X01.a(CyLib.o)
 .text.CyXTAL_EnableErrStatus
                0x00000000       0x10 .\CortexM3\ARM_GCC_541\Debug\VCNL4030X01.a(CyLib.o)
 .text.CyXTAL_DisableErrStatus
                0x00000000       0x10 .\CortexM3\ARM_GCC_541\Debug\VCNL4030X01.a(CyLib.o)
 .text.CyXTAL_ReadStatus
                0x00000000       0x18 .\CortexM3\ARM_GCC_541\Debug\VCNL4030X01.a(CyLib.o)
 .text.CyXTAL_EnableFaultRecovery
                0x00000000       0x10 .\CortexM3\ARM_GCC_541\Debug\VCNL4030X01.a(CyLib.o)
 .text.CyXTAL_DisableFaultRecovery
                0x00000000       0x10 .\CortexM3\ARM_GCC_541\Debug\VCNL4030X01.a(CyLib.o)
 .text.CyXTAL_SetStartup
                0x00000000       0x18 .\CortexM3\ARM_GCC_541\Debug\VCNL4030X01.a(CyLib.o)
 .text.CyXTAL_SetFbVoltage
                0x00000000       0x18 .\CortexM3\ARM_GCC_541\Debug\VCNL4030X01.a(CyLib.o)
 .text.CyXTAL_SetWdVoltage
                0x00000000       0x18 .\CortexM3\ARM_GCC_541\Debug\VCNL4030X01.a(CyLib.o)
 .text.CyPLL_OUT_SetPQ
                0x00000000       0x60 .\CortexM3\ARM_GCC_541\Debug\VCNL4030X01.a(CyLib.o)
 .text.CyPLL_OUT_SetSource
                0x00000000       0x34 .\CortexM3\ARM_GCC_541\Debug\VCNL4030X01.a(CyLib.o)
 .text.CyIMO_SetTrimValue
                0x00000000       0xcc .\CortexM3\ARM_GCC_541\Debug\VCNL4030X01.a(CyLib.o)
 .text.CyIMO_SetFreq
                0x00000000       0xf4 .\CortexM3\ARM_GCC_541\Debug\VCNL4030X01.a(CyLib.o)
 .text.CyIMO_SetSource
                0x00000000       0x58 .\CortexM3\ARM_GCC_541\Debug\VCNL4030X01.a(CyLib.o)
 .text.CySoftwareReset
                0x00000000       0x10 .\CortexM3\ARM_GCC_541\Debug\VCNL4030X01.a(CyLib.o)
 .text.CyXTAL_32KHZ_SetPowerMode
                0x00000000       0x84 .\CortexM3\ARM_GCC_541\Debug\VCNL4030X01.a(CyLib.o)
 .text.CyXTAL_32KHZ_Start
                0x00000000       0x74 .\CortexM3\ARM_GCC_541\Debug\VCNL4030X01.a(CyLib.o)
 .text.CyDelayFreq
                0x00000000       0x4c .\CortexM3\ARM_GCC_541\Debug\VCNL4030X01.a(CyLib.o)
 .text.CyWdtStart
                0x00000000       0x40 .\CortexM3\ARM_GCC_541\Debug\VCNL4030X01.a(CyLib.o)
 .text.CyWdtClear
                0x00000000        0xc .\CortexM3\ARM_GCC_541\Debug\VCNL4030X01.a(CyLib.o)
 .text.CyVdStickyStatus
                0x00000000       0x2c .\CortexM3\ARM_GCC_541\Debug\VCNL4030X01.a(CyLib.o)
 .text.CyVdLvDigitEnable
                0x00000000       0x84 .\CortexM3\ARM_GCC_541\Debug\VCNL4030X01.a(CyLib.o)
 .text.CyVdLvAnalogEnable
                0x00000000       0x80 .\CortexM3\ARM_GCC_541\Debug\VCNL4030X01.a(CyLib.o)
 .text.CyVdLvDigitDisable
                0x00000000       0x30 .\CortexM3\ARM_GCC_541\Debug\VCNL4030X01.a(CyLib.o)
 .text.CyVdLvAnalogDisable
                0x00000000       0x28 .\CortexM3\ARM_GCC_541\Debug\VCNL4030X01.a(CyLib.o)
 .text.CyVdHvAnalogEnable
                0x00000000       0x54 .\CortexM3\ARM_GCC_541\Debug\VCNL4030X01.a(CyLib.o)
 .text.CyVdHvAnalogDisable
                0x00000000       0x20 .\CortexM3\ARM_GCC_541\Debug\VCNL4030X01.a(CyLib.o)
 .text.CyVdRealTimeStatus
                0x00000000       0x1c .\CortexM3\ARM_GCC_541\Debug\VCNL4030X01.a(CyLib.o)
 .text.CyDisableInts
                0x00000000       0x1c .\CortexM3\ARM_GCC_541\Debug\VCNL4030X01.a(CyLib.o)
 .text.CyEnableInts
                0x00000000       0x18 .\CortexM3\ARM_GCC_541\Debug\VCNL4030X01.a(CyLib.o)
 .text.CyFlushCache
                0x00000000       0x44 .\CortexM3\ARM_GCC_541\Debug\VCNL4030X01.a(CyLib.o)
 .text.CyIntSetSysVector
                0x00000000       0x28 .\CortexM3\ARM_GCC_541\Debug\VCNL4030X01.a(CyLib.o)
 .text.CyIntGetSysVector
                0x00000000       0x20 .\CortexM3\ARM_GCC_541\Debug\VCNL4030X01.a(CyLib.o)
 .text.CyIntGetVector
                0x00000000       0x24 .\CortexM3\ARM_GCC_541\Debug\VCNL4030X01.a(CyLib.o)
 .text.CyIntGetPriority
                0x00000000       0x20 .\CortexM3\ARM_GCC_541\Debug\VCNL4030X01.a(CyLib.o)
 .text.CyIntGetState
                0x00000000       0x24 .\CortexM3\ARM_GCC_541\Debug\VCNL4030X01.a(CyLib.o)
 .text.CySysTickStop
                0x00000000       0x10 .\CortexM3\ARM_GCC_541\Debug\VCNL4030X01.a(CyLib.o)
 .text.CySysTickEnableInterrupt
                0x00000000       0x10 .\CortexM3\ARM_GCC_541\Debug\VCNL4030X01.a(CyLib.o)
 .text.CySysTickEnable
                0x00000000       0x18 .\CortexM3\ARM_GCC_541\Debug\VCNL4030X01.a(CyLib.o)
 .text.CySysTickDisableInterrupt
                0x00000000       0x10 .\CortexM3\ARM_GCC_541\Debug\VCNL4030X01.a(CyLib.o)
 .text.CySysTickSetReload
                0x00000000       0x10 .\CortexM3\ARM_GCC_541\Debug\VCNL4030X01.a(CyLib.o)
 .text.CySysTickGetReload
                0x00000000       0x10 .\CortexM3\ARM_GCC_541\Debug\VCNL4030X01.a(CyLib.o)
 .text.CySysTickGetValue
                0x00000000       0x10 .\CortexM3\ARM_GCC_541\Debug\VCNL4030X01.a(CyLib.o)
 .text.CySysTickSetClockSource
                0x00000000       0x20 .\CortexM3\ARM_GCC_541\Debug\VCNL4030X01.a(CyLib.o)
 .text.CySysTickGetClockSource
                0x00000000       0x10 .\CortexM3\ARM_GCC_541\Debug\VCNL4030X01.a(CyLib.o)
 .text.CySysTickGetCountFlag
                0x00000000       0x10 .\CortexM3\ARM_GCC_541\Debug\VCNL4030X01.a(CyLib.o)
 .text.CySysTickServiceCallbacks
                0x00000000       0x28 .\CortexM3\ARM_GCC_541\Debug\VCNL4030X01.a(CyLib.o)
 .text.CySysTickClear
                0x00000000        0xc .\CortexM3\ARM_GCC_541\Debug\VCNL4030X01.a(CyLib.o)
 .text.CySysTickInit
                0x00000000       0x58 .\CortexM3\ARM_GCC_541\Debug\VCNL4030X01.a(CyLib.o)
 .text.CySysTickStart
                0x00000000       0x1c .\CortexM3\ARM_GCC_541\Debug\VCNL4030X01.a(CyLib.o)
 .text.CySysTickSetCallback
                0x00000000       0x10 .\CortexM3\ARM_GCC_541\Debug\VCNL4030X01.a(CyLib.o)
 .text.CySysTickGetCallback
                0x00000000       0x10 .\CortexM3\ARM_GCC_541\Debug\VCNL4030X01.a(CyLib.o)
 .text          0x00000000        0x0 .\CortexM3\ARM_GCC_541\Debug\VCNL4030X01.a(cyPm.o)
 .data          0x00000000        0x0 .\CortexM3\ARM_GCC_541\Debug\VCNL4030X01.a(cyPm.o)
 .bss           0x00000000       0x43 .\CortexM3\ARM_GCC_541\Debug\VCNL4030X01.a(cyPm.o)
 .text.CyPmHibSlpSaveSet
                0x00000000      0x1dc .\CortexM3\ARM_GCC_541\Debug\VCNL4030X01.a(cyPm.o)
 .text.CyPmHibSlpRestore
                0x00000000       0xd8 .\CortexM3\ARM_GCC_541\Debug\VCNL4030X01.a(cyPm.o)
 .text.CyPmHviLviSaveDisable
                0x00000000       0xa0 .\CortexM3\ARM_GCC_541\Debug\VCNL4030X01.a(cyPm.o)
 .text.CyPmHibSaveSet
                0x00000000       0x98 .\CortexM3\ARM_GCC_541\Debug\VCNL4030X01.a(cyPm.o)
 .text.CyPmHviLviRestore
                0x00000000       0x48 .\CortexM3\ARM_GCC_541\Debug\VCNL4030X01.a(cyPm.o)
 .text.CyPmHibRestore
                0x00000000       0x60 .\CortexM3\ARM_GCC_541\Debug\VCNL4030X01.a(cyPm.o)
 .text.CyPmSaveClocks
                0x00000000      0x218 .\CortexM3\ARM_GCC_541\Debug\VCNL4030X01.a(cyPm.o)
 .text.CyPmRestoreClocks
                0x00000000      0x24c .\CortexM3\ARM_GCC_541\Debug\VCNL4030X01.a(cyPm.o)
 .text.CyPmAltAct
                0x00000000       0x6c .\CortexM3\ARM_GCC_541\Debug\VCNL4030X01.a(cyPm.o)
 .text.CyPmSleep
                0x00000000       0xf4 .\CortexM3\ARM_GCC_541\Debug\VCNL4030X01.a(cyPm.o)
 .text.CyPmHibernateEx
                0x00000000       0xf4 .\CortexM3\ARM_GCC_541\Debug\VCNL4030X01.a(cyPm.o)
 .text.CyPmHibernate
                0x00000000        0xc .\CortexM3\ARM_GCC_541\Debug\VCNL4030X01.a(cyPm.o)
 .text.CyPmReadStatus
                0x00000000       0x30 .\CortexM3\ARM_GCC_541\Debug\VCNL4030X01.a(cyPm.o)
 .text.CyPmCtwSetInterval
                0x00000000       0x5c .\CortexM3\ARM_GCC_541\Debug\VCNL4030X01.a(cyPm.o)
 .text.CyPmOppsSet
                0x00000000       0x2c .\CortexM3\ARM_GCC_541\Debug\VCNL4030X01.a(cyPm.o)
 .text.CyPmFtwSetInterval
                0x00000000       0x5c .\CortexM3\ARM_GCC_541\Debug\VCNL4030X01.a(cyPm.o)
 .rodata        0x00000000        0xf .\CortexM3\ARM_GCC_541\Debug\VCNL4030X01.a(cyPm.o)
 .data          0x00000000        0x0 .\CortexM3\ARM_GCC_541\Debug\VCNL4030X01.a(CyBootAsmGnu.o)
 .bss           0x00000000        0x0 .\CortexM3\ARM_GCC_541\Debug\VCNL4030X01.a(CyBootAsmGnu.o)
 .text          0x00000000        0x0 .\CortexM3\ARM_GCC_541\Debug\VCNL4030X01.a(CDC_cls.o)
 .data          0x00000000        0x0 .\CortexM3\ARM_GCC_541\Debug\VCNL4030X01.a(CDC_cls.o)
 .bss           0x00000000        0x0 .\CortexM3\ARM_GCC_541\Debug\VCNL4030X01.a(CDC_cls.o)
 .text          0x00000000        0x0 .\CortexM3\ARM_GCC_541\Debug\VCNL4030X01.a(CDC_descr.o)
 .data          0x00000000        0x0 .\CortexM3\ARM_GCC_541\Debug\VCNL4030X01.a(CDC_descr.o)
 .bss           0x00000000        0x0 .\CortexM3\ARM_GCC_541\Debug\VCNL4030X01.a(CDC_descr.o)
 .text          0x00000000        0x0 .\CortexM3\ARM_GCC_541\Debug\VCNL4030X01.a(CyFlash.o)
 .data          0x00000000        0x0 .\CortexM3\ARM_GCC_541\Debug\VCNL4030X01.a(CyFlash.o)
 .bss           0x00000000        0x0 .\CortexM3\ARM_GCC_541\Debug\VCNL4030X01.a(CyFlash.o)
 .text.CySetTempInt
                0x00000000       0x60 .\CortexM3\ARM_GCC_541\Debug\VCNL4030X01.a(CyFlash.o)
 .text.CyFlash_Start
                0x00000000       0x54 .\CortexM3\ARM_GCC_541\Debug\VCNL4030X01.a(CyFlash.o)
 .text.CyFlash_Stop
                0x00000000       0x24 .\CortexM3\ARM_GCC_541\Debug\VCNL4030X01.a(CyFlash.o)
 .text.CyFlash_EraseRow
                0x00000000       0x78 .\CortexM3\ARM_GCC_541\Debug\VCNL4030X01.a(CyFlash.o)
 .text.CyFlashGetSpcAlgorithm
                0x00000000       0x4c .\CortexM3\ARM_GCC_541\Debug\VCNL4030X01.a(CyFlash.o)
 .text.CySetTemp
                0x00000000       0x14 .\CortexM3\ARM_GCC_541\Debug\VCNL4030X01.a(CyFlash.o)
 .text.CySetFlashEEBuffer
                0x00000000       0x20 .\CortexM3\ARM_GCC_541\Debug\VCNL4030X01.a(CyFlash.o)
 .text.CyWriteRowFull
                0x00000000       0xf8 .\CortexM3\ARM_GCC_541\Debug\VCNL4030X01.a(CyFlash.o)
 .text.CyWriteRowData
                0x00000000       0x14 .\CortexM3\ARM_GCC_541\Debug\VCNL4030X01.a(CyFlash.o)
 .text.CyFlash_SetWaitCycles
                0x00000000       0x7c .\CortexM3\ARM_GCC_541\Debug\VCNL4030X01.a(CyFlash.o)
 .text.CyEEPROM_Start
                0x00000000       0x54 .\CortexM3\ARM_GCC_541\Debug\VCNL4030X01.a(CyFlash.o)
 .text.CyEEPROM_Stop
                0x00000000       0x24 .\CortexM3\ARM_GCC_541\Debug\VCNL4030X01.a(CyFlash.o)
 .text.CyEEPROM_ReadReserve
                0x00000000       0x1c .\CortexM3\ARM_GCC_541\Debug\VCNL4030X01.a(CyFlash.o)
 .text.CyEEPROM_ReadRelease
                0x00000000       0x10 .\CortexM3\ARM_GCC_541\Debug\VCNL4030X01.a(CyFlash.o)
 COMMON         0x00000000        0x2 .\CortexM3\ARM_GCC_541\Debug\VCNL4030X01.a(CyFlash.o)
 .text          0x00000000        0x0 .\CortexM3\ARM_GCC_541\Debug\VCNL4030X01.a(CySpc.o)
 .data          0x00000000        0x0 .\CortexM3\ARM_GCC_541\Debug\VCNL4030X01.a(CySpc.o)
 .bss           0x00000000        0x8 .\CortexM3\ARM_GCC_541\Debug\VCNL4030X01.a(CySpc.o)
 .text.CySpcStart
                0x00000000       0x24 .\CortexM3\ARM_GCC_541\Debug\VCNL4030X01.a(CySpc.o)
 .text.CySpcStop
                0x00000000       0x24 .\CortexM3\ARM_GCC_541\Debug\VCNL4030X01.a(CySpc.o)
 .text.CySpcReadData
                0x00000000       0x34 .\CortexM3\ARM_GCC_541\Debug\VCNL4030X01.a(CySpc.o)
 .text.CySpcLoadMultiByte
                0x00000000       0x78 .\CortexM3\ARM_GCC_541\Debug\VCNL4030X01.a(CySpc.o)
 .text.CySpcLoadRow
                0x00000000       0x50 .\CortexM3\ARM_GCC_541\Debug\VCNL4030X01.a(CySpc.o)
 .text.CySpcLoadRowFull
                0x00000000       0x80 .\CortexM3\ARM_GCC_541\Debug\VCNL4030X01.a(CySpc.o)
 .text.CySpcWriteRow
                0x00000000       0x4c .\CortexM3\ARM_GCC_541\Debug\VCNL4030X01.a(CySpc.o)
 .text.CySpcEraseSector
                0x00000000       0x3c .\CortexM3\ARM_GCC_541\Debug\VCNL4030X01.a(CySpc.o)
 .text.CySpcEraseRow
                0x00000000       0x4c .\CortexM3\ARM_GCC_541\Debug\VCNL4030X01.a(CySpc.o)
 .text.CySpcGetTemp
                0x00000000       0x3c .\CortexM3\ARM_GCC_541\Debug\VCNL4030X01.a(CySpc.o)
 .text.CySpcLock
                0x00000000       0x4c .\CortexM3\ARM_GCC_541\Debug\VCNL4030X01.a(CySpc.o)
 .text.CySpcUnlock
                0x00000000       0x38 .\CortexM3\ARM_GCC_541\Debug\VCNL4030X01.a(CySpc.o)
 .text.CySpcGetAlgorithm
                0x00000000       0x28 .\CortexM3\ARM_GCC_541\Debug\VCNL4030X01.a(CySpc.o)
 .text          0x00000000        0x0 c:/program files (x86)/cypress/psoc creator/4.3/psoc creator/import/gnu/arm/5.4.1/bin/../lib/gcc/arm-none-eabi/5.4.1/../../../../arm-none-eabi/lib/armv7-m\libm.a(lib_a-w_pow.o)
 .data          0x00000000        0x0 c:/program files (x86)/cypress/psoc creator/4.3/psoc creator/import/gnu/arm/5.4.1/bin/../lib/gcc/arm-none-eabi/5.4.1/../../../../arm-none-eabi/lib/armv7-m\libm.a(lib_a-w_pow.o)
 .bss           0x00000000        0x0 c:/program files (x86)/cypress/psoc creator/4.3/psoc creator/import/gnu/arm/5.4.1/bin/../lib/gcc/arm-none-eabi/5.4.1/../../../../arm-none-eabi/lib/armv7-m\libm.a(lib_a-w_pow.o)
 .text          0x00000000        0x0 c:/program files (x86)/cypress/psoc creator/4.3/psoc creator/import/gnu/arm/5.4.1/bin/../lib/gcc/arm-none-eabi/5.4.1/../../../../arm-none-eabi/lib/armv7-m\libm.a(lib_a-e_pow.o)
 .data          0x00000000        0x0 c:/program files (x86)/cypress/psoc creator/4.3/psoc creator/import/gnu/arm/5.4.1/bin/../lib/gcc/arm-none-eabi/5.4.1/../../../../arm-none-eabi/lib/armv7-m\libm.a(lib_a-e_pow.o)
 .bss           0x00000000        0x0 c:/program files (x86)/cypress/psoc creator/4.3/psoc creator/import/gnu/arm/5.4.1/bin/../lib/gcc/arm-none-eabi/5.4.1/../../../../arm-none-eabi/lib/armv7-m\libm.a(lib_a-e_pow.o)
 .text          0x00000000        0x0 c:/program files (x86)/cypress/psoc creator/4.3/psoc creator/import/gnu/arm/5.4.1/bin/../lib/gcc/arm-none-eabi/5.4.1/../../../../arm-none-eabi/lib/armv7-m\libm.a(lib_a-e_sqrt.o)
 .data          0x00000000        0x0 c:/program files (x86)/cypress/psoc creator/4.3/psoc creator/import/gnu/arm/5.4.1/bin/../lib/gcc/arm-none-eabi/5.4.1/../../../../arm-none-eabi/lib/armv7-m\libm.a(lib_a-e_sqrt.o)
 .bss           0x00000000        0x0 c:/program files (x86)/cypress/psoc creator/4.3/psoc creator/import/gnu/arm/5.4.1/bin/../lib/gcc/arm-none-eabi/5.4.1/../../../../arm-none-eabi/lib/armv7-m\libm.a(lib_a-e_sqrt.o)
 .text          0x00000000        0x0 c:/program files (x86)/cypress/psoc creator/4.3/psoc creator/import/gnu/arm/5.4.1/bin/../lib/gcc/arm-none-eabi/5.4.1/../../../../arm-none-eabi/lib/armv7-m\libm.a(lib_a-s_fabs.o)
 .data          0x00000000        0x0 c:/program files (x86)/cypress/psoc creator/4.3/psoc creator/import/gnu/arm/5.4.1/bin/../lib/gcc/arm-none-eabi/5.4.1/../../../../arm-none-eabi/lib/armv7-m\libm.a(lib_a-s_fabs.o)
 .bss           0x00000000        0x0 c:/program files (x86)/cypress/psoc creator/4.3/psoc creator/import/gnu/arm/5.4.1/bin/../lib/gcc/arm-none-eabi/5.4.1/../../../../arm-none-eabi/lib/armv7-m\libm.a(lib_a-s_fabs.o)
 .text          0x00000000        0x0 c:/program files (x86)/cypress/psoc creator/4.3/psoc creator/import/gnu/arm/5.4.1/bin/../lib/gcc/arm-none-eabi/5.4.1/../../../../arm-none-eabi/lib/armv7-m\libm.a(lib_a-s_finite.o)
 .data          0x00000000        0x0 c:/program files (x86)/cypress/psoc creator/4.3/psoc creator/import/gnu/arm/5.4.1/bin/../lib/gcc/arm-none-eabi/5.4.1/../../../../arm-none-eabi/lib/armv7-m\libm.a(lib_a-s_finite.o)
 .bss           0x00000000        0x0 c:/program files (x86)/cypress/psoc creator/4.3/psoc creator/import/gnu/arm/5.4.1/bin/../lib/gcc/arm-none-eabi/5.4.1/../../../../arm-none-eabi/lib/armv7-m\libm.a(lib_a-s_finite.o)
 .text          0x00000000        0x0 c:/program files (x86)/cypress/psoc creator/4.3/psoc creator/import/gnu/arm/5.4.1/bin/../lib/gcc/arm-none-eabi/5.4.1/../../../../arm-none-eabi/lib/armv7-m\libm.a(lib_a-s_lib_ver.o)
 .data          0x00000000        0x0 c:/program files (x86)/cypress/psoc creator/4.3/psoc creator/import/gnu/arm/5.4.1/bin/../lib/gcc/arm-none-eabi/5.4.1/../../../../arm-none-eabi/lib/armv7-m\libm.a(lib_a-s_lib_ver.o)
 .bss           0x00000000        0x0 c:/program files (x86)/cypress/psoc creator/4.3/psoc creator/import/gnu/arm/5.4.1/bin/../lib/gcc/arm-none-eabi/5.4.1/../../../../arm-none-eabi/lib/armv7-m\libm.a(lib_a-s_lib_ver.o)
 .text          0x00000000        0x0 c:/program files (x86)/cypress/psoc creator/4.3/psoc creator/import/gnu/arm/5.4.1/bin/../lib/gcc/arm-none-eabi/5.4.1/../../../../arm-none-eabi/lib/armv7-m\libm.a(lib_a-s_matherr.o)
 .data          0x00000000        0x0 c:/program files (x86)/cypress/psoc creator/4.3/psoc creator/import/gnu/arm/5.4.1/bin/../lib/gcc/arm-none-eabi/5.4.1/../../../../arm-none-eabi/lib/armv7-m\libm.a(lib_a-s_matherr.o)
 .bss           0x00000000        0x0 c:/program files (x86)/cypress/psoc creator/4.3/psoc creator/import/gnu/arm/5.4.1/bin/../lib/gcc/arm-none-eabi/5.4.1/../../../../arm-none-eabi/lib/armv7-m\libm.a(lib_a-s_matherr.o)
 .text          0x00000000        0x0 c:/program files (x86)/cypress/psoc creator/4.3/psoc creator/import/gnu/arm/5.4.1/bin/../lib/gcc/arm-none-eabi/5.4.1/../../../../arm-none-eabi/lib/armv7-m\libm.a(lib_a-s_nan.o)
 .data          0x00000000        0x0 c:/program files (x86)/cypress/psoc creator/4.3/psoc creator/import/gnu/arm/5.4.1/bin/../lib/gcc/arm-none-eabi/5.4.1/../../../../arm-none-eabi/lib/armv7-m\libm.a(lib_a-s_nan.o)
 .bss           0x00000000        0x0 c:/program files (x86)/cypress/psoc creator/4.3/psoc creator/import/gnu/arm/5.4.1/bin/../lib/gcc/arm-none-eabi/5.4.1/../../../../arm-none-eabi/lib/armv7-m\libm.a(lib_a-s_nan.o)
 .text          0x00000000        0x0 c:/program files (x86)/cypress/psoc creator/4.3/psoc creator/import/gnu/arm/5.4.1/bin/../lib/gcc/arm-none-eabi/5.4.1/../../../../arm-none-eabi/lib/armv7-m\libm.a(lib_a-s_rint.o)
 .data          0x00000000        0x0 c:/program files (x86)/cypress/psoc creator/4.3/psoc creator/import/gnu/arm/5.4.1/bin/../lib/gcc/arm-none-eabi/5.4.1/../../../../arm-none-eabi/lib/armv7-m\libm.a(lib_a-s_rint.o)
 .bss           0x00000000        0x0 c:/program files (x86)/cypress/psoc creator/4.3/psoc creator/import/gnu/arm/5.4.1/bin/../lib/gcc/arm-none-eabi/5.4.1/../../../../arm-none-eabi/lib/armv7-m\libm.a(lib_a-s_rint.o)
 .text          0x00000000        0x0 c:/program files (x86)/cypress/psoc creator/4.3/psoc creator/import/gnu/arm/5.4.1/bin/../lib/gcc/arm-none-eabi/5.4.1/../../../../arm-none-eabi/lib/armv7-m\libm.a(lib_a-s_scalbn.o)
 .data          0x00000000        0x0 c:/program files (x86)/cypress/psoc creator/4.3/psoc creator/import/gnu/arm/5.4.1/bin/../lib/gcc/arm-none-eabi/5.4.1/../../../../arm-none-eabi/lib/armv7-m\libm.a(lib_a-s_scalbn.o)
 .bss           0x00000000        0x0 c:/program files (x86)/cypress/psoc creator/4.3/psoc creator/import/gnu/arm/5.4.1/bin/../lib/gcc/arm-none-eabi/5.4.1/../../../../arm-none-eabi/lib/armv7-m\libm.a(lib_a-s_scalbn.o)
 .text          0x00000000        0x0 c:/program files (x86)/cypress/psoc creator/4.3/psoc creator/import/gnu/arm/5.4.1/bin/../lib/gcc/arm-none-eabi/5.4.1/../../../../arm-none-eabi/lib/armv7-m\libm.a(lib_a-s_copysign.o)
 .data          0x00000000        0x0 c:/program files (x86)/cypress/psoc creator/4.3/psoc creator/import/gnu/arm/5.4.1/bin/../lib/gcc/arm-none-eabi/5.4.1/../../../../arm-none-eabi/lib/armv7-m\libm.a(lib_a-s_copysign.o)
 .bss           0x00000000        0x0 c:/program files (x86)/cypress/psoc creator/4.3/psoc creator/import/gnu/arm/5.4.1/bin/../lib/gcc/arm-none-eabi/5.4.1/../../../../arm-none-eabi/lib/armv7-m\libm.a(lib_a-s_copysign.o)
 .data          0x00000000        0x0 c:/program files (x86)/cypress/psoc creator/4.3/psoc creator/import/gnu/arm/5.4.1/bin/../lib/gcc/arm-none-eabi/5.4.1/armv7-m\libgcc.a(_arm_addsubdf3.o)
 .bss           0x00000000        0x0 c:/program files (x86)/cypress/psoc creator/4.3/psoc creator/import/gnu/arm/5.4.1/bin/../lib/gcc/arm-none-eabi/5.4.1/armv7-m\libgcc.a(_arm_addsubdf3.o)
 .data          0x00000000        0x0 c:/program files (x86)/cypress/psoc creator/4.3/psoc creator/import/gnu/arm/5.4.1/bin/../lib/gcc/arm-none-eabi/5.4.1/armv7-m\libgcc.a(_arm_muldivdf3.o)
 .bss           0x00000000        0x0 c:/program files (x86)/cypress/psoc creator/4.3/psoc creator/import/gnu/arm/5.4.1/bin/../lib/gcc/arm-none-eabi/5.4.1/armv7-m\libgcc.a(_arm_muldivdf3.o)
 .data          0x00000000        0x0 c:/program files (x86)/cypress/psoc creator/4.3/psoc creator/import/gnu/arm/5.4.1/bin/../lib/gcc/arm-none-eabi/5.4.1/armv7-m\libgcc.a(_arm_cmpdf2.o)
 .bss           0x00000000        0x0 c:/program files (x86)/cypress/psoc creator/4.3/psoc creator/import/gnu/arm/5.4.1/bin/../lib/gcc/arm-none-eabi/5.4.1/armv7-m\libgcc.a(_arm_cmpdf2.o)
 .data          0x00000000        0x0 c:/program files (x86)/cypress/psoc creator/4.3/psoc creator/import/gnu/arm/5.4.1/bin/../lib/gcc/arm-none-eabi/5.4.1/armv7-m\libgcc.a(_arm_unorddf2.o)
 .bss           0x00000000        0x0 c:/program files (x86)/cypress/psoc creator/4.3/psoc creator/import/gnu/arm/5.4.1/bin/../lib/gcc/arm-none-eabi/5.4.1/armv7-m\libgcc.a(_arm_unorddf2.o)
 .data          0x00000000        0x0 c:/program files (x86)/cypress/psoc creator/4.3/psoc creator/import/gnu/arm/5.4.1/bin/../lib/gcc/arm-none-eabi/5.4.1/armv7-m\libgcc.a(_arm_truncdfsf2.o)
 .bss           0x00000000        0x0 c:/program files (x86)/cypress/psoc creator/4.3/psoc creator/import/gnu/arm/5.4.1/bin/../lib/gcc/arm-none-eabi/5.4.1/armv7-m\libgcc.a(_arm_truncdfsf2.o)
 .data          0x00000000        0x0 c:/program files (x86)/cypress/psoc creator/4.3/psoc creator/import/gnu/arm/5.4.1/bin/../lib/gcc/arm-none-eabi/5.4.1/armv7-m\libgcc.a(_arm_addsubsf3.o)
 .bss           0x00000000        0x0 c:/program files (x86)/cypress/psoc creator/4.3/psoc creator/import/gnu/arm/5.4.1/bin/../lib/gcc/arm-none-eabi/5.4.1/armv7-m\libgcc.a(_arm_addsubsf3.o)
 .data          0x00000000        0x0 c:/program files (x86)/cypress/psoc creator/4.3/psoc creator/import/gnu/arm/5.4.1/bin/../lib/gcc/arm-none-eabi/5.4.1/armv7-m\libgcc.a(_arm_muldivsf3.o)
 .bss           0x00000000        0x0 c:/program files (x86)/cypress/psoc creator/4.3/psoc creator/import/gnu/arm/5.4.1/bin/../lib/gcc/arm-none-eabi/5.4.1/armv7-m\libgcc.a(_arm_muldivsf3.o)
 .data          0x00000000        0x0 c:/program files (x86)/cypress/psoc creator/4.3/psoc creator/import/gnu/arm/5.4.1/bin/../lib/gcc/arm-none-eabi/5.4.1/armv7-m\libgcc.a(_arm_fixsfsi.o)
 .bss           0x00000000        0x0 c:/program files (x86)/cypress/psoc creator/4.3/psoc creator/import/gnu/arm/5.4.1/bin/../lib/gcc/arm-none-eabi/5.4.1/armv7-m\libgcc.a(_arm_fixsfsi.o)
 .text          0x00000000        0x0 c:/program files (x86)/cypress/psoc creator/4.3/psoc creator/import/gnu/arm/5.4.1/bin/../lib/gcc/arm-none-eabi/5.4.1/../../../../arm-none-eabi/lib/armv7-m\libg_nano.a(lib_a-errno.o)
 .data          0x00000000        0x0 c:/program files (x86)/cypress/psoc creator/4.3/psoc creator/import/gnu/arm/5.4.1/bin/../lib/gcc/arm-none-eabi/5.4.1/../../../../arm-none-eabi/lib/armv7-m\libg_nano.a(lib_a-errno.o)
 .bss           0x00000000        0x0 c:/program files (x86)/cypress/psoc creator/4.3/psoc creator/import/gnu/arm/5.4.1/bin/../lib/gcc/arm-none-eabi/5.4.1/../../../../arm-none-eabi/lib/armv7-m\libg_nano.a(lib_a-errno.o)
 .text          0x00000000        0x0 c:/program files (x86)/cypress/psoc creator/4.3/psoc creator/import/gnu/arm/5.4.1/bin/../lib/gcc/arm-none-eabi/5.4.1/../../../../arm-none-eabi/lib/armv7-m\libg_nano.a(lib_a-exit.o)
 .data          0x00000000        0x0 c:/program files (x86)/cypress/psoc creator/4.3/psoc creator/import/gnu/arm/5.4.1/bin/../lib/gcc/arm-none-eabi/5.4.1/../../../../arm-none-eabi/lib/armv7-m\libg_nano.a(lib_a-exit.o)
 .bss           0x00000000        0x0 c:/program files (x86)/cypress/psoc creator/4.3/psoc creator/import/gnu/arm/5.4.1/bin/../lib/gcc/arm-none-eabi/5.4.1/../../../../arm-none-eabi/lib/armv7-m\libg_nano.a(lib_a-exit.o)
 .text.exit     0x00000000       0x28 c:/program files (x86)/cypress/psoc creator/4.3/psoc creator/import/gnu/arm/5.4.1/bin/../lib/gcc/arm-none-eabi/5.4.1/../../../../arm-none-eabi/lib/armv7-m\libg_nano.a(lib_a-exit.o)
 .text          0x00000000        0x0 c:/program files (x86)/cypress/psoc creator/4.3/psoc creator/import/gnu/arm/5.4.1/bin/../lib/gcc/arm-none-eabi/5.4.1/../../../../arm-none-eabi/lib/armv7-m\libg_nano.a(lib_a-impure.o)
 .data          0x00000000        0x0 c:/program files (x86)/cypress/psoc creator/4.3/psoc creator/import/gnu/arm/5.4.1/bin/../lib/gcc/arm-none-eabi/5.4.1/../../../../arm-none-eabi/lib/armv7-m\libg_nano.a(lib_a-impure.o)
 .bss           0x00000000        0x0 c:/program files (x86)/cypress/psoc creator/4.3/psoc creator/import/gnu/arm/5.4.1/bin/../lib/gcc/arm-none-eabi/5.4.1/../../../../arm-none-eabi/lib/armv7-m\libg_nano.a(lib_a-impure.o)
 .rodata._global_impure_ptr
                0x00000000        0x4 c:/program files (x86)/cypress/psoc creator/4.3/psoc creator/import/gnu/arm/5.4.1/bin/../lib/gcc/arm-none-eabi/5.4.1/../../../../arm-none-eabi/lib/armv7-m\libg_nano.a(lib_a-impure.o)
 .text          0x00000000        0x0 c:/program files (x86)/cypress/psoc creator/4.3/psoc creator/import/gnu/arm/5.4.1/bin/../lib/gcc/arm-none-eabi/5.4.1/../../../../arm-none-eabi/lib/armv7-m\libg_nano.a(lib_a-init.o)
 .data          0x00000000        0x0 c:/program files (x86)/cypress/psoc creator/4.3/psoc creator/import/gnu/arm/5.4.1/bin/../lib/gcc/arm-none-eabi/5.4.1/../../../../arm-none-eabi/lib/armv7-m\libg_nano.a(lib_a-init.o)
 .bss           0x00000000        0x0 c:/program files (x86)/cypress/psoc creator/4.3/psoc creator/import/gnu/arm/5.4.1/bin/../lib/gcc/arm-none-eabi/5.4.1/../../../../arm-none-eabi/lib/armv7-m\libg_nano.a(lib_a-init.o)
 .text          0x00000000        0x0 c:/program files (x86)/cypress/psoc creator/4.3/psoc creator/import/gnu/arm/5.4.1/bin/../lib/gcc/arm-none-eabi/5.4.1/../../../../arm-none-eabi/lib/armv7-m\libg_nano.a(lib_a-memcpy-stub.o)
 .data          0x00000000        0x0 c:/program files (x86)/cypress/psoc creator/4.3/psoc creator/import/gnu/arm/5.4.1/bin/../lib/gcc/arm-none-eabi/5.4.1/../../../../arm-none-eabi/lib/armv7-m\libg_nano.a(lib_a-memcpy-stub.o)
 .bss           0x00000000        0x0 c:/program files (x86)/cypress/psoc creator/4.3/psoc creator/import/gnu/arm/5.4.1/bin/../lib/gcc/arm-none-eabi/5.4.1/../../../../arm-none-eabi/lib/armv7-m\libg_nano.a(lib_a-memcpy-stub.o)
 .text          0x00000000        0x0 c:/program files (x86)/cypress/psoc creator/4.3/psoc creator/import/gnu/arm/5.4.1/bin/../lib/gcc/arm-none-eabi/5.4.1/../../../../arm-none-eabi/lib/armv7-m\libg_nano.a(lib_a-memset.o)
 .data          0x00000000        0x0 c:/program files (x86)/cypress/psoc creator/4.3/psoc creator/import/gnu/arm/5.4.1/bin/../lib/gcc/arm-none-eabi/5.4.1/../../../../arm-none-eabi/lib/armv7-m\libg_nano.a(lib_a-memset.o)
 .bss           0x00000000        0x0 c:/program files (x86)/cypress/psoc creator/4.3/psoc creator/import/gnu/arm/5.4.1/bin/../lib/gcc/arm-none-eabi/5.4.1/../../../../arm-none-eabi/lib/armv7-m\libg_nano.a(lib_a-memset.o)
 .text          0x00000000        0x0 c:/program files (x86)/cypress/psoc creator/4.3/psoc creator/import/gnu/arm/5.4.1/bin/../lib/gcc/arm-none-eabi/5.4.1/../../../../arm-none-eabi/lib/armv7-m\libg_nano.a(lib_a-sprintf.o)
 .data          0x00000000        0x0 c:/program files (x86)/cypress/psoc creator/4.3/psoc creator/import/gnu/arm/5.4.1/bin/../lib/gcc/arm-none-eabi/5.4.1/../../../../arm-none-eabi/lib/armv7-m\libg_nano.a(lib_a-sprintf.o)
 .bss           0x00000000        0x0 c:/program files (x86)/cypress/psoc creator/4.3/psoc creator/import/gnu/arm/5.4.1/bin/../lib/gcc/arm-none-eabi/5.4.1/../../../../arm-none-eabi/lib/armv7-m\libg_nano.a(lib_a-sprintf.o)
 .text._sprintf_r
                0x00000000       0x40 c:/program files (x86)/cypress/psoc creator/4.3/psoc creator/import/gnu/arm/5.4.1/bin/../lib/gcc/arm-none-eabi/5.4.1/../../../../arm-none-eabi/lib/armv7-m\libg_nano.a(lib_a-sprintf.o)
 .text          0x00000000        0x0 c:/program files (x86)/cypress/psoc creator/4.3/psoc creator/import/gnu/arm/5.4.1/bin/../lib/gcc/arm-none-eabi/5.4.1/../../../../arm-none-eabi/lib/armv7-m\libg_nano.a(lib_a-nano-svfprintf.o)
 .data          0x00000000        0x0 c:/program files (x86)/cypress/psoc creator/4.3/psoc creator/import/gnu/arm/5.4.1/bin/../lib/gcc/arm-none-eabi/5.4.1/../../../../arm-none-eabi/lib/armv7-m\libg_nano.a(lib_a-nano-svfprintf.o)
 .bss           0x00000000        0x0 c:/program files (x86)/cypress/psoc creator/4.3/psoc creator/import/gnu/arm/5.4.1/bin/../lib/gcc/arm-none-eabi/5.4.1/../../../../arm-none-eabi/lib/armv7-m\libg_nano.a(lib_a-nano-svfprintf.o)
 .text.__ssprint_r
                0x00000000       0xfe c:/program files (x86)/cypress/psoc creator/4.3/psoc creator/import/gnu/arm/5.4.1/bin/../lib/gcc/arm-none-eabi/5.4.1/../../../../arm-none-eabi/lib/armv7-m\libg_nano.a(lib_a-nano-svfprintf.o)
 .text          0x00000000        0x0 c:/program files (x86)/cypress/psoc creator/4.3/psoc creator/import/gnu/arm/5.4.1/bin/../lib/gcc/arm-none-eabi/5.4.1/../../../../arm-none-eabi/lib/armv7-m\libg_nano.a(lib_a-nano-vfprintf_i.o)
 .data          0x00000000        0x0 c:/program files (x86)/cypress/psoc creator/4.3/psoc creator/import/gnu/arm/5.4.1/bin/../lib/gcc/arm-none-eabi/5.4.1/../../../../arm-none-eabi/lib/armv7-m\libg_nano.a(lib_a-nano-vfprintf_i.o)
 .bss           0x00000000        0x0 c:/program files (x86)/cypress/psoc creator/4.3/psoc creator/import/gnu/arm/5.4.1/bin/../lib/gcc/arm-none-eabi/5.4.1/../../../../arm-none-eabi/lib/armv7-m\libg_nano.a(lib_a-nano-vfprintf_i.o)
 .text          0x00000000        0x0 c:/program files (x86)/cypress/psoc creator/4.3/psoc creator/import/gnu/arm/5.4.1/bin/../lib/gcc/arm-none-eabi/5.4.1/../../../../arm-none-eabi/lib/armv7-m\libg_nano.a(lib_a-memchr-stub.o)
 .data          0x00000000        0x0 c:/program files (x86)/cypress/psoc creator/4.3/psoc creator/import/gnu/arm/5.4.1/bin/../lib/gcc/arm-none-eabi/5.4.1/../../../../arm-none-eabi/lib/armv7-m\libg_nano.a(lib_a-memchr-stub.o)
 .bss           0x00000000        0x0 c:/program files (x86)/cypress/psoc creator/4.3/psoc creator/import/gnu/arm/5.4.1/bin/../lib/gcc/arm-none-eabi/5.4.1/../../../../arm-none-eabi/lib/armv7-m\libg_nano.a(lib_a-memchr-stub.o)
 .text          0x00000000        0x0 c:/program files (x86)/cypress/psoc creator/4.3/psoc creator/import/gnu/arm/5.4.1/bin/../lib/gcc/arm-none-eabi/5.4.1/../../../../arm-none-eabi/lib/armv7-m\libg_nano.a(lib_a-memmove.o)
 .data          0x00000000        0x0 c:/program files (x86)/cypress/psoc creator/4.3/psoc creator/import/gnu/arm/5.4.1/bin/../lib/gcc/arm-none-eabi/5.4.1/../../../../arm-none-eabi/lib/armv7-m\libg_nano.a(lib_a-memmove.o)
 .bss           0x00000000        0x0 c:/program files (x86)/cypress/psoc creator/4.3/psoc creator/import/gnu/arm/5.4.1/bin/../lib/gcc/arm-none-eabi/5.4.1/../../../../arm-none-eabi/lib/armv7-m\libg_nano.a(lib_a-memmove.o)
 .text          0x00000000        0x0 c:/program files (x86)/cypress/psoc creator/4.3/psoc creator/import/gnu/arm/5.4.1/bin/../lib/gcc/arm-none-eabi/5.4.1/../../../../arm-none-eabi/lib/armv7-m\libg_nano.a(lib_a-nano-freer.o)
 .data          0x00000000        0x0 c:/program files (x86)/cypress/psoc creator/4.3/psoc creator/import/gnu/arm/5.4.1/bin/../lib/gcc/arm-none-eabi/5.4.1/../../../../arm-none-eabi/lib/armv7-m\libg_nano.a(lib_a-nano-freer.o)
 .bss           0x00000000        0x0 c:/program files (x86)/cypress/psoc creator/4.3/psoc creator/import/gnu/arm/5.4.1/bin/../lib/gcc/arm-none-eabi/5.4.1/../../../../arm-none-eabi/lib/armv7-m\libg_nano.a(lib_a-nano-freer.o)
 .text          0x00000000        0x0 c:/program files (x86)/cypress/psoc creator/4.3/psoc creator/import/gnu/arm/5.4.1/bin/../lib/gcc/arm-none-eabi/5.4.1/../../../../arm-none-eabi/lib/armv7-m\libg_nano.a(lib_a-nano-mallocr.o)
 .data          0x00000000        0x0 c:/program files (x86)/cypress/psoc creator/4.3/psoc creator/import/gnu/arm/5.4.1/bin/../lib/gcc/arm-none-eabi/5.4.1/../../../../arm-none-eabi/lib/armv7-m\libg_nano.a(lib_a-nano-mallocr.o)
 .bss           0x00000000        0x0 c:/program files (x86)/cypress/psoc creator/4.3/psoc creator/import/gnu/arm/5.4.1/bin/../lib/gcc/arm-none-eabi/5.4.1/../../../../arm-none-eabi/lib/armv7-m\libg_nano.a(lib_a-nano-mallocr.o)
 .text          0x00000000        0x0 c:/program files (x86)/cypress/psoc creator/4.3/psoc creator/import/gnu/arm/5.4.1/bin/../lib/gcc/arm-none-eabi/5.4.1/../../../../arm-none-eabi/lib/armv7-m\libg_nano.a(lib_a-nano-reallocr.o)
 .data          0x00000000        0x0 c:/program files (x86)/cypress/psoc creator/4.3/psoc creator/import/gnu/arm/5.4.1/bin/../lib/gcc/arm-none-eabi/5.4.1/../../../../arm-none-eabi/lib/armv7-m\libg_nano.a(lib_a-nano-reallocr.o)
 .bss           0x00000000        0x0 c:/program files (x86)/cypress/psoc creator/4.3/psoc creator/import/gnu/arm/5.4.1/bin/../lib/gcc/arm-none-eabi/5.4.1/../../../../arm-none-eabi/lib/armv7-m\libg_nano.a(lib_a-nano-reallocr.o)
 .text          0x00000000        0x0 c:/program files (x86)/cypress/psoc creator/4.3/psoc creator/import/gnu/arm/5.4.1/bin/../lib/gcc/arm-none-eabi/5.4.1/../../../../arm-none-eabi/lib/armv7-m\libg_nano.a(lib_a-sbrkr.o)
 .data          0x00000000        0x0 c:/program files (x86)/cypress/psoc creator/4.3/psoc creator/import/gnu/arm/5.4.1/bin/../lib/gcc/arm-none-eabi/5.4.1/../../../../arm-none-eabi/lib/armv7-m\libg_nano.a(lib_a-sbrkr.o)
 .bss           0x00000000        0x0 c:/program files (x86)/cypress/psoc creator/4.3/psoc creator/import/gnu/arm/5.4.1/bin/../lib/gcc/arm-none-eabi/5.4.1/../../../../arm-none-eabi/lib/armv7-m\libg_nano.a(lib_a-sbrkr.o)
 .text          0x00000000        0x0 c:/program files (x86)/cypress/psoc creator/4.3/psoc creator/import/gnu/arm/5.4.1/bin/../lib/gcc/arm-none-eabi/5.4.1/../../../../arm-none-eabi/lib/armv7-m\libg_nano.a(lib_a-mlock.o)
 .data          0x00000000        0x0 c:/program files (x86)/cypress/psoc creator/4.3/psoc creator/import/gnu/arm/5.4.1/bin/../lib/gcc/arm-none-eabi/5.4.1/../../../../arm-none-eabi/lib/armv7-m\libg_nano.a(lib_a-mlock.o)
 .bss           0x00000000        0x0 c:/program files (x86)/cypress/psoc creator/4.3/psoc creator/import/gnu/arm/5.4.1/bin/../lib/gcc/arm-none-eabi/5.4.1/../../../../arm-none-eabi/lib/armv7-m\libg_nano.a(lib_a-mlock.o)
 .text          0x00000000        0x0 c:/program files (x86)/cypress/psoc creator/4.3/psoc creator/import/gnu/arm/5.4.1/bin/../lib/gcc/arm-none-eabi/5.4.1/../../../../arm-none-eabi/lib/armv7-m\libg_nano.a(lib_a-nano-msizer.o)
 .data          0x00000000        0x0 c:/program files (x86)/cypress/psoc creator/4.3/psoc creator/import/gnu/arm/5.4.1/bin/../lib/gcc/arm-none-eabi/5.4.1/../../../../arm-none-eabi/lib/armv7-m\libg_nano.a(lib_a-nano-msizer.o)
 .bss           0x00000000        0x0 c:/program files (x86)/cypress/psoc creator/4.3/psoc creator/import/gnu/arm/5.4.1/bin/../lib/gcc/arm-none-eabi/5.4.1/../../../../arm-none-eabi/lib/armv7-m\libg_nano.a(lib_a-nano-msizer.o)
 .text          0x00000000        0x0 c:/program files (x86)/cypress/psoc creator/4.3/psoc creator/import/gnu/arm/5.4.1/bin/../lib/gcc/arm-none-eabi/5.4.1/../../../../arm-none-eabi/lib/armv7-m\libg_nano.a(lib_a-reent.o)
 .data          0x00000000        0x0 c:/program files (x86)/cypress/psoc creator/4.3/psoc creator/import/gnu/arm/5.4.1/bin/../lib/gcc/arm-none-eabi/5.4.1/../../../../arm-none-eabi/lib/armv7-m\libg_nano.a(lib_a-reent.o)
 .bss           0x00000000        0x0 c:/program files (x86)/cypress/psoc creator/4.3/psoc creator/import/gnu/arm/5.4.1/bin/../lib/gcc/arm-none-eabi/5.4.1/../../../../arm-none-eabi/lib/armv7-m\libg_nano.a(lib_a-reent.o)
 .text.cleanup_glue
                0x00000000       0x1a c:/program files (x86)/cypress/psoc creator/4.3/psoc creator/import/gnu/arm/5.4.1/bin/../lib/gcc/arm-none-eabi/5.4.1/../../../../arm-none-eabi/lib/armv7-m\libg_nano.a(lib_a-reent.o)
 .text._reclaim_reent
                0x00000000       0xb4 c:/program files (x86)/cypress/psoc creator/4.3/psoc creator/import/gnu/arm/5.4.1/bin/../lib/gcc/arm-none-eabi/5.4.1/../../../../arm-none-eabi/lib/armv7-m\libg_nano.a(lib_a-reent.o)
 .text          0x00000000        0x0 c:/program files (x86)/cypress/psoc creator/4.3/psoc creator/import/gnu/arm/5.4.1/bin/../lib/gcc/arm-none-eabi/5.4.1/armv7-m/crtend.o
 .data          0x00000000        0x0 c:/program files (x86)/cypress/psoc creator/4.3/psoc creator/import/gnu/arm/5.4.1/bin/../lib/gcc/arm-none-eabi/5.4.1/armv7-m/crtend.o
 .bss           0x00000000        0x0 c:/program files (x86)/cypress/psoc creator/4.3/psoc creator/import/gnu/arm/5.4.1/bin/../lib/gcc/arm-none-eabi/5.4.1/armv7-m/crtend.o
 .text          0x00000000        0x0 c:/program files (x86)/cypress/psoc creator/4.3/psoc creator/import/gnu/arm/5.4.1/bin/../lib/gcc/arm-none-eabi/5.4.1/armv7-m/crtn.o
 .data          0x00000000        0x0 c:/program files (x86)/cypress/psoc creator/4.3/psoc creator/import/gnu/arm/5.4.1/bin/../lib/gcc/arm-none-eabi/5.4.1/armv7-m/crtn.o
 .bss           0x00000000        0x0 c:/program files (x86)/cypress/psoc creator/4.3/psoc creator/import/gnu/arm/5.4.1/bin/../lib/gcc/arm-none-eabi/5.4.1/armv7-m/crtn.o

Memory Configuration

Name             Origin             Length             Attributes
rom              0x00000000         0x00040000         xr
ram              0x1fff8000         0x00010000         xrw
*default*        0x00000000         0xffffffff

Linker script and memory map

LOAD c:/program files (x86)/cypress/psoc creator/4.3/psoc creator/import/gnu/arm/5.4.1/bin/../lib/gcc/arm-none-eabi/5.4.1/armv7-m/crti.o
LOAD c:/program files (x86)/cypress/psoc creator/4.3/psoc creator/import/gnu/arm/5.4.1/bin/../lib/gcc/arm-none-eabi/5.4.1/armv7-m/crtbegin.o
LOAD c:/program files (x86)/cypress/psoc creator/4.3/psoc creator/import/gnu/arm/5.4.1/bin/../lib/gcc/arm-none-eabi/5.4.1/../../../../arm-none-eabi/lib/armv7-m/crt0.o
START GROUP
LOAD .\CortexM3\ARM_GCC_541\Debug\main.o
LOAD .\CortexM3\ARM_GCC_541\Debug\I2C_Functions.o
LOAD .\CortexM3\ARM_GCC_541\Debug\VCNL4030X01_PS.o
LOAD .\CortexM3\ARM_GCC_541\Debug\VCNL4030X01_ALS.o
LOAD .\CortexM3\ARM_GCC_541\Debug\VCNL4030X01_Application_Library.o
LOAD .\CortexM3\ARM_GCC_541\Debug\cyfitter_cfg.o
LOAD .\CortexM3\ARM_GCC_541\Debug\cymetadata.o
LOAD .\CortexM3\ARM_GCC_541\Debug\Cm3Start.o
LOAD .\CortexM3\ARM_GCC_541\Debug\VCNL4030X01.a
LOAD C:\Program Files (x86)\Cypress\PSoC Creator\4.3\PSoC Creator\psoc\content\cycomponentlibrary\CyComponentLibrary.cylib\CortexM3\ARM_GCC_541\Debug\CyComponentLibrary.a
LOAD c:/program files (x86)/cypress/psoc creator/4.3/psoc creator/import/gnu/arm/5.4.1/bin/../lib/gcc/arm-none-eabi/5.4.1/../../../../arm-none-eabi/lib/armv7-m\libm.a
END GROUP
START GROUP
LOAD c:/program files (x86)/cypress/psoc creator/4.3/psoc creator/import/gnu/arm/5.4.1/bin/../lib/gcc/arm-none-eabi/5.4.1/armv7-m\libgcc.a
LOAD c:/program files (x86)/cypress/psoc creator/4.3/psoc creator/import/gnu/arm/5.4.1/bin/../lib/gcc/arm-none-eabi/5.4.1/../../../../arm-none-eabi/lib/armv7-m\libg_nano.a
LOAD c:/program files (x86)/cypress/psoc creator/4.3/psoc creator/import/gnu/arm/5.4.1/bin/../lib/gcc/arm-none-eabi/5.4.1/../../../../arm-none-eabi/lib/armv7-m\libc_nano.a
END GROUP
START GROUP
LOAD c:/program files (x86)/cypress/psoc creator/4.3/psoc creator/import/gnu/arm/5.4.1/bin/../lib/gcc/arm-none-eabi/5.4.1/armv7-m\libgcc.a
LOAD c:/program files (x86)/cypress/psoc creator/4.3/psoc creator/import/gnu/arm/5.4.1/bin/../lib/gcc/arm-none-eabi/5.4.1/../../../../arm-none-eabi/lib/armv7-m\libc_nano.a
END GROUP
LOAD c:/program files (x86)/cypress/psoc creator/4.3/psoc creator/import/gnu/arm/5.4.1/bin/../lib/gcc/arm-none-eabi/5.4.1/armv7-m/crtend.o
LOAD c:/program files (x86)/cypress/psoc creator/4.3/psoc creator/import/gnu/arm/5.4.1/bin/../lib/gcc/arm-none-eabi/5.4.1/armv7-m/crtn.o
START GROUP
LOAD c:/program files (x86)/cypress/psoc creator/4.3/psoc creator/import/gnu/arm/5.4.1/bin/../lib/gcc/arm-none-eabi/5.4.1/armv7-m\libgcc.a
LOAD c:/program files (x86)/cypress/psoc creator/4.3/psoc creator/import/gnu/arm/5.4.1/bin/../lib/gcc/arm-none-eabi/5.4.1/../../../../arm-none-eabi/lib/armv7-m\libc.a
LOAD c:/program files (x86)/cypress/psoc creator/4.3/psoc creator/import/gnu/arm/5.4.1/bin/../lib/gcc/arm-none-eabi/5.4.1/../../../../arm-none-eabi/lib/armv7-m\libnosys.a
END GROUP
                0x00000000                CY_APPL_ORIGIN = 0x0
                0x00000100                CY_FLASH_ROW_SIZE = 0x100
                0x00000020                CY_ECC_ROW_SIZE = 0x20
                0x00000000                CY_EE_IN_BTLDR = 0x0
                0x00000000                CY_APPL_LOADABLE = 0x0
                0x00000800                CY_EE_SIZE = 0x800
                0x00000001                CY_APPL_NUM = 0x1
                0x00000001                CY_APPL_MAX = 0x1
                0x00000040                CY_METADATA_SIZE = 0x40
                0x00000000                CY_APPL_LOADABLE = 0x0
                0x00000000                CY_CHECKSUM_EXCLUDE_SIZE = ALIGN (0x0, CY_FLASH_ROW_SIZE)
                [!provide]                PROVIDE (__cy_heap_start, _end)
                0x00000001                PROVIDE (__cy_region_num, ((__cy_regions_end - __cy_regions) / 0x10))
                0x20008000                PROVIDE (__cy_stack, (ORIGIN (ram) + LENGTH (ram)))
                [!provide]                PROVIDE (__cy_heap_end, (__cy_stack - 0x800))

.cybootloader   0x00000000        0x0
 *(.cybootloader)
                0x00000000                appl1_start = CY_APPL_ORIGIN?CY_APPL_ORIGIN:ALIGN (CY_FLASH_ROW_SIZE)
                0x0001ff00                appl2_start = (appl1_start + ALIGN ((((LENGTH (rom) - appl1_start) - (0x2 * CY_FLASH_ROW_SIZE)) / 0x2), CY_FLASH_ROW_SIZE))
                0x00000000                appl_start = (CY_APPL_NUM == 0x1)?appl1_start:appl2_start
                0x00000000                ecc_offset = ((appl_start / CY_FLASH_ROW_SIZE) * CY_ECC_ROW_SIZE)
                0x00000000                ee_offset = (CY_APPL_LOADABLE && ! (CY_EE_IN_BTLDR))?((CY_EE_SIZE / CY_APPL_MAX) * (CY_APPL_NUM - 0x1)):0x0
                0x00000800                ee_size = (CY_APPL_LOADABLE && ! (CY_EE_IN_BTLDR))?(CY_EE_SIZE / CY_APPL_MAX):CY_EE_SIZE
                [!provide]                PROVIDE (CY_ECC_OFFSET, ecc_offset)

.text           0x00000000     0x551c
 CREATE_OBJECT_SYMBOLS
                0x00000000                PROVIDE (__cy_interrupt_vector, RomVectors)
 *(.romvectors)
 .romvectors    0x00000000       0x10 .\CortexM3\ARM_GCC_541\Debug\Cm3Start.o
                0x00000000                RomVectors
                0x00000001                ASSERT ((. != __cy_interrupt_vector), No interrupt vector)
                0x00000001                ASSERT (CY_APPL_ORIGIN?(SIZEOF (.cybootloader) <= CY_APPL_ORIGIN):0x1, Wrong image location)
                0x00000010                PROVIDE (__cy_reset, Reset)
 *(.text.Reset)
 .text.Reset    0x00000010       0x18 .\CortexM3\ARM_GCC_541\Debug\Cm3Start.o
                0x00000010                Reset
                0x00000001                ASSERT ((. != __cy_reset), No reset code)
 *(.dma_init)
                0x00000001                ASSERT ((((appl_start + .) <= 0x10000) || 0x1), DMA Init must be within the first 64k of flash)
 *(.text .text.* .gnu.linkonce.t.*)
 .text          0x00000028       0x5c c:/program files (x86)/cypress/psoc creator/4.3/psoc creator/import/gnu/arm/5.4.1/bin/../lib/gcc/arm-none-eabi/5.4.1/armv7-m/crtbegin.o
 .text.Basic_Initialization_Auto_Mode
                0x00000084       0x40 .\CortexM3\ARM_GCC_541\Debug\main.o
                0x00000084                Basic_Initialization_Auto_Mode
 .text.main     0x000000c4       0x24 .\CortexM3\ARM_GCC_541\Debug\main.o
                0x000000c4                main
 .text.WriteI2C_Bus
                0x000000e8       0x48 .\CortexM3\ARM_GCC_541\Debug\I2C_Functions.o
                0x000000e8                WriteI2C_Bus
 .text.ReadI2C_Bus
                0x00000130       0x50 .\CortexM3\ARM_GCC_541\Debug\I2C_Functions.o
                0x00000130                ReadI2C_Bus
 .text.VCNL4030X01_SET_PS_IT
                0x00000180       0x44 .\CortexM3\ARM_GCC_541\Debug\VCNL4030X01_PS.o
                0x00000180                VCNL4030X01_SET_PS_IT
 .text.VCNL4030X01_SET_PS_SD
                0x000001c4       0x44 .\CortexM3\ARM_GCC_541\Debug\VCNL4030X01_PS.o
                0x000001c4                VCNL4030X01_SET_PS_SD
 .text.VCNL4030X01_SET_PS_HD
                0x00000208       0x44 .\CortexM3\ARM_GCC_541\Debug\VCNL4030X01_PS.o
                0x00000208                VCNL4030X01_SET_PS_HD
 .text.VCNL4030X01_SET_PS_AF
                0x0000024c       0x44 .\CortexM3\ARM_GCC_541\Debug\VCNL4030X01_PS.o
                0x0000024c                VCNL4030X01_SET_PS_AF
 .text.VCNL4030X01_SET_PS_TRIG
                0x00000290       0x44 .\CortexM3\ARM_GCC_541\Debug\VCNL4030X01_PS.o
                0x00000290                VCNL4030X01_SET_PS_TRIG
 .text.VCNL4030X01_SET_PS_SC_EN
                0x000002d4       0x44 .\CortexM3\ARM_GCC_541\Debug\VCNL4030X01_PS.o
                0x000002d4                VCNL4030X01_SET_PS_SC_EN
 .text.VCNL4030X01_SET_PS_LED_I
                0x00000318       0x44 .\CortexM3\ARM_GCC_541\Debug\VCNL4030X01_PS.o
                0x00000318                VCNL4030X01_SET_PS_LED_I
 .text.VCNL4030X01_GET_PS_Interrupt
                0x0000035c       0x34 .\CortexM3\ARM_GCC_541\Debug\VCNL4030X01_PS.o
                0x0000035c                VCNL4030X01_GET_PS_Interrupt
 .text.VCNL4030X01_READ_Reg
                0x00000390       0x34 .\CortexM3\ARM_GCC_541\Debug\VCNL4030X01_PS.o
                0x00000390                VCNL4030X01_READ_Reg
 .text.VCNL4030X01_GET_PS_SD_Bit
                0x000003c4       0x38 .\CortexM3\ARM_GCC_541\Debug\VCNL4030X01_PS.o
                0x000003c4                VCNL4030X01_GET_PS_SD_Bit
 .text.VCNL4030X01_GET_PS_AF_Bit
                0x000003fc       0x38 .\CortexM3\ARM_GCC_541\Debug\VCNL4030X01_PS.o
                0x000003fc                VCNL4030X01_GET_PS_AF_Bit
 .text.VCNL4030X01_GET_LED_I_LOW_Bit
                0x00000434       0x38 .\CortexM3\ARM_GCC_541\Debug\VCNL4030X01_PS.o
                0x00000434                VCNL4030X01_GET_LED_I_LOW_Bit
 .text.VCNL4030X01_GET_ALS_Data
                0x0000046c       0x34 .\CortexM3\ARM_GCC_541\Debug\VCNL4030X01_ALS.o
                0x0000046c                VCNL4030X01_GET_ALS_Data
 .text.VCNL4030X01_GET_White_Data
                0x000004a0       0x34 .\CortexM3\ARM_GCC_541\Debug\VCNL4030X01_ALS.o
                0x000004a0                VCNL4030X01_GET_White_Data
 .text.VCNL4030X01_GET_ALS_Interrupt
                0x000004d4       0x34 .\CortexM3\ARM_GCC_541\Debug\VCNL4030X01_ALS.o
                0x000004d4                VCNL4030X01_GET_ALS_Interrupt
 .text.VCNL4030X01_GET_ALS_SD_Bit
                0x00000508       0x38 .\CortexM3\ARM_GCC_541\Debug\VCNL4030X01_ALS.o
                0x00000508                VCNL4030X01_GET_ALS_SD_Bit
 .text.VCNL4030X01_GET_WHITE_SD_Bit
                0x00000540       0x38 .\CortexM3\ARM_GCC_541\Debug\VCNL4030X01_ALS.o
                0x00000540                VCNL4030X01_GET_WHITE_SD_Bit
 .text.VCNL4030X01_GET_ALS_IT_Bits
                0x00000578       0x70 .\CortexM3\ARM_GCC_541\Debug\VCNL4030X01_ALS.o
                0x00000578                VCNL4030X01_GET_ALS_IT_Bits
 .text.VCNL4030X01_CAL_Sensitivity
                0x000005e8       0x34 .\CortexM3\ARM_GCC_541\Debug\VCNL4030X01_Application_Library.o
                0x000005e8                VCNL4030X01_CAL_Sensitivity
 .text.VCNL4030X01_CAL_Lux
                0x0000061c        0x8 .\CortexM3\ARM_GCC_541\Debug\VCNL4030X01_Application_Library.o
                0x0000061c                VCNL4030X01_CAL_Lux
 .text.VCNL4030X01_GET_Delay
                0x00000624       0x60 .\CortexM3\ARM_GCC_541\Debug\VCNL4030X01_Application_Library.o
                0x00000624                VCNL4030X01_GET_Delay
 .text.VCNL4030X01_GET_ALS_IT
                0x00000684       0x68 .\CortexM3\ARM_GCC_541\Debug\VCNL4030X01_Application_Library.o
                0x00000684                VCNL4030X01_GET_ALS_IT
 .text.VCNL4030X01_GET_PS_Mode
                0x000006ec       0x30 .\CortexM3\ARM_GCC_541\Debug\VCNL4030X01_Application_Library.o
                0x000006ec                VCNL4030X01_GET_PS_Mode
 .text.VCNL4030X01_GET_ALS_Mode
                0x0000071c       0x28 .\CortexM3\ARM_GCC_541\Debug\VCNL4030X01_Application_Library.o
                0x0000071c                VCNL4030X01_GET_ALS_Mode
 .text.Reset_Sensor
                0x00000744      0x120 .\CortexM3\ARM_GCC_541\Debug\VCNL4030X01_Application_Library.o
                0x00000744                Reset_Sensor
 .text.reverse  0x00000864       0x1c .\CortexM3\ARM_GCC_541\Debug\VCNL4030X01_Application_Library.o
                0x00000864                reverse
 .text.intToStr
                0x00000880       0x4c .\CortexM3\ARM_GCC_541\Debug\VCNL4030X01_Application_Library.o
                0x00000880                intToStr
 .text.ftoa     0x000008cc       0x70 .\CortexM3\ARM_GCC_541\Debug\VCNL4030X01_Application_Library.o
                0x000008cc                ftoa
 .text.Print_Data_Only
                0x0000093c      0x45c .\CortexM3\ARM_GCC_541\Debug\VCNL4030X01_Application_Library.o
                0x0000093c                Print_Data_Only
 .text.CyClockStartupError
                0x00000d98        0x4 .\CortexM3\ARM_GCC_541\Debug\cyfitter_cfg.o
 .text.cfg_write_bytes32
                0x00000d9c       0x34 .\CortexM3\ARM_GCC_541\Debug\cyfitter_cfg.o
 .text.AnalogSetDefault
                0x00000dd0       0x28 .\CortexM3\ARM_GCC_541\Debug\cyfitter_cfg.o
 .text.CYMEMZERO
                0x00000df8        0xc .\CortexM3\ARM_GCC_541\Debug\cyfitter_cfg.o
 .text.ClockSetup
                0x00000e04       0xa0 .\CortexM3\ARM_GCC_541\Debug\cyfitter_cfg.o
 .text.CYCONFIGCPY
                0x00000ea4        0x8 .\CortexM3\ARM_GCC_541\Debug\cyfitter_cfg.o
 .text.cyfitter_cfg
                0x00000eac       0xcc .\CortexM3\ARM_GCC_541\Debug\cyfitter_cfg.o
                0x00000eac                cyfitter_cfg
 .text.IntDefaultHandler
                0x00000f78       0x10 .\CortexM3\ARM_GCC_541\Debug\Cm3Start.o
                0x00000f78                IntDefaultHandler
 .text._sbrk    0x00000f88       0x30 .\CortexM3\ARM_GCC_541\Debug\Cm3Start.o
                0x00000f88                _sbrk
 .text.Start_c  0x00000fb8       0x4c .\CortexM3\ARM_GCC_541\Debug\Cm3Start.o
                0x00000fb8                Start_c
 .text.initialize_psoc
                0x00001004       0x68 .\CortexM3\ARM_GCC_541\Debug\Cm3Start.o
                0x00001004                initialize_psoc
 .text.I2C_1_Init
                0x0000106c       0x68 .\CortexM3\ARM_GCC_541\Debug\VCNL4030X01.a(I2C_1.o)
                0x0000106c                I2C_1_Init
 .text.I2C_1_Enable
                0x000010d4       0x24 .\CortexM3\ARM_GCC_541\Debug\VCNL4030X01.a(I2C_1.o)
                0x000010d4                I2C_1_Enable
 .text.I2C_1_Start
                0x000010f8       0x28 .\CortexM3\ARM_GCC_541\Debug\VCNL4030X01.a(I2C_1.o)
                0x000010f8                I2C_1_Start
 .text.I2C_1_ISR
                0x00001120      0x2d0 .\CortexM3\ARM_GCC_541\Debug\VCNL4030X01.a(I2C_1_INT.o)
                0x00001120                I2C_1_ISR
 .text.I2C_1_MasterSendStart
                0x000013f0       0x80 .\CortexM3\ARM_GCC_541\Debug\VCNL4030X01.a(I2C_1_MASTER.o)
                0x000013f0                I2C_1_MasterSendStart
 .text.I2C_1_MasterSendRestart
                0x00001470       0x6c .\CortexM3\ARM_GCC_541\Debug\VCNL4030X01.a(I2C_1_MASTER.o)
                0x00001470                I2C_1_MasterSendRestart
 .text.I2C_1_MasterSendStop
                0x000014dc       0x38 .\CortexM3\ARM_GCC_541\Debug\VCNL4030X01.a(I2C_1_MASTER.o)
                0x000014dc                I2C_1_MasterSendStop
 .text.I2C_1_MasterWriteByte
                0x00001514       0x58 .\CortexM3\ARM_GCC_541\Debug\VCNL4030X01.a(I2C_1_MASTER.o)
                0x00001514                I2C_1_MasterWriteByte
 .text.I2C_1_MasterReadByte
                0x0000156c       0x58 .\CortexM3\ARM_GCC_541\Debug\VCNL4030X01.a(I2C_1_MASTER.o)
                0x0000156c                I2C_1_MasterReadByte
 .text.I2C_1_MasterStatus
                0x000015c4       0x38 .\CortexM3\ARM_GCC_541\Debug\VCNL4030X01.a(I2C_1_MASTER.o)
                0x000015c4                I2C_1_MasterStatus
 .text.I2C_1_MasterClearReadBuf
                0x000015fc       0x30 .\CortexM3\ARM_GCC_541\Debug\VCNL4030X01.a(I2C_1_MASTER.o)
                0x000015fc                I2C_1_MasterClearReadBuf
 .text.I2C_1_MasterClearWriteBuf
                0x0000162c       0x30 .\CortexM3\ARM_GCC_541\Debug\VCNL4030X01.a(I2C_1_MASTER.o)
                0x0000162c                I2C_1_MasterClearWriteBuf
 .text.CDC_Init
                0x0000165c      0x140 .\CortexM3\ARM_GCC_541\Debug\VCNL4030X01.a(CDC.o)
                0x0000165c                CDC_Init
 .text.CDC_InitComponent
                0x0000179c       0xb8 .\CortexM3\ARM_GCC_541\Debug\VCNL4030X01.a(CDC.o)
                0x0000179c                CDC_InitComponent
 .text.CDC_Start
                0x00001854       0x24 .\CortexM3\ARM_GCC_541\Debug\VCNL4030X01.a(CDC.o)
                0x00001854                CDC_Start
 .text.CDC_ReInitComponent
                0x00001878       0x4c .\CortexM3\ARM_GCC_541\Debug\VCNL4030X01.a(CDC.o)
                0x00001878                CDC_ReInitComponent
 .text.CDC_GetEPState
                0x000018c4       0x14 .\CortexM3\ARM_GCC_541\Debug\VCNL4030X01.a(CDC.o)
                0x000018c4                CDC_GetEPState
 .text.CDC_LoadInEP
                0x000018d8       0x94 .\CortexM3\ARM_GCC_541\Debug\VCNL4030X01.a(CDC.o)
                0x000018d8                CDC_LoadInEP
 .text.CDC_EnableOutEP
                0x0000196c       0x2c .\CortexM3\ARM_GCC_541\Debug\VCNL4030X01.a(CDC.o)
                0x0000196c                CDC_EnableOutEP
 .text.CDC_StrLen
                0x00001998       0x14 .\CortexM3\ARM_GCC_541\Debug\VCNL4030X01.a(CDC_cdc.o)
 .text.CDC_GetInterfaceComPort
                0x000019ac       0x38 .\CortexM3\ARM_GCC_541\Debug\VCNL4030X01.a(CDC_cdc.o)
                0x000019ac                CDC_GetInterfaceComPort
 .text.CDC_DispatchCDCClassRqst
                0x000019e4       0x98 .\CortexM3\ARM_GCC_541\Debug\VCNL4030X01.a(CDC_cdc.o)
                0x000019e4                CDC_DispatchCDCClassRqst
 .text.CDC_CDC_Init
                0x00001a7c       0x98 .\CortexM3\ARM_GCC_541\Debug\VCNL4030X01.a(CDC_cdc.o)
                0x00001a7c                CDC_CDC_Init
 .text.CDC_PutString
                0x00001b14       0xa0 .\CortexM3\ARM_GCC_541\Debug\VCNL4030X01.a(CDC_cdc.o)
                0x00001b14                CDC_PutString
 .text.CDC_CDCIsReady
                0x00001bb4       0x18 .\CortexM3\ARM_GCC_541\Debug\VCNL4030X01.a(CDC_cdc.o)
                0x00001bb4                CDC_CDCIsReady
 .text.CDC_Cdc_EpInit
                0x00001bcc       0x50 .\CortexM3\ARM_GCC_541\Debug\VCNL4030X01.a(CDC_cdc.o)
                0x00001bcc                CDC_Cdc_EpInit
 .text.CDC_LoadEP0
                0x00001c1c       0x98 .\CortexM3\ARM_GCC_541\Debug\VCNL4030X01.a(CDC_drv.o)
                0x00001c1c                CDC_LoadEP0
 .text.CDC_InitZeroLengthControlTransfer
                0x00001cb4       0x34 .\CortexM3\ARM_GCC_541\Debug\VCNL4030X01.a(CDC_drv.o)
                0x00001cb4                CDC_InitZeroLengthControlTransfer
 .text.CDC_ControlReadDataStage
                0x00001ce8        0x8 .\CortexM3\ARM_GCC_541\Debug\VCNL4030X01.a(CDC_drv.o)
                0x00001ce8                CDC_ControlReadDataStage
 .text.CDC_ControlWriteDataStage
                0x00001cf0       0x84 .\CortexM3\ARM_GCC_541\Debug\VCNL4030X01.a(CDC_drv.o)
                0x00001cf0                CDC_ControlWriteDataStage
 .text.CDC_InitNoDataControlTransfer
                0x00001d74       0x2c .\CortexM3\ARM_GCC_541\Debug\VCNL4030X01.a(CDC_drv.o)
                0x00001d74                CDC_InitNoDataControlTransfer
 .text.CDC_UpdateStatusBlock
                0x00001da0       0x24 .\CortexM3\ARM_GCC_541\Debug\VCNL4030X01.a(CDC_drv.o)
                0x00001da0                CDC_UpdateStatusBlock
 .text.CDC_HandleSetup
                0x00001dc4       0x5c .\CortexM3\ARM_GCC_541\Debug\VCNL4030X01.a(CDC_drv.o)
                0x00001dc4                CDC_HandleSetup
 .text.CDC_ControlReadStatusStage
                0x00001e20       0x38 .\CortexM3\ARM_GCC_541\Debug\VCNL4030X01.a(CDC_drv.o)
                0x00001e20                CDC_ControlReadStatusStage
 .text.CDC_HandleOUT
                0x00001e58       0x38 .\CortexM3\ARM_GCC_541\Debug\VCNL4030X01.a(CDC_drv.o)
                0x00001e58                CDC_HandleOUT
 .text.CDC_ControlWriteStatusStage
                0x00001e90       0x20 .\CortexM3\ARM_GCC_541\Debug\VCNL4030X01.a(CDC_drv.o)
                0x00001e90                CDC_ControlWriteStatusStage
 .text.CDC_NoDataControlStatusStage
                0x00001eb0       0x40 .\CortexM3\ARM_GCC_541\Debug\VCNL4030X01.a(CDC_drv.o)
                0x00001eb0                CDC_NoDataControlStatusStage
 .text.CDC_HandleIN
                0x00001ef0       0x2c .\CortexM3\ARM_GCC_541\Debug\VCNL4030X01.a(CDC_drv.o)
                0x00001ef0                CDC_HandleIN
 .text.CDC_EP_0_ISR
                0x00001f1c       0xb8 .\CortexM3\ARM_GCC_541\Debug\VCNL4030X01.a(CDC_drv.o)
                0x00001f1c                CDC_EP_0_ISR
 .text.CDC_InitializeStatusBlock
                0x00001fd4       0x24 .\CortexM3\ARM_GCC_541\Debug\VCNL4030X01.a(CDC_drv.o)
                0x00001fd4                CDC_InitializeStatusBlock
 .text.CDC_InitControlRead
                0x00001ff8       0x50 .\CortexM3\ARM_GCC_541\Debug\VCNL4030X01.a(CDC_drv.o)
                0x00001ff8                CDC_InitControlRead
 .text.CDC_InitControlWrite
                0x00002048       0x48 .\CortexM3\ARM_GCC_541\Debug\VCNL4030X01.a(CDC_drv.o)
                0x00002048                CDC_InitControlWrite
 .text.CDC_EP_1_ISR
                0x00002090       0x30 .\CortexM3\ARM_GCC_541\Debug\VCNL4030X01.a(CDC_episr.o)
                0x00002090                CDC_EP_1_ISR
 .text.CDC_EP_2_ISR
                0x000020c0       0x34 .\CortexM3\ARM_GCC_541\Debug\VCNL4030X01.a(CDC_episr.o)
                0x000020c0                CDC_EP_2_ISR
 .text.CDC_EP_3_ISR
                0x000020f4       0x3c .\CortexM3\ARM_GCC_541\Debug\VCNL4030X01.a(CDC_episr.o)
                0x000020f4                CDC_EP_3_ISR
 .text.CDC_SOF_ISR
                0x00002130        0x4 .\CortexM3\ARM_GCC_541\Debug\VCNL4030X01.a(CDC_episr.o)
                0x00002130                CDC_SOF_ISR
 .text.CDC_BUS_RESET_ISR
                0x00002134        0x8 .\CortexM3\ARM_GCC_541\Debug\VCNL4030X01.a(CDC_episr.o)
                0x00002134                CDC_BUS_RESET_ISR
 .text.CDC_DP_ISR
                0x0000213c        0x8 .\CortexM3\ARM_GCC_541\Debug\VCNL4030X01.a(CDC_pm.o)
                0x0000213c                CDC_DP_ISR
 .text.CDC_ReadDieID
                0x00002144       0x6c .\CortexM3\ARM_GCC_541\Debug\VCNL4030X01.a(CDC_std.o)
                0x00002144                CDC_ReadDieID
 .text.CDC_ConfigReg
                0x000021b0       0xa4 .\CortexM3\ARM_GCC_541\Debug\VCNL4030X01.a(CDC_std.o)
                0x000021b0                CDC_ConfigReg
 .text.CDC_GetConfigTablePtr
                0x00002254       0x28 .\CortexM3\ARM_GCC_541\Debug\VCNL4030X01.a(CDC_std.o)
                0x00002254                CDC_GetConfigTablePtr
 .text.CDC_ConfigAltChanged
                0x0000227c      0x11c .\CortexM3\ARM_GCC_541\Debug\VCNL4030X01.a(CDC_std.o)
                0x0000227c                CDC_ConfigAltChanged
 .text.CDC_GetDeviceTablePtr
                0x00002398       0x18 .\CortexM3\ARM_GCC_541\Debug\VCNL4030X01.a(CDC_std.o)
                0x00002398                CDC_GetDeviceTablePtr
 .text.CDC_GetInterfaceClassTablePtr
                0x000023b0       0x28 .\CortexM3\ARM_GCC_541\Debug\VCNL4030X01.a(CDC_std.o)
                0x000023b0                CDC_GetInterfaceClassTablePtr
 .text.CDC_Config
                0x000023d8      0x1ec .\CortexM3\ARM_GCC_541\Debug\VCNL4030X01.a(CDC_std.o)
                0x000023d8                CDC_Config
 .text.CDC_SetEndpointHalt
                0x000025c4       0x64 .\CortexM3\ARM_GCC_541\Debug\VCNL4030X01.a(CDC_std.o)
                0x000025c4                CDC_SetEndpointHalt
 .text.CDC_ClearEndpointHalt
                0x00002628       0xac .\CortexM3\ARM_GCC_541\Debug\VCNL4030X01.a(CDC_std.o)
                0x00002628                CDC_ClearEndpointHalt
 .text.CDC_ValidateAlternateSetting
                0x000026d4       0x4c .\CortexM3\ARM_GCC_541\Debug\VCNL4030X01.a(CDC_std.o)
                0x000026d4                CDC_ValidateAlternateSetting
 .text.CDC_HandleStandardRqst
                0x00002720      0x354 .\CortexM3\ARM_GCC_541\Debug\VCNL4030X01.a(CDC_std.o)
                0x00002720                CDC_HandleStandardRqst
 .text.CDC_HandleVendorRqst
                0x00002a74       0x18 .\CortexM3\ARM_GCC_541\Debug\VCNL4030X01.a(CDC_vnd.o)
                0x00002a74                CDC_HandleVendorRqst
 .text.CDC_Dp_ClearInterrupt
                0x00002a8c       0x10 .\CortexM3\ARM_GCC_541\Debug\VCNL4030X01.a(CDC_Dp.o)
                0x00002a8c                CDC_Dp_ClearInterrupt
 .text.CyHalt   0x00002a9c        0x4 .\CortexM3\ARM_GCC_541\Debug\VCNL4030X01.a(CyLib.o)
                0x00002a9c                CyHalt
 .text.CyDelay  0x00002aa0       0x2c .\CortexM3\ARM_GCC_541\Debug\VCNL4030X01.a(CyLib.o)
                0x00002aa0                CyDelay
 .text.CyDelayUs
                0x00002acc       0x14 .\CortexM3\ARM_GCC_541\Debug\VCNL4030X01.a(CyLib.o)
                0x00002acc                CyDelayUs
 .text.CyIntSetVector
                0x00002ae0       0x28 .\CortexM3\ARM_GCC_541\Debug\VCNL4030X01.a(CyLib.o)
                0x00002ae0                CyIntSetVector
 .text.CyIntSetPriority
                0x00002b08       0x30 .\CortexM3\ARM_GCC_541\Debug\VCNL4030X01.a(CyLib.o)
                0x00002b08                CyIntSetPriority
 .text.CyGetUniqueId
                0x00002b38       0x70 .\CortexM3\ARM_GCC_541\Debug\VCNL4030X01.a(CyLib.o)
                0x00002b38                CyGetUniqueId
 .text          0x00002ba8       0x20 .\CortexM3\ARM_GCC_541\Debug\VCNL4030X01.a(CyBootAsmGnu.o)
                0x00002ba8                CyDelayCycles
                0x00002bb8                CyEnterCriticalSection
                0x00002bc0                CyExitCriticalSection
 .text.CDC_DispatchClassRqst
                0x00002bc8       0x60 .\CortexM3\ARM_GCC_541\Debug\VCNL4030X01.a(CDC_cls.o)
                0x00002bc8                CDC_DispatchClassRqst
 .text.pow      0x00002c28      0x330 c:/program files (x86)/cypress/psoc creator/4.3/psoc creator/import/gnu/arm/5.4.1/bin/../lib/gcc/arm-none-eabi/5.4.1/../../../../arm-none-eabi/lib/armv7-m\libm.a(lib_a-w_pow.o)
                0x00002c28                pow
 .text.__ieee754_pow
                0x00002f58      0xac4 c:/program files (x86)/cypress/psoc creator/4.3/psoc creator/import/gnu/arm/5.4.1/bin/../lib/gcc/arm-none-eabi/5.4.1/../../../../arm-none-eabi/lib/armv7-m\libm.a(lib_a-e_pow.o)
                0x00002f58                __ieee754_pow
 .text.__ieee754_sqrt
                0x00003a1c      0x188 c:/program files (x86)/cypress/psoc creator/4.3/psoc creator/import/gnu/arm/5.4.1/bin/../lib/gcc/arm-none-eabi/5.4.1/../../../../arm-none-eabi/lib/armv7-m\libm.a(lib_a-e_sqrt.o)
                0x00003a1c                __ieee754_sqrt
 .text.fabs     0x00003ba4        0x8 c:/program files (x86)/cypress/psoc creator/4.3/psoc creator/import/gnu/arm/5.4.1/bin/../lib/gcc/arm-none-eabi/5.4.1/../../../../arm-none-eabi/lib/armv7-m\libm.a(lib_a-s_fabs.o)
                0x00003ba4                fabs
 .text.finite   0x00003bac        0xc c:/program files (x86)/cypress/psoc creator/4.3/psoc creator/import/gnu/arm/5.4.1/bin/../lib/gcc/arm-none-eabi/5.4.1/../../../../arm-none-eabi/lib/armv7-m\libm.a(lib_a-s_finite.o)
                0x00003bac                finite
 .text.matherr  0x00003bb8        0x4 c:/program files (x86)/cypress/psoc creator/4.3/psoc creator/import/gnu/arm/5.4.1/bin/../lib/gcc/arm-none-eabi/5.4.1/../../../../arm-none-eabi/lib/armv7-m\libm.a(lib_a-s_matherr.o)
                0x00003bb8                matherr
 .text.nan      0x00003bbc        0xc c:/program files (x86)/cypress/psoc creator/4.3/psoc creator/import/gnu/arm/5.4.1/bin/../lib/gcc/arm-none-eabi/5.4.1/../../../../arm-none-eabi/lib/armv7-m\libm.a(lib_a-s_nan.o)
                0x00003bbc                nan
 .text.rint     0x00003bc8      0x120 c:/program files (x86)/cypress/psoc creator/4.3/psoc creator/import/gnu/arm/5.4.1/bin/../lib/gcc/arm-none-eabi/5.4.1/../../../../arm-none-eabi/lib/armv7-m\libm.a(lib_a-s_rint.o)
                0x00003bc8                rint
 .text.scalbn   0x00003ce8       0xe4 c:/program files (x86)/cypress/psoc creator/4.3/psoc creator/import/gnu/arm/5.4.1/bin/../lib/gcc/arm-none-eabi/5.4.1/../../../../arm-none-eabi/lib/armv7-m\libm.a(lib_a-s_scalbn.o)
                0x00003ce8                scalbn
 .text.copysign
                0x00003dcc       0x10 c:/program files (x86)/cypress/psoc creator/4.3/psoc creator/import/gnu/arm/5.4.1/bin/../lib/gcc/arm-none-eabi/5.4.1/../../../../arm-none-eabi/lib/armv7-m\libm.a(lib_a-s_copysign.o)
                0x00003dcc                copysign
 .text          0x00003ddc      0x370 c:/program files (x86)/cypress/psoc creator/4.3/psoc creator/import/gnu/arm/5.4.1/bin/../lib/gcc/arm-none-eabi/5.4.1/armv7-m\libgcc.a(_arm_addsubdf3.o)
                0x00003ddc                __aeabi_drsub
                0x00003de4                __aeabi_dsub
                0x00003de4                __subdf3
                0x00003de8                __aeabi_dadd
                0x00003de8                __adddf3
                0x00004060                __floatunsidf
                0x00004060                __aeabi_ui2d
                0x00004080                __floatsidf
                0x00004080                __aeabi_i2d
                0x000040a4                __aeabi_f2d
                0x000040a4                __extendsfdf2
                0x000040e0                __floatundidf
                0x000040e0                __aeabi_ul2d
                0x000040f0                __floatdidf
                0x000040f0                __aeabi_l2d
 .text          0x0000414c      0x424 c:/program files (x86)/cypress/psoc creator/4.3/psoc creator/import/gnu/arm/5.4.1/bin/../lib/gcc/arm-none-eabi/5.4.1/armv7-m\libgcc.a(_arm_muldivdf3.o)
                0x0000414c                __aeabi_dmul
                0x0000414c                __muldf3
                0x000043a0                __divdf3
                0x000043a0                __aeabi_ddiv
 .text          0x00004570      0x110 c:/program files (x86)/cypress/psoc creator/4.3/psoc creator/import/gnu/arm/5.4.1/bin/../lib/gcc/arm-none-eabi/5.4.1/armv7-m\libgcc.a(_arm_cmpdf2.o)
                0x00004570                __gtdf2
                0x00004570                __gedf2
                0x00004578                __ltdf2
                0x00004578                __ledf2
                0x00004580                __nedf2
                0x00004580                __eqdf2
                0x00004580                __cmpdf2
                0x000045fc                __aeabi_cdrcmple
                0x0000460c                __aeabi_cdcmpeq
                0x0000460c                __aeabi_cdcmple
                0x0000461c                __aeabi_dcmpeq
                0x00004630                __aeabi_dcmplt
                0x00004644                __aeabi_dcmple
                0x00004658                __aeabi_dcmpge
                0x0000466c                __aeabi_dcmpgt
 .text          0x00004680       0x2c c:/program files (x86)/cypress/psoc creator/4.3/psoc creator/import/gnu/arm/5.4.1/bin/../lib/gcc/arm-none-eabi/5.4.1/armv7-m\libgcc.a(_arm_unorddf2.o)
                0x00004680                __unorddf2
                0x00004680                __aeabi_dcmpun
 .text          0x000046ac       0xa0 c:/program files (x86)/cypress/psoc creator/4.3/psoc creator/import/gnu/arm/5.4.1/bin/../lib/gcc/arm-none-eabi/5.4.1/armv7-m\libgcc.a(_arm_truncdfsf2.o)
                0x000046ac                __truncdfsf2
                0x000046ac                __aeabi_d2f
 .text          0x0000474c      0x21c c:/program files (x86)/cypress/psoc creator/4.3/psoc creator/import/gnu/arm/5.4.1/bin/../lib/gcc/arm-none-eabi/5.4.1/armv7-m\libgcc.a(_arm_addsubsf3.o)
                0x0000474c                __aeabi_frsub
                0x00004754                __subsf3
                0x00004754                __aeabi_fsub
                0x00004758                __aeabi_fadd
                0x00004758                __addsf3
                0x000048b8                __aeabi_ui2f
                0x000048b8                __floatunsisf
                0x000048c0                __aeabi_i2f
                0x000048c0                __floatsisf
                0x000048dc                __aeabi_ul2f
                0x000048dc                __floatundisf
                0x000048ec                __aeabi_l2f
                0x000048ec                __floatdisf
 .text          0x00004968      0x2a0 c:/program files (x86)/cypress/psoc creator/4.3/psoc creator/import/gnu/arm/5.4.1/bin/../lib/gcc/arm-none-eabi/5.4.1/armv7-m\libgcc.a(_arm_muldivsf3.o)
                0x00004968                __mulsf3
                0x00004968                __aeabi_fmul
                0x00004ad0                __aeabi_fdiv
                0x00004ad0                __divsf3
 .text          0x00004c08       0x4c c:/program files (x86)/cypress/psoc creator/4.3/psoc creator/import/gnu/arm/5.4.1/bin/../lib/gcc/arm-none-eabi/5.4.1/armv7-m\libgcc.a(_arm_fixsfsi.o)
                0x00004c08                __aeabi_f2iz
                0x00004c08                __fixsfsi
 .text.__errno  0x00004c54        0xc c:/program files (x86)/cypress/psoc creator/4.3/psoc creator/import/gnu/arm/5.4.1/bin/../lib/gcc/arm-none-eabi/5.4.1/../../../../arm-none-eabi/lib/armv7-m\libg_nano.a(lib_a-errno.o)
                0x00004c54                __errno
 .text.__libc_init_array
                0x00004c60       0x4c c:/program files (x86)/cypress/psoc creator/4.3/psoc creator/import/gnu/arm/5.4.1/bin/../lib/gcc/arm-none-eabi/5.4.1/../../../../arm-none-eabi/lib/armv7-m\libg_nano.a(lib_a-init.o)
                0x00004c60                __libc_init_array
 .text.memcpy   0x00004cac       0x16 c:/program files (x86)/cypress/psoc creator/4.3/psoc creator/import/gnu/arm/5.4.1/bin/../lib/gcc/arm-none-eabi/5.4.1/../../../../arm-none-eabi/lib/armv7-m\libg_nano.a(lib_a-memcpy-stub.o)
                0x00004cac                memcpy
 .text.memset   0x00004cc2       0x10 c:/program files (x86)/cypress/psoc creator/4.3/psoc creator/import/gnu/arm/5.4.1/bin/../lib/gcc/arm-none-eabi/5.4.1/../../../../arm-none-eabi/lib/armv7-m\libg_nano.a(lib_a-memset.o)
                0x00004cc2                memset
 *fill*         0x00004cd2        0x2 
 .text.sprintf  0x00004cd4       0x48 c:/program files (x86)/cypress/psoc creator/4.3/psoc creator/import/gnu/arm/5.4.1/bin/../lib/gcc/arm-none-eabi/5.4.1/../../../../arm-none-eabi/lib/armv7-m\libg_nano.a(lib_a-sprintf.o)
                0x00004cd4                siprintf
                0x00004cd4                sprintf
 .text.__ssputs_r
                0x00004d1c       0xb2 c:/program files (x86)/cypress/psoc creator/4.3/psoc creator/import/gnu/arm/5.4.1/bin/../lib/gcc/arm-none-eabi/5.4.1/../../../../arm-none-eabi/lib/armv7-m\libg_nano.a(lib_a-nano-svfprintf.o)
                0x00004d1c                __ssputs_r
 *fill*         0x00004dce        0x2 
 .text._svfprintf_r
                0x00004dd0      0x1e8 c:/program files (x86)/cypress/psoc creator/4.3/psoc creator/import/gnu/arm/5.4.1/bin/../lib/gcc/arm-none-eabi/5.4.1/../../../../arm-none-eabi/lib/armv7-m\libg_nano.a(lib_a-nano-svfprintf.o)
                0x00004dd0                _svfiprintf_r
                0x00004dd0                _svfprintf_r
 .text._printf_common
                0x00004fb8       0xec c:/program files (x86)/cypress/psoc creator/4.3/psoc creator/import/gnu/arm/5.4.1/bin/../lib/gcc/arm-none-eabi/5.4.1/../../../../arm-none-eabi/lib/armv7-m\libg_nano.a(lib_a-nano-vfprintf_i.o)
                0x00004fb8                _printf_common
 .text._printf_i
                0x000050a4      0x24c c:/program files (x86)/cypress/psoc creator/4.3/psoc creator/import/gnu/arm/5.4.1/bin/../lib/gcc/arm-none-eabi/5.4.1/../../../../arm-none-eabi/lib/armv7-m\libg_nano.a(lib_a-nano-vfprintf_i.o)
                0x000050a4                _printf_i
 .text.memchr   0x000052f0       0x1c c:/program files (x86)/cypress/psoc creator/4.3/psoc creator/import/gnu/arm/5.4.1/bin/../lib/gcc/arm-none-eabi/5.4.1/../../../../arm-none-eabi/lib/armv7-m\libg_nano.a(lib_a-memchr-stub.o)
                0x000052f0                memchr
 .text.memmove  0x0000530c       0x36 c:/program files (x86)/cypress/psoc creator/4.3/psoc creator/import/gnu/arm/5.4.1/bin/../lib/gcc/arm-none-eabi/5.4.1/../../../../arm-none-eabi/lib/armv7-m\libg_nano.a(lib_a-memmove.o)
                0x0000530c                memmove
 *fill*         0x00005342        0x2 
 .text._free_r  0x00005344       0x98 c:/program files (x86)/cypress/psoc creator/4.3/psoc creator/import/gnu/arm/5.4.1/bin/../lib/gcc/arm-none-eabi/5.4.1/../../../../arm-none-eabi/lib/armv7-m\libg_nano.a(lib_a-nano-freer.o)
                0x00005344                _free_r
 .text._malloc_r
                0x000053dc       0xbc c:/program files (x86)/cypress/psoc creator/4.3/psoc creator/import/gnu/arm/5.4.1/bin/../lib/gcc/arm-none-eabi/5.4.1/../../../../arm-none-eabi/lib/armv7-m\libg_nano.a(lib_a-nano-mallocr.o)
                0x000053dc                _malloc_r
 .text._realloc_r
                0x00005498       0x4c c:/program files (x86)/cypress/psoc creator/4.3/psoc creator/import/gnu/arm/5.4.1/bin/../lib/gcc/arm-none-eabi/5.4.1/../../../../arm-none-eabi/lib/armv7-m\libg_nano.a(lib_a-nano-reallocr.o)
                0x00005498                _realloc_r
 .text._sbrk_r  0x000054e4       0x20 c:/program files (x86)/cypress/psoc creator/4.3/psoc creator/import/gnu/arm/5.4.1/bin/../lib/gcc/arm-none-eabi/5.4.1/../../../../arm-none-eabi/lib/armv7-m\libg_nano.a(lib_a-sbrkr.o)
                0x000054e4                _sbrk_r
 .text.__malloc_lock
                0x00005504        0x2 c:/program files (x86)/cypress/psoc creator/4.3/psoc creator/import/gnu/arm/5.4.1/bin/../lib/gcc/arm-none-eabi/5.4.1/../../../../arm-none-eabi/lib/armv7-m\libg_nano.a(lib_a-mlock.o)
                0x00005504                __malloc_lock
 .text.__malloc_unlock
                0x00005506        0x2 c:/program files (x86)/cypress/psoc creator/4.3/psoc creator/import/gnu/arm/5.4.1/bin/../lib/gcc/arm-none-eabi/5.4.1/../../../../arm-none-eabi/lib/armv7-m\libg_nano.a(lib_a-mlock.o)
                0x00005506                __malloc_unlock
 .text._malloc_usable_size_r
                0x00005508       0x14 c:/program files (x86)/cypress/psoc creator/4.3/psoc creator/import/gnu/arm/5.4.1/bin/../lib/gcc/arm-none-eabi/5.4.1/../../../../arm-none-eabi/lib/armv7-m\libg_nano.a(lib_a-nano-msizer.o)
                0x00005508                _malloc_usable_size_r
 *(.plt)
 *(.gnu.warning)
 *(.glue_7t)
 .glue_7t       0x0000551c        0x0 linker stubs
 *(.glue_7)
 .glue_7        0x0000551c        0x0 linker stubs
 *(.vfp11_veneer)
 .vfp11_veneer  0x0000551c        0x0 linker stubs
 *(.bootloader)
 *(.ARM.extab* .gnu.linkonce.armextab.*)
 *(.gcc_except_table)

.v4_bx          0x0000551c        0x0
 .v4_bx         0x0000551c        0x0 linker stubs

.iplt           0x0000551c        0x0
 .iplt          0x0000551c        0x0 c:/program files (x86)/cypress/psoc creator/4.3/psoc creator/import/gnu/arm/5.4.1/bin/../lib/gcc/arm-none-eabi/5.4.1/armv7-m/crtbegin.o

.eh_frame_hdr
 *(.eh_frame_hdr)

.eh_frame       0x0000551c        0x4
 *(.eh_frame)
 .eh_frame      0x0000551c        0x0 c:/program files (x86)/cypress/psoc creator/4.3/psoc creator/import/gnu/arm/5.4.1/bin/../lib/gcc/arm-none-eabi/5.4.1/armv7-m/crtbegin.o
 .eh_frame      0x0000551c        0x4 c:/program files (x86)/cypress/psoc creator/4.3/psoc creator/import/gnu/arm/5.4.1/bin/../lib/gcc/arm-none-eabi/5.4.1/armv7-m/crtend.o
                [!provide]                PROVIDE (__exidx_start, .)

.ARM.exidx
 *(.ARM.exidx* .gnu.linkonce.armexidx.*)
                0x00005520                __exidx_end = .

.rodata         0x00005520      0x668
 *(.rodata .rodata.* .gnu.linkonce.r.*)
 .rodata.str1.4
                0x00005520      0x43d .\CortexM3\ARM_GCC_541\Debug\VCNL4030X01_Application_Library.o
 *fill*         0x0000595d        0x3 
 .rodata        0x00005960       0x30 .\CortexM3\ARM_GCC_541\Debug\cyfitter_cfg.o
 .rodata.str1.4
                0x00005990       0x11 .\CortexM3\ARM_GCC_541\Debug\VCNL4030X01.a(CDC_std.o)
 *fill*         0x000059a1        0x3 
 .rodata        0x000059a4      0x15e .\CortexM3\ARM_GCC_541\Debug\VCNL4030X01.a(CDC_descr.o)
                0x000059a4                CDC_TABLE
                0x000059ac                CDC_DEVICE0_TABLE
                0x000059c4                CDC_DEVICE0_CONFIGURATION0_TABLE
                0x000059ec                CDC_DEVICE0_CONFIGURATION0_INTERFACE_CLASS
                0x000059f0                CDC_DEVICE0_CONFIGURATION0_EP_SETTINGS_TABLE
                0x00005a08                CDC_SN_STRING_DESCRIPTOR
                0x00005a0c                CDC_STRING_DESCRIPTORS
                0x00005aac                CDC_DEVICE0_CONFIGURATION0_DESCR
                0x00005af0                CDC_DEVICE0_DESCR
 *fill*         0x00005b02        0x2 
 .rodata.str1.4
                0x00005b04        0x4 c:/program files (x86)/cypress/psoc creator/4.3/psoc creator/import/gnu/arm/5.4.1/bin/../lib/gcc/arm-none-eabi/5.4.1/../../../../arm-none-eabi/lib/armv7-m\libm.a(lib_a-w_pow.o)
 .rodata.str1.4
                0x00005b08        0x4 c:/program files (x86)/cypress/psoc creator/4.3/psoc creator/import/gnu/arm/5.4.1/bin/../lib/gcc/arm-none-eabi/5.4.1/../../../../arm-none-eabi/lib/armv7-m\libm.a(lib_a-e_pow.o)
                                  0x1 (size before relaxing)
 .rodata.TWO52  0x00005b08       0x10 c:/program files (x86)/cypress/psoc creator/4.3/psoc creator/import/gnu/arm/5.4.1/bin/../lib/gcc/arm-none-eabi/5.4.1/../../../../arm-none-eabi/lib/armv7-m\libm.a(lib_a-s_rint.o)
 .rodata.str1.1
                0x00005b18        0x2 c:/program files (x86)/cypress/psoc creator/4.3/psoc creator/import/gnu/arm/5.4.1/bin/../lib/gcc/arm-none-eabi/5.4.1/../../../../arm-none-eabi/lib/armv7-m\libg_nano.a(lib_a-impure.o)
 .rodata.str1.1
                0x00005b1a       0x11 c:/program files (x86)/cypress/psoc creator/4.3/psoc creator/import/gnu/arm/5.4.1/bin/../lib/gcc/arm-none-eabi/5.4.1/../../../../arm-none-eabi/lib/armv7-m\libg_nano.a(lib_a-nano-svfprintf.o)
 .rodata.str1.1
                0x00005b2b       0x22 c:/program files (x86)/cypress/psoc creator/4.3/psoc creator/import/gnu/arm/5.4.1/bin/../lib/gcc/arm-none-eabi/5.4.1/../../../../arm-none-eabi/lib/armv7-m\libg_nano.a(lib_a-nano-vfprintf_i.o)
                0x00005b50                . = ALIGN (0x4)
 *fill*         0x00005b4d        0x3 
 *(.init)
 .init          0x00005b50        0x4 c:/program files (x86)/cypress/psoc creator/4.3/psoc creator/import/gnu/arm/5.4.1/bin/../lib/gcc/arm-none-eabi/5.4.1/armv7-m/crti.o
                0x00005b50                _init
 .init          0x00005b54        0x8 c:/program files (x86)/cypress/psoc creator/4.3/psoc creator/import/gnu/arm/5.4.1/bin/../lib/gcc/arm-none-eabi/5.4.1/armv7-m/crtn.o
                0x00005b5c                . = ALIGN (0x4)
                0x00005b5c                __preinit_array_start = .
 *(.preinit_array)
                0x00005b5c                __preinit_array_end = .
                0x00005b5c                . = ALIGN (0x4)
                0x00005b5c                __init_array_start = .
 *(SORT(.init_array.*))
 *(.init_array)
 .init_array    0x00005b5c        0x4 c:/program files (x86)/cypress/psoc creator/4.3/psoc creator/import/gnu/arm/5.4.1/bin/../lib/gcc/arm-none-eabi/5.4.1/armv7-m/crtbegin.o
 .init_array    0x00005b60        0x4 .\CortexM3\ARM_GCC_541\Debug\Cm3Start.o
                0x00005b64                __init_array_end = .
                0x00005b64                . = ALIGN (0x4)
 *(.fini)
 .fini          0x00005b64        0x4 c:/program files (x86)/cypress/psoc creator/4.3/psoc creator/import/gnu/arm/5.4.1/bin/../lib/gcc/arm-none-eabi/5.4.1/armv7-m/crti.o
                0x00005b64                _fini
 .fini          0x00005b68        0x8 c:/program files (x86)/cypress/psoc creator/4.3/psoc creator/import/gnu/arm/5.4.1/bin/../lib/gcc/arm-none-eabi/5.4.1/armv7-m/crtn.o
                0x00005b70                . = ALIGN (0x4)
                0x00005b70                __fini_array_start = .
 *(.fini_array)
 .fini_array    0x00005b70        0x4 c:/program files (x86)/cypress/psoc creator/4.3/psoc creator/import/gnu/arm/5.4.1/bin/../lib/gcc/arm-none-eabi/5.4.1/armv7-m/crtbegin.o
 *(SORT(.fini_array.*))
                0x00005b74                __fini_array_end = .
                0x00005b74                . = ALIGN (0x4)
 *crtbegin.o(.ctors)
 *(EXCLUDE_FILE(*crtend.o) .ctors)
 *(SORT(.ctors.*))
 *crtend.o(.ctors)
                0x00005b74                . = ALIGN (0x4)
 *crtbegin.o(.dtors)
 *(EXCLUDE_FILE(*crtend.o) .dtors)
 *(SORT(.dtors.*))
 *crtend.o(.dtors)
                0x00005b74                . = ALIGN (0x4)
                0x00005b74                __cy_regions = .
                0x00005b74        0x4 LONG 0x5b88 __cy_region_init_ram
                0x00005b78        0x4 LONG 0x1fff80c8 __cy_region_start_data
                0x00005b7c        0x4 LONG 0xa8 __cy_region_init_size_ram
                0x00005b80        0x4 LONG 0x120 __cy_region_zero_size_ram
                0x00005b84                __cy_regions_end = .
                0x00005b88                . = ALIGN (0x8)
 *fill*         0x00005b84        0x4 
                0x00005b88                _etext = .

.cy_checksum_exclude
                0x00005b88        0x0
 *(.cy_checksum_exclude)

.ramvectors     0x1fff8000       0xc0
                0x1fff8000                __cy_region_start_ram = .
 *(.ramvectors)
 .ramvectors    0x1fff8000       0xc0 .\CortexM3\ARM_GCC_541\Debug\Cm3Start.o
                0x1fff8000                CyRamVectors

.noinit         0x1fff80c0        0x1
 *(.noinit)
 .noinit        0x1fff80c0        0x1 .\CortexM3\ARM_GCC_541\Debug\VCNL4030X01.a(CyLib.o)
                0x1fff80c0                CyResetStatus

.data           0x1fff80c8       0xa8 load address 0x00005b88
                0x1fff80c8                __cy_region_start_data = .
 *(.jcr)
 .jcr           0x1fff80c8        0x0 c:/program files (x86)/cypress/psoc creator/4.3/psoc creator/import/gnu/arm/5.4.1/bin/../lib/gcc/arm-none-eabi/5.4.1/armv7-m/crtbegin.o
 .jcr           0x1fff80c8        0x4 c:/program files (x86)/cypress/psoc creator/4.3/psoc creator/import/gnu/arm/5.4.1/bin/../lib/gcc/arm-none-eabi/5.4.1/armv7-m/crtend.o
 *(.got.plt)
 *(.got)
 *(.shdata)
 *(.data .data.* .gnu.linkonce.d.*)
 .data          0x1fff80cc        0x8 .\CortexM3\ARM_GCC_541\Debug\main.o
                0x1fff80cc                AverageCount
                0x1fff80d0                I2C_Bus
 .data          0x1fff80d4        0x4 .\CortexM3\ARM_GCC_541\Debug\Cm3Start.o
 .data          0x1fff80d8       0x1a .\CortexM3\ARM_GCC_541\Debug\VCNL4030X01.a(CDC_cdc.o)
                0x1fff80d8                CDC_linesCoding
 *fill*         0x1fff80f2        0x2 
 .data          0x1fff80f4       0x10 .\CortexM3\ARM_GCC_541\Debug\VCNL4030X01.a(CyLib.o)
                0x1fff80f4                cydelay_32k_ms
                0x1fff80f8                cydelay_freq_khz
                0x1fff80fc                cydelay_freq_mhz
                0x1fff8100                cydelay_freq_hz
 .data.__fdlib_version
                0x1fff8104        0x1 c:/program files (x86)/cypress/psoc creator/4.3/psoc creator/import/gnu/arm/5.4.1/bin/../lib/gcc/arm-none-eabi/5.4.1/../../../../arm-none-eabi/lib/armv7-m\libm.a(lib_a-s_lib_ver.o)
                0x1fff8104                __fdlib_version
 *fill*         0x1fff8105        0x3 
 .data.impure_data
                0x1fff8108       0x60 c:/program files (x86)/cypress/psoc creator/4.3/psoc creator/import/gnu/arm/5.4.1/bin/../lib/gcc/arm-none-eabi/5.4.1/../../../../arm-none-eabi/lib/armv7-m\libg_nano.a(lib_a-impure.o)
 .data._impure_ptr
                0x1fff8168        0x4 c:/program files (x86)/cypress/psoc creator/4.3/psoc creator/import/gnu/arm/5.4.1/bin/../lib/gcc/arm-none-eabi/5.4.1/../../../../arm-none-eabi/lib/armv7-m\libg_nano.a(lib_a-impure.o)
                0x1fff8168                _impure_ptr
                0x1fff8170                . = ALIGN (0x8)
 *fill*         0x1fff816c        0x4 
 *(.ram)
                0x1fff8170                _edata = .

.igot.plt       0x1fff8170        0x0 load address 0x00005c30
 .igot.plt      0x1fff8170        0x0 c:/program files (x86)/cypress/psoc creator/4.3/psoc creator/import/gnu/arm/5.4.1/bin/../lib/gcc/arm-none-eabi/5.4.1/armv7-m/crtbegin.o

.bss            0x1fff8170      0x120 load address 0x00005c30
                0x1fff8170                PROVIDE (__bss_start__, .)
 *(.shbss)
 *(.bss .bss.* .gnu.linkonce.b.*)
 .bss           0x1fff8170       0x1c c:/program files (x86)/cypress/psoc creator/4.3/psoc creator/import/gnu/arm/5.4.1/bin/../lib/gcc/arm-none-eabi/5.4.1/armv7-m/crtbegin.o
 .bss           0x1fff818c        0x1 .\CortexM3\ARM_GCC_541\Debug\VCNL4030X01.a(I2C_1.o)
                0x1fff818c                I2C_1_initVar
 .bss           0x1fff818d        0x1 .\CortexM3\ARM_GCC_541\Debug\VCNL4030X01.a(CDC.o)
                0x1fff818d                CDC_initVar
 .bss           0x1fff818e        0x1 .\CortexM3\ARM_GCC_541\Debug\VCNL4030X01.a(CDC_cdc.o)
 *fill*         0x1fff818f        0x1 
 .bss           0x1fff8190        0x2 .\CortexM3\ARM_GCC_541\Debug\VCNL4030X01.a(CDC_std.o)
 *fill*         0x1fff8192        0x2 
 .bss.__malloc_sbrk_start
                0x1fff8194        0x4 c:/program files (x86)/cypress/psoc creator/4.3/psoc creator/import/gnu/arm/5.4.1/bin/../lib/gcc/arm-none-eabi/5.4.1/../../../../arm-none-eabi/lib/armv7-m\libg_nano.a(lib_a-nano-mallocr.o)
                0x1fff8194                __malloc_sbrk_start
 .bss.__malloc_free_list
                0x1fff8198        0x4 c:/program files (x86)/cypress/psoc creator/4.3/psoc creator/import/gnu/arm/5.4.1/bin/../lib/gcc/arm-none-eabi/5.4.1/../../../../arm-none-eabi/lib/armv7-m\libg_nano.a(lib_a-nano-mallocr.o)
                0x1fff8198                __malloc_free_list
 *(COMMON)
 COMMON         0x1fff819c        0x1 .\CortexM3\ARM_GCC_541\Debug\VCNL4030X01.a(I2C_1.o)
                0x1fff819c                I2C_1_state
 *fill*         0x1fff819d        0x3 
 COMMON         0x1fff81a0       0x11 .\CortexM3\ARM_GCC_541\Debug\VCNL4030X01.a(I2C_1_MASTER.o)
                0x1fff81a0                I2C_1_mstrWrBufIndex
                0x1fff81a1                I2C_1_mstrControl
                0x1fff81a2                I2C_1_mstrStatus
                0x1fff81a3                I2C_1_mstrWrBufSize
                0x1fff81a4                I2C_1_mstrRdBufIndex
                0x1fff81a8                I2C_1_mstrWrBufPtr
                0x1fff81ac                I2C_1_mstrRdBufPtr
                0x1fff81b0                I2C_1_mstrRdBufSize
 *fill*         0x1fff81b1        0x3 
 COMMON         0x1fff81b4       0x18 .\CortexM3\ARM_GCC_541\Debug\VCNL4030X01.a(CDC_cdc.o)
                0x1fff81b4                CDC_linesControlBitmap
                0x1fff81b8                CDC_cdcDataOutEp
                0x1fff81bc                CDC_linesChanged
                0x1fff81c0                CDC_cdcCommInInterruptEp
                0x1fff81c4                CDC_cdcDataInEp
                0x1fff81c8                CDC_serialStateBitmap
 COMMON         0x1fff81cc       0x9b .\CortexM3\ARM_GCC_541\Debug\VCNL4030X01.a(CDC_drv.o)
                0x1fff81cc                CDC_device
                0x1fff81d0                CDC_interfaceSettingLast
                0x1fff81d4                CDC_EP
                0x1fff8240                CDC_transferState
                0x1fff8241                CDC_ep0Toggle
                0x1fff8242                CDC_configurationChanged
                0x1fff8243                CDC_ep0Count
                0x1fff8244                CDC_deviceStatus
                0x1fff8245                CDC_configuration
                0x1fff8248                CDC_interfaceClass
                0x1fff824c                CDC_ep0Mode
                0x1fff8250                CDC_interfaceStatus
                0x1fff8252                CDC_transferByteCount
                0x1fff8254                CDC_currentTD
                0x1fff8260                CDC_deviceAddress
                0x1fff8261                CDC_interfaceNumber
                0x1fff8264                CDC_interfaceSetting
                0x1fff8266                CDC_lastPacketSize
 *fill*         0x1fff8267        0x1 
 COMMON         0x1fff8268       0x22 .\CortexM3\ARM_GCC_541\Debug\VCNL4030X01.a(CDC_descr.o)
                0x1fff8268                CDC_idSerialNumberStringDescriptor
 *fill*         0x1fff828a        0x2 
 COMMON         0x1fff828c        0x4 c:/program files (x86)/cypress/psoc creator/4.3/psoc creator/import/gnu/arm/5.4.1/bin/../lib/gcc/arm-none-eabi/5.4.1/../../../../arm-none-eabi/lib/armv7-m\libg_nano.a(lib_a-reent.o)
                0x1fff828c                errno
                0x1fff8290                . = ALIGN (0x8)
 *(.ram.b)
                0x1fff8290                _end = .
                0x1fff8290                __end = .
                0x1fff8290                PROVIDE (end, .)
                0x1fff8290                PROVIDE (__bss_end__, .)
                0x00005b88                __cy_region_init_ram = LOADADDR (.data)
                0x000000a8                __cy_region_init_size_ram = (_edata - ADDR (.data))
                0x00000120                __cy_region_zero_size_ram = (_end - _edata)

.heap           0x1fff8290       0x80 load address 0x00005c30
                0x1fff8290                . = _end
                0x1fff8310                . = (. + 0x80)
 *fill*         0x1fff8290       0x80 
                0x1fff8310                __cy_heap_limit = .

.stack          0x20007800      0x800
                0x20007800                __cy_stack_limit = .
                0x20008000                . = (. + 0x800)
 *fill*         0x20007800      0x800 
                0x00000001                ASSERT ((__cy_stack_limit >= __cy_heap_limit), region RAM overflowed with stack)
                0x00000000                cy_checksum_exclude_size = (CY_APPL_LOADABLE == 0x1)?SIZEOF (.cy_checksum_exclude):0x0
                0x00000001                ASSERT ((cy_checksum_exclude_size <= CY_CHECKSUM_EXCLUDE_SIZE), CY_BOOT: Section .cy_checksum_exclude size exceedes specified limit.)

.cyloadermeta
 *(.cyloadermeta)

.cyloadablemeta
 *(.cyloadablemeta)

.cyconfigecc    0x80000000       0xf4
 *(.cyconfigecc)
 .cyconfigecc   0x80000000       0xf4 .\CortexM3\ARM_GCC_541\Debug\cymetadata.o
                0x80000000                cy_meta_configecc

.cycustnvl      0x90000000        0x4
 *(.cycustnvl)
 .cycustnvl     0x90000000        0x4 .\CortexM3\ARM_GCC_541\Debug\cymetadata.o
                0x90000000                cy_meta_custnvl

.cywolatch      0x90100000        0x4
 *(.cywolatch)
 .cywolatch     0x90100000        0x4 .\CortexM3\ARM_GCC_541\Debug\cymetadata.o
                0x90100000                cy_meta_wonvl

.cyeeprom       0x90200000        0x0
 *(.cyeeprom)
                0x00000001                ASSERT ((. <= ((0x90200000 + ee_offset) + ee_size)), .cyeeprom data will not fit in EEPROM)

.cyflashprotect
                0x90400000      0x100
 *(.cyflashprotect)
 .cyflashprotect
                0x90400000      0x100 .\CortexM3\ARM_GCC_541\Debug\cymetadata.o
                0x90400000                cy_meta_flashprotect

.cymeta         0x90500000        0xc
 *(.cymeta)
 .cymeta        0x90500000        0xc .\CortexM3\ARM_GCC_541\Debug\cymetadata.o
                0x90500000                cy_metadata

.rel.dyn        0x00005c30        0x0 load address 0x9050000c
 .rel.iplt      0x00005c30        0x0 c:/program files (x86)/cypress/psoc creator/4.3/psoc creator/import/gnu/arm/5.4.1/bin/../lib/gcc/arm-none-eabi/5.4.1/armv7-m/crtbegin.o

.stab
 *(.stab)

.stabstr
 *(.stabstr)

.debug
 *(.debug)

.line
 *(.line)

.debug_srcinfo
 *(.debug_srcinfo)

.debug_sfnames
 *(.debug_sfnames)

.debug_aranges  0x00000000      0xc98
 *(.debug_aranges)
 .debug_aranges
                0x00000000       0x50 .\CortexM3\ARM_GCC_541\Debug\main.o
 .debug_aranges
                0x00000050       0x28 .\CortexM3\ARM_GCC_541\Debug\I2C_Functions.o
 .debug_aranges
                0x00000078       0xf8 .\CortexM3\ARM_GCC_541\Debug\VCNL4030X01_PS.o
 .debug_aranges
                0x00000170       0x90 .\CortexM3\ARM_GCC_541\Debug\VCNL4030X01_ALS.o
 .debug_aranges
                0x00000200       0x88 .\CortexM3\ARM_GCC_541\Debug\VCNL4030X01_Application_Library.o
 .debug_aranges
                0x00000288       0x58 .\CortexM3\ARM_GCC_541\Debug\cyfitter_cfg.o
 .debug_aranges
                0x000002e0       0x18 .\CortexM3\ARM_GCC_541\Debug\cymetadata.o
 .debug_aranges
                0x000002f8       0x48 .\CortexM3\ARM_GCC_541\Debug\Cm3Start.o
 .debug_aranges
                0x00000340       0x38 .\CortexM3\ARM_GCC_541\Debug\VCNL4030X01.a(I2C_1.o)
 .debug_aranges
                0x00000378       0x20 .\CortexM3\ARM_GCC_541\Debug\VCNL4030X01.a(I2C_1_INT.o)
 .debug_aranges
                0x00000398       0x38 .\CortexM3\ARM_GCC_541\Debug\VCNL4030X01.a(I2C_1_PM.o)
 .debug_aranges
                0x000003d0       0x80 .\CortexM3\ARM_GCC_541\Debug\VCNL4030X01.a(I2C_1_MASTER.o)
 .debug_aranges
                0x00000450       0xc8 .\CortexM3\ARM_GCC_541\Debug\VCNL4030X01.a(CDC.o)
 .debug_aranges
                0x00000518       0xe8 .\CortexM3\ARM_GCC_541\Debug\VCNL4030X01.a(CDC_cdc.o)
 .debug_aranges
                0x00000600       0x98 .\CortexM3\ARM_GCC_541\Debug\VCNL4030X01.a(CDC_drv.o)
 .debug_aranges
                0x00000698       0x40 .\CortexM3\ARM_GCC_541\Debug\VCNL4030X01.a(CDC_episr.o)
 .debug_aranges
                0x000006d8       0x40 .\CortexM3\ARM_GCC_541\Debug\VCNL4030X01.a(CDC_pm.o)
 .debug_aranges
                0x00000718       0x80 .\CortexM3\ARM_GCC_541\Debug\VCNL4030X01.a(CDC_std.o)
 .debug_aranges
                0x00000798       0x20 .\CortexM3\ARM_GCC_541\Debug\VCNL4030X01.a(CDC_vnd.o)
 .debug_aranges
                0x000007b8       0x48 .\CortexM3\ARM_GCC_541\Debug\VCNL4030X01.a(CDC_Dp.o)
 .debug_aranges
                0x00000800      0x2a0 .\CortexM3\ARM_GCC_541\Debug\VCNL4030X01.a(CyLib.o)
 .debug_aranges
                0x00000aa0       0x98 .\CortexM3\ARM_GCC_541\Debug\VCNL4030X01.a(cyPm.o)
 .debug_aranges
                0x00000b38       0x20 .\CortexM3\ARM_GCC_541\Debug\VCNL4030X01.a(CyBootAsmGnu.o)
 .debug_aranges
                0x00000b58       0x20 .\CortexM3\ARM_GCC_541\Debug\VCNL4030X01.a(CDC_cls.o)
 .debug_aranges
                0x00000b78       0x18 .\CortexM3\ARM_GCC_541\Debug\VCNL4030X01.a(CDC_descr.o)
 .debug_aranges
                0x00000b90       0x88 .\CortexM3\ARM_GCC_541\Debug\VCNL4030X01.a(CyFlash.o)
 .debug_aranges
                0x00000c18       0x80 .\CortexM3\ARM_GCC_541\Debug\VCNL4030X01.a(CySpc.o)

.debug_pubnames
 *(.debug_pubnames)

.debug_info     0x00000000     0xa881
 *(.debug_info .gnu.linkonce.wi.*)
 .debug_info    0x00000000      0xba9 .\CortexM3\ARM_GCC_541\Debug\main.o
 .debug_info    0x00000ba9      0x2ce .\CortexM3\ARM_GCC_541\Debug\I2C_Functions.o
 .debug_info    0x00000e77      0xaad .\CortexM3\ARM_GCC_541\Debug\VCNL4030X01_PS.o
 .debug_info    0x00001924      0x5f9 .\CortexM3\ARM_GCC_541\Debug\VCNL4030X01_ALS.o
 .debug_info    0x00001f1d     0x1989 .\CortexM3\ARM_GCC_541\Debug\VCNL4030X01_Application_Library.o
 .debug_info    0x000038a6      0x4cc .\CortexM3\ARM_GCC_541\Debug\cyfitter_cfg.o
 .debug_info    0x00003d72      0x134 .\CortexM3\ARM_GCC_541\Debug\cymetadata.o
 .debug_info    0x00003ea6      0x3bb .\CortexM3\ARM_GCC_541\Debug\Cm3Start.o
 .debug_info    0x00004261      0x2ad .\CortexM3\ARM_GCC_541\Debug\VCNL4030X01.a(I2C_1.o)
 .debug_info    0x0000450e      0x184 .\CortexM3\ARM_GCC_541\Debug\VCNL4030X01.a(I2C_1_INT.o)
 .debug_info    0x00004692      0x207 .\CortexM3\ARM_GCC_541\Debug\VCNL4030X01.a(I2C_1_PM.o)
 .debug_info    0x00004899      0x407 .\CortexM3\ARM_GCC_541\Debug\VCNL4030X01.a(I2C_1_MASTER.o)
 .debug_info    0x00004ca0      0x995 .\CortexM3\ARM_GCC_541\Debug\VCNL4030X01.a(CDC.o)
 .debug_info    0x00005635      0xaf7 .\CortexM3\ARM_GCC_541\Debug\VCNL4030X01.a(CDC_cdc.o)
 .debug_info    0x0000612c      0x655 .\CortexM3\ARM_GCC_541\Debug\VCNL4030X01.a(CDC_drv.o)
 .debug_info    0x00006781      0x254 .\CortexM3\ARM_GCC_541\Debug\VCNL4030X01.a(CDC_episr.o)
 .debug_info    0x000069d5      0x2e4 .\CortexM3\ARM_GCC_541\Debug\VCNL4030X01.a(CDC_pm.o)
 .debug_info    0x00006cb9      0xb26 .\CortexM3\ARM_GCC_541\Debug\VCNL4030X01.a(CDC_std.o)
 .debug_info    0x000077df       0xed .\CortexM3\ARM_GCC_541\Debug\VCNL4030X01.a(CDC_vnd.o)
 .debug_info    0x000078cc      0x174 .\CortexM3\ARM_GCC_541\Debug\VCNL4030X01.a(CDC_Dp.o)
 .debug_info    0x00007a40     0x1374 .\CortexM3\ARM_GCC_541\Debug\VCNL4030X01.a(CyLib.o)
 .debug_info    0x00008db4      0xa2a .\CortexM3\ARM_GCC_541\Debug\VCNL4030X01.a(cyPm.o)
 .debug_info    0x000097de       0x85 .\CortexM3\ARM_GCC_541\Debug\VCNL4030X01.a(CyBootAsmGnu.o)
 .debug_info    0x00009863      0x1de .\CortexM3\ARM_GCC_541\Debug\VCNL4030X01.a(CDC_cls.o)
 .debug_info    0x00009a41      0x2a3 .\CortexM3\ARM_GCC_541\Debug\VCNL4030X01.a(CDC_descr.o)
 .debug_info    0x00009ce4      0x64d .\CortexM3\ARM_GCC_541\Debug\VCNL4030X01.a(CyFlash.o)
 .debug_info    0x0000a331      0x550 .\CortexM3\ARM_GCC_541\Debug\VCNL4030X01.a(CySpc.o)

.debug_abbrev   0x00000000     0x2431
 *(.debug_abbrev)
 .debug_abbrev  0x00000000      0x129 .\CortexM3\ARM_GCC_541\Debug\main.o
 .debug_abbrev  0x00000129      0x106 .\CortexM3\ARM_GCC_541\Debug\I2C_Functions.o
 .debug_abbrev  0x0000022f      0x189 .\CortexM3\ARM_GCC_541\Debug\VCNL4030X01_PS.o
 .debug_abbrev  0x000003b8      0x15e .\CortexM3\ARM_GCC_541\Debug\VCNL4030X01_ALS.o
 .debug_abbrev  0x00000516      0x2c0 .\CortexM3\ARM_GCC_541\Debug\VCNL4030X01_Application_Library.o
 .debug_abbrev  0x000007d6      0x1fe .\CortexM3\ARM_GCC_541\Debug\cyfitter_cfg.o
 .debug_abbrev  0x000009d4       0x5d .\CortexM3\ARM_GCC_541\Debug\cymetadata.o
 .debug_abbrev  0x00000a31      0x1e8 .\CortexM3\ARM_GCC_541\Debug\Cm3Start.o
 .debug_abbrev  0x00000c19      0x10a .\CortexM3\ARM_GCC_541\Debug\VCNL4030X01.a(I2C_1.o)
 .debug_abbrev  0x00000d23       0xb6 .\CortexM3\ARM_GCC_541\Debug\VCNL4030X01.a(I2C_1_INT.o)
 .debug_abbrev  0x00000dd9       0xfe .\CortexM3\ARM_GCC_541\Debug\VCNL4030X01.a(I2C_1_PM.o)
 .debug_abbrev  0x00000ed7      0x13c .\CortexM3\ARM_GCC_541\Debug\VCNL4030X01.a(I2C_1_MASTER.o)
 .debug_abbrev  0x00001013      0x215 .\CortexM3\ARM_GCC_541\Debug\VCNL4030X01.a(CDC.o)
 .debug_abbrev  0x00001228      0x245 .\CortexM3\ARM_GCC_541\Debug\VCNL4030X01.a(CDC_cdc.o)
 .debug_abbrev  0x0000146d      0x189 .\CortexM3\ARM_GCC_541\Debug\VCNL4030X01.a(CDC_drv.o)
 .debug_abbrev  0x000015f6      0x11b .\CortexM3\ARM_GCC_541\Debug\VCNL4030X01.a(CDC_episr.o)
 .debug_abbrev  0x00001711      0x108 .\CortexM3\ARM_GCC_541\Debug\VCNL4030X01.a(CDC_pm.o)
 .debug_abbrev  0x00001819      0x20a .\CortexM3\ARM_GCC_541\Debug\VCNL4030X01.a(CDC_std.o)
 .debug_abbrev  0x00001a23       0x9b .\CortexM3\ARM_GCC_541\Debug\VCNL4030X01.a(CDC_vnd.o)
 .debug_abbrev  0x00001abe       0x90 .\CortexM3\ARM_GCC_541\Debug\VCNL4030X01.a(CDC_Dp.o)
 .debug_abbrev  0x00001b4e      0x254 .\CortexM3\ARM_GCC_541\Debug\VCNL4030X01.a(CyLib.o)
 .debug_abbrev  0x00001da2      0x1ab .\CortexM3\ARM_GCC_541\Debug\VCNL4030X01.a(cyPm.o)
 .debug_abbrev  0x00001f4d       0x14 .\CortexM3\ARM_GCC_541\Debug\VCNL4030X01.a(CyBootAsmGnu.o)
 .debug_abbrev  0x00001f61       0xe1 .\CortexM3\ARM_GCC_541\Debug\VCNL4030X01.a(CDC_cls.o)
 .debug_abbrev  0x00002042       0xb4 .\CortexM3\ARM_GCC_541\Debug\VCNL4030X01.a(CDC_descr.o)
 .debug_abbrev  0x000020f6      0x1a7 .\CortexM3\ARM_GCC_541\Debug\VCNL4030X01.a(CyFlash.o)
 .debug_abbrev  0x0000229d      0x194 .\CortexM3\ARM_GCC_541\Debug\VCNL4030X01.a(CySpc.o)

.debug_line     0x00000000     0x3ae6
 *(.debug_line)
 .debug_line    0x00000000      0x30c .\CortexM3\ARM_GCC_541\Debug\main.o
 .debug_line    0x0000030c      0x1d8 .\CortexM3\ARM_GCC_541\Debug\I2C_Functions.o
 .debug_line    0x000004e4      0x40d .\CortexM3\ARM_GCC_541\Debug\VCNL4030X01_PS.o
 .debug_line    0x000008f1      0x2e8 .\CortexM3\ARM_GCC_541\Debug\VCNL4030X01_ALS.o
 .debug_line    0x00000bd9      0x53a .\CortexM3\ARM_GCC_541\Debug\VCNL4030X01_Application_Library.o
 .debug_line    0x00001113      0x1d1 .\CortexM3\ARM_GCC_541\Debug\cyfitter_cfg.o
 .debug_line    0x000012e4      0x141 .\CortexM3\ARM_GCC_541\Debug\cymetadata.o
 .debug_line    0x00001425      0x234 .\CortexM3\ARM_GCC_541\Debug\Cm3Start.o
 .debug_line    0x00001659       0xdf .\CortexM3\ARM_GCC_541\Debug\VCNL4030X01.a(I2C_1.o)
 .debug_line    0x00001738      0x118 .\CortexM3\ARM_GCC_541\Debug\VCNL4030X01.a(I2C_1_INT.o)
 .debug_line    0x00001850       0xbf .\CortexM3\ARM_GCC_541\Debug\VCNL4030X01.a(I2C_1_PM.o)
 .debug_line    0x0000190f      0x201 .\CortexM3\ARM_GCC_541\Debug\VCNL4030X01.a(I2C_1_MASTER.o)
 .debug_line    0x00001b10      0x2cc .\CortexM3\ARM_GCC_541\Debug\VCNL4030X01.a(CDC.o)
 .debug_line    0x00001ddc      0x2e6 .\CortexM3\ARM_GCC_541\Debug\VCNL4030X01.a(CDC_cdc.o)
 .debug_line    0x000020c2      0x215 .\CortexM3\ARM_GCC_541\Debug\VCNL4030X01.a(CDC_drv.o)
 .debug_line    0x000022d7       0xda .\CortexM3\ARM_GCC_541\Debug\VCNL4030X01.a(CDC_episr.o)
 .debug_line    0x000023b1       0xfe .\CortexM3\ARM_GCC_541\Debug\VCNL4030X01.a(CDC_pm.o)
 .debug_line    0x000024af      0x3d6 .\CortexM3\ARM_GCC_541\Debug\VCNL4030X01.a(CDC_std.o)
 .debug_line    0x00002885       0x6b .\CortexM3\ARM_GCC_541\Debug\VCNL4030X01.a(CDC_vnd.o)
 .debug_line    0x000028f0       0xb7 .\CortexM3\ARM_GCC_541\Debug\VCNL4030X01.a(CDC_Dp.o)
 .debug_line    0x000029a7      0x816 .\CortexM3\ARM_GCC_541\Debug\VCNL4030X01.a(CyLib.o)
 .debug_line    0x000031bd      0x367 .\CortexM3\ARM_GCC_541\Debug\VCNL4030X01.a(cyPm.o)
 .debug_line    0x00003524       0x66 .\CortexM3\ARM_GCC_541\Debug\VCNL4030X01.a(CyBootAsmGnu.o)
 .debug_line    0x0000358a       0x89 .\CortexM3\ARM_GCC_541\Debug\VCNL4030X01.a(CDC_cls.o)
 .debug_line    0x00003613       0x59 .\CortexM3\ARM_GCC_541\Debug\VCNL4030X01.a(CDC_descr.o)
 .debug_line    0x0000366c      0x21a .\CortexM3\ARM_GCC_541\Debug\VCNL4030X01.a(CyFlash.o)
 .debug_line    0x00003886      0x260 .\CortexM3\ARM_GCC_541\Debug\VCNL4030X01.a(CySpc.o)

.debug_frame    0x00000000     0x278c
 *(.debug_frame)
 .debug_frame   0x00000000       0xd4 .\CortexM3\ARM_GCC_541\Debug\main.o
 .debug_frame   0x000000d4       0x4c .\CortexM3\ARM_GCC_541\Debug\I2C_Functions.o
 .debug_frame   0x00000120      0x368 .\CortexM3\ARM_GCC_541\Debug\VCNL4030X01_PS.o
 .debug_frame   0x00000488      0x1d0 .\CortexM3\ARM_GCC_541\Debug\VCNL4030X01_ALS.o
 .debug_frame   0x00000658      0x1e0 .\CortexM3\ARM_GCC_541\Debug\VCNL4030X01_Application_Library.o
 .debug_frame   0x00000838       0xe4 .\CortexM3\ARM_GCC_541\Debug\cyfitter_cfg.o
 .debug_frame   0x0000091c       0xb8 .\CortexM3\ARM_GCC_541\Debug\Cm3Start.o
 .debug_frame   0x000009d4       0x94 .\CortexM3\ARM_GCC_541\Debug\VCNL4030X01.a(I2C_1.o)
 .debug_frame   0x00000a68       0x30 .\CortexM3\ARM_GCC_541\Debug\VCNL4030X01.a(I2C_1_INT.o)
 .debug_frame   0x00000a98       0x74 .\CortexM3\ARM_GCC_541\Debug\VCNL4030X01.a(I2C_1_PM.o)
 .debug_frame   0x00000b0c      0x138 .\CortexM3\ARM_GCC_541\Debug\VCNL4030X01.a(I2C_1_MASTER.o)
 .debug_frame   0x00000c44      0x1dc .\CortexM3\ARM_GCC_541\Debug\VCNL4030X01.a(CDC.o)
 .debug_frame   0x00000e20      0x27c .\CortexM3\ARM_GCC_541\Debug\VCNL4030X01.a(CDC_cdc.o)
 .debug_frame   0x0000109c      0x194 .\CortexM3\ARM_GCC_541\Debug\VCNL4030X01.a(CDC_drv.o)
 .debug_frame   0x00001230       0x6c .\CortexM3\ARM_GCC_541\Debug\VCNL4030X01.a(CDC_episr.o)
 .debug_frame   0x0000129c       0xa0 .\CortexM3\ARM_GCC_541\Debug\VCNL4030X01.a(CDC_pm.o)
 .debug_frame   0x0000133c      0x17c .\CortexM3\ARM_GCC_541\Debug\VCNL4030X01.a(CDC_std.o)
 .debug_frame   0x000014b8       0x20 .\CortexM3\ARM_GCC_541\Debug\VCNL4030X01.a(CDC_vnd.o)
 .debug_frame   0x000014d8       0x70 .\CortexM3\ARM_GCC_541\Debug\VCNL4030X01.a(CDC_Dp.o)
 .debug_frame   0x00001548      0x738 .\CortexM3\ARM_GCC_541\Debug\VCNL4030X01.a(CyLib.o)
 .debug_frame   0x00001c80      0x1f8 .\CortexM3\ARM_GCC_541\Debug\VCNL4030X01.a(cyPm.o)
 .debug_frame   0x00001e78       0x2c .\CortexM3\ARM_GCC_541\Debug\VCNL4030X01.a(CDC_cls.o)
 .debug_frame   0x00001ea4      0x194 .\CortexM3\ARM_GCC_541\Debug\VCNL4030X01.a(CyFlash.o)
 .debug_frame   0x00002038      0x180 .\CortexM3\ARM_GCC_541\Debug\VCNL4030X01.a(CySpc.o)
 .debug_frame   0x000021b8       0x4c c:/program files (x86)/cypress/psoc creator/4.3/psoc creator/import/gnu/arm/5.4.1/bin/../lib/gcc/arm-none-eabi/5.4.1/../../../../arm-none-eabi/lib/armv7-m\libm.a(lib_a-w_pow.o)
 .debug_frame   0x00002204       0x68 c:/program files (x86)/cypress/psoc creator/4.3/psoc creator/import/gnu/arm/5.4.1/bin/../lib/gcc/arm-none-eabi/5.4.1/../../../../arm-none-eabi/lib/armv7-m\libm.a(lib_a-e_pow.o)
 .debug_frame   0x0000226c       0x30 c:/program files (x86)/cypress/psoc creator/4.3/psoc creator/import/gnu/arm/5.4.1/bin/../lib/gcc/arm-none-eabi/5.4.1/../../../../arm-none-eabi/lib/armv7-m\libm.a(lib_a-e_sqrt.o)
 .debug_frame   0x0000229c       0x20 c:/program files (x86)/cypress/psoc creator/4.3/psoc creator/import/gnu/arm/5.4.1/bin/../lib/gcc/arm-none-eabi/5.4.1/../../../../arm-none-eabi/lib/armv7-m\libm.a(lib_a-s_fabs.o)
 .debug_frame   0x000022bc       0x20 c:/program files (x86)/cypress/psoc creator/4.3/psoc creator/import/gnu/arm/5.4.1/bin/../lib/gcc/arm-none-eabi/5.4.1/../../../../arm-none-eabi/lib/armv7-m\libm.a(lib_a-s_finite.o)
 .debug_frame   0x000022dc       0x20 c:/program files (x86)/cypress/psoc creator/4.3/psoc creator/import/gnu/arm/5.4.1/bin/../lib/gcc/arm-none-eabi/5.4.1/../../../../arm-none-eabi/lib/armv7-m\libm.a(lib_a-s_matherr.o)
 .debug_frame   0x000022fc       0x20 c:/program files (x86)/cypress/psoc creator/4.3/psoc creator/import/gnu/arm/5.4.1/bin/../lib/gcc/arm-none-eabi/5.4.1/../../../../arm-none-eabi/lib/armv7-m\libm.a(lib_a-s_nan.o)
 .debug_frame   0x0000231c       0x3c c:/program files (x86)/cypress/psoc creator/4.3/psoc creator/import/gnu/arm/5.4.1/bin/../lib/gcc/arm-none-eabi/5.4.1/../../../../arm-none-eabi/lib/armv7-m\libm.a(lib_a-s_rint.o)
 .debug_frame   0x00002358       0x30 c:/program files (x86)/cypress/psoc creator/4.3/psoc creator/import/gnu/arm/5.4.1/bin/../lib/gcc/arm-none-eabi/5.4.1/../../../../arm-none-eabi/lib/armv7-m\libm.a(lib_a-s_scalbn.o)
 .debug_frame   0x00002388       0x20 c:/program files (x86)/cypress/psoc creator/4.3/psoc creator/import/gnu/arm/5.4.1/bin/../lib/gcc/arm-none-eabi/5.4.1/../../../../arm-none-eabi/lib/armv7-m\libm.a(lib_a-s_copysign.o)
 .debug_frame   0x000023a8       0x20 c:/program files (x86)/cypress/psoc creator/4.3/psoc creator/import/gnu/arm/5.4.1/bin/../lib/gcc/arm-none-eabi/5.4.1/../../../../arm-none-eabi/lib/armv7-m\libg_nano.a(lib_a-errno.o)
 .debug_frame   0x000023c8       0x28 c:/program files (x86)/cypress/psoc creator/4.3/psoc creator/import/gnu/arm/5.4.1/bin/../lib/gcc/arm-none-eabi/5.4.1/../../../../arm-none-eabi/lib/armv7-m\libg_nano.a(lib_a-exit.o)
 .debug_frame   0x000023f0       0x2c c:/program files (x86)/cypress/psoc creator/4.3/psoc creator/import/gnu/arm/5.4.1/bin/../lib/gcc/arm-none-eabi/5.4.1/../../../../arm-none-eabi/lib/armv7-m\libg_nano.a(lib_a-init.o)
 .debug_frame   0x0000241c       0x28 c:/program files (x86)/cypress/psoc creator/4.3/psoc creator/import/gnu/arm/5.4.1/bin/../lib/gcc/arm-none-eabi/5.4.1/../../../../arm-none-eabi/lib/armv7-m\libg_nano.a(lib_a-memcpy-stub.o)
 .debug_frame   0x00002444       0x20 c:/program files (x86)/cypress/psoc creator/4.3/psoc creator/import/gnu/arm/5.4.1/bin/../lib/gcc/arm-none-eabi/5.4.1/../../../../arm-none-eabi/lib/armv7-m\libg_nano.a(lib_a-memset.o)
 .debug_frame   0x00002464       0x70 c:/program files (x86)/cypress/psoc creator/4.3/psoc creator/import/gnu/arm/5.4.1/bin/../lib/gcc/arm-none-eabi/5.4.1/../../../../arm-none-eabi/lib/armv7-m\libg_nano.a(lib_a-sprintf.o)
 .debug_frame   0x000024d4       0x90 c:/program files (x86)/cypress/psoc creator/4.3/psoc creator/import/gnu/arm/5.4.1/bin/../lib/gcc/arm-none-eabi/5.4.1/../../../../arm-none-eabi/lib/armv7-m\libg_nano.a(lib_a-nano-svfprintf.o)
 .debug_frame   0x00002564       0x60 c:/program files (x86)/cypress/psoc creator/4.3/psoc creator/import/gnu/arm/5.4.1/bin/../lib/gcc/arm-none-eabi/5.4.1/../../../../arm-none-eabi/lib/armv7-m\libg_nano.a(lib_a-nano-vfprintf_i.o)
 .debug_frame   0x000025c4       0x28 c:/program files (x86)/cypress/psoc creator/4.3/psoc creator/import/gnu/arm/5.4.1/bin/../lib/gcc/arm-none-eabi/5.4.1/../../../../arm-none-eabi/lib/armv7-m\libg_nano.a(lib_a-memchr-stub.o)
 .debug_frame   0x000025ec       0x28 c:/program files (x86)/cypress/psoc creator/4.3/psoc creator/import/gnu/arm/5.4.1/bin/../lib/gcc/arm-none-eabi/5.4.1/../../../../arm-none-eabi/lib/armv7-m\libg_nano.a(lib_a-memmove.o)
 .debug_frame   0x00002614       0x38 c:/program files (x86)/cypress/psoc creator/4.3/psoc creator/import/gnu/arm/5.4.1/bin/../lib/gcc/arm-none-eabi/5.4.1/../../../../arm-none-eabi/lib/armv7-m\libg_nano.a(lib_a-nano-freer.o)
 .debug_frame   0x0000264c       0x2c c:/program files (x86)/cypress/psoc creator/4.3/psoc creator/import/gnu/arm/5.4.1/bin/../lib/gcc/arm-none-eabi/5.4.1/../../../../arm-none-eabi/lib/armv7-m\libg_nano.a(lib_a-nano-mallocr.o)
 .debug_frame   0x00002678       0x3c c:/program files (x86)/cypress/psoc creator/4.3/psoc creator/import/gnu/arm/5.4.1/bin/../lib/gcc/arm-none-eabi/5.4.1/../../../../arm-none-eabi/lib/armv7-m\libg_nano.a(lib_a-nano-reallocr.o)
 .debug_frame   0x000026b4       0x2c c:/program files (x86)/cypress/psoc creator/4.3/psoc creator/import/gnu/arm/5.4.1/bin/../lib/gcc/arm-none-eabi/5.4.1/../../../../arm-none-eabi/lib/armv7-m\libg_nano.a(lib_a-sbrkr.o)
 .debug_frame   0x000026e0       0x30 c:/program files (x86)/cypress/psoc creator/4.3/psoc creator/import/gnu/arm/5.4.1/bin/../lib/gcc/arm-none-eabi/5.4.1/../../../../arm-none-eabi/lib/armv7-m\libg_nano.a(lib_a-mlock.o)
 .debug_frame   0x00002710       0x20 c:/program files (x86)/cypress/psoc creator/4.3/psoc creator/import/gnu/arm/5.4.1/bin/../lib/gcc/arm-none-eabi/5.4.1/../../../../arm-none-eabi/lib/armv7-m\libg_nano.a(lib_a-nano-msizer.o)
 .debug_frame   0x00002730       0x5c c:/program files (x86)/cypress/psoc creator/4.3/psoc creator/import/gnu/arm/5.4.1/bin/../lib/gcc/arm-none-eabi/5.4.1/../../../../arm-none-eabi/lib/armv7-m\libg_nano.a(lib_a-reent.o)

.debug_str      0x00000000     0x2cb1
 *(.debug_str)
 .debug_str     0x00000000      0x533 .\CortexM3\ARM_GCC_541\Debug\main.o
                                0x596 (size before relaxing)
 .debug_str     0x00000533      0x121 .\CortexM3\ARM_GCC_541\Debug\I2C_Functions.o
                                0x2d6 (size before relaxing)
 .debug_str     0x00000654      0x158 .\CortexM3\ARM_GCC_541\Debug\VCNL4030X01_PS.o
                                0x5e7 (size before relaxing)
 .debug_str     0x000007ac       0xc8 .\CortexM3\ARM_GCC_541\Debug\VCNL4030X01_ALS.o
                                0x444 (size before relaxing)
 .debug_str     0x00000874      0x15c .\CortexM3\ARM_GCC_541\Debug\VCNL4030X01_Application_Library.o
                                0x519 (size before relaxing)
 .debug_str     0x000009d0      0x181 .\CortexM3\ARM_GCC_541\Debug\cyfitter_cfg.o
                                0x304 (size before relaxing)
 .debug_str     0x00000b51       0x75 .\CortexM3\ARM_GCC_541\Debug\cymetadata.o
                                0x1d9 (size before relaxing)
 .debug_str     0x00000bc6      0x144 .\CortexM3\ARM_GCC_541\Debug\Cm3Start.o
                                0x2ff (size before relaxing)
 .debug_str     0x00000d0a      0x145 .\CortexM3\ARM_GCC_541\Debug\VCNL4030X01.a(I2C_1.o)
                                0x2ee (size before relaxing)
 .debug_str     0x00000e4f       0x94 .\CortexM3\ARM_GCC_541\Debug\VCNL4030X01.a(I2C_1_INT.o)
                                0x26a (size before relaxing)
 .debug_str     0x00000ee3       0x60 .\CortexM3\ARM_GCC_541\Debug\VCNL4030X01.a(I2C_1_PM.o)
                                0x284 (size before relaxing)
 .debug_str     0x00000f43       0xdd .\CortexM3\ARM_GCC_541\Debug\VCNL4030X01.a(I2C_1_MASTER.o)
                                0x3c7 (size before relaxing)
 .debug_str     0x00001020      0x394 .\CortexM3\ARM_GCC_541\Debug\VCNL4030X01.a(CDC.o)
                                0x5bf (size before relaxing)
 .debug_str     0x000013b4      0x44e .\CortexM3\ARM_GCC_541\Debug\VCNL4030X01.a(CDC_cdc.o)
                                0x6f2 (size before relaxing)
 .debug_str     0x00001802      0x231 .\CortexM3\ARM_GCC_541\Debug\VCNL4030X01.a(CDC_drv.o)
                                0x595 (size before relaxing)
 .debug_str     0x00001a33       0x68 .\CortexM3\ARM_GCC_541\Debug\VCNL4030X01.a(CDC_episr.o)
                                0x2a8 (size before relaxing)
 .debug_str     0x00001a9b       0x9e .\CortexM3\ARM_GCC_541\Debug\VCNL4030X01.a(CDC_pm.o)
                                0x2b5 (size before relaxing)
 .debug_str     0x00001b39      0x22c .\CortexM3\ARM_GCC_541\Debug\VCNL4030X01.a(CDC_std.o)
                                0x6f8 (size before relaxing)
 .debug_str     0x00001d65       0x21 .\CortexM3\ARM_GCC_541\Debug\VCNL4030X01.a(CDC_vnd.o)
                                0x1d6 (size before relaxing)
 .debug_str     0x00001d86       0x8c .\CortexM3\ARM_GCC_541\Debug\VCNL4030X01.a(CDC_Dp.o)
                                0x21a (size before relaxing)
 .debug_str     0x00001e12      0x7ca .\CortexM3\ARM_GCC_541\Debug\VCNL4030X01.a(CyLib.o)
                                0xa3c (size before relaxing)
 .debug_str     0x000025dc      0x365 .\CortexM3\ARM_GCC_541\Debug\VCNL4030X01.a(cyPm.o)
                                0x728 (size before relaxing)
 .debug_str     0x00002941       0x21 .\CortexM3\ARM_GCC_541\Debug\VCNL4030X01.a(CDC_cls.o)
                                0x285 (size before relaxing)
 .debug_str     0x00002962       0xe8 .\CortexM3\ARM_GCC_541\Debug\VCNL4030X01.a(CDC_descr.o)
                                0x31a (size before relaxing)
 .debug_str     0x00002a4a      0x1bb .\CortexM3\ARM_GCC_541\Debug\VCNL4030X01.a(CyFlash.o)
                                0x3b5 (size before relaxing)
 .debug_str     0x00002c05       0xac .\CortexM3\ARM_GCC_541\Debug\VCNL4030X01.a(CySpc.o)
                                0x32d (size before relaxing)

.debug_loc      0x00000000     0x3fe3
 *(.debug_loc)
 .debug_loc     0x00000000       0x5d .\CortexM3\ARM_GCC_541\Debug\main.o
 .debug_loc     0x0000005d       0xc3 .\CortexM3\ARM_GCC_541\Debug\I2C_Functions.o
 .debug_loc     0x00000120      0x432 .\CortexM3\ARM_GCC_541\Debug\VCNL4030X01_PS.o
 .debug_loc     0x00000552      0x1a9 .\CortexM3\ARM_GCC_541\Debug\VCNL4030X01_ALS.o
 .debug_loc     0x000006fb      0x47b .\CortexM3\ARM_GCC_541\Debug\VCNL4030X01_Application_Library.o
 .debug_loc     0x00000b76      0x1d7 .\CortexM3\ARM_GCC_541\Debug\cyfitter_cfg.o
 .debug_loc     0x00000d4d      0x144 .\CortexM3\ARM_GCC_541\Debug\Cm3Start.o
 .debug_loc     0x00000e91       0x39 .\CortexM3\ARM_GCC_541\Debug\VCNL4030X01.a(I2C_1.o)
 .debug_loc     0x00000eca       0x29 .\CortexM3\ARM_GCC_541\Debug\VCNL4030X01.a(I2C_1_INT.o)
 .debug_loc     0x00000ef3       0x13 .\CortexM3\ARM_GCC_541\Debug\VCNL4030X01.a(I2C_1_PM.o)
 .debug_loc     0x00000f06      0x52f .\CortexM3\ARM_GCC_541\Debug\VCNL4030X01.a(I2C_1_MASTER.o)
 .debug_loc     0x00001435      0x3e1 .\CortexM3\ARM_GCC_541\Debug\VCNL4030X01.a(CDC.o)
 .debug_loc     0x00001816      0x557 .\CortexM3\ARM_GCC_541\Debug\VCNL4030X01.a(CDC_cdc.o)
 .debug_loc     0x00001d6d      0x171 .\CortexM3\ARM_GCC_541\Debug\VCNL4030X01.a(CDC_drv.o)
 .debug_loc     0x00001ede       0x26 .\CortexM3\ARM_GCC_541\Debug\VCNL4030X01.a(CDC_pm.o)
 .debug_loc     0x00001f04      0x945 .\CortexM3\ARM_GCC_541\Debug\VCNL4030X01.a(CDC_std.o)
 .debug_loc     0x00002849       0x84 .\CortexM3\ARM_GCC_541\Debug\VCNL4030X01.a(CDC_Dp.o)
 .debug_loc     0x000028cd      0xa11 .\CortexM3\ARM_GCC_541\Debug\VCNL4030X01.a(CyLib.o)
 .debug_loc     0x000032de      0x1e4 .\CortexM3\ARM_GCC_541\Debug\VCNL4030X01.a(cyPm.o)
 .debug_loc     0x000034c2       0x6a .\CortexM3\ARM_GCC_541\Debug\VCNL4030X01.a(CDC_cls.o)
 .debug_loc     0x0000352c      0x3b2 .\CortexM3\ARM_GCC_541\Debug\VCNL4030X01.a(CyFlash.o)
 .debug_loc     0x000038de      0x705 .\CortexM3\ARM_GCC_541\Debug\VCNL4030X01.a(CySpc.o)

.debug_macinfo
 *(.debug_macinfo)

.debug_ranges   0x00000000      0xae0
 *(.debug_ranges)
 .debug_ranges  0x00000000       0x40 .\CortexM3\ARM_GCC_541\Debug\main.o
 .debug_ranges  0x00000040       0x18 .\CortexM3\ARM_GCC_541\Debug\I2C_Functions.o
 .debug_ranges  0x00000058       0xe8 .\CortexM3\ARM_GCC_541\Debug\VCNL4030X01_PS.o
 .debug_ranges  0x00000140       0x80 .\CortexM3\ARM_GCC_541\Debug\VCNL4030X01_ALS.o
 .debug_ranges  0x000001c0       0x78 .\CortexM3\ARM_GCC_541\Debug\VCNL4030X01_Application_Library.o
 .debug_ranges  0x00000238       0x48 .\CortexM3\ARM_GCC_541\Debug\cyfitter_cfg.o
 .debug_ranges  0x00000280       0x38 .\CortexM3\ARM_GCC_541\Debug\Cm3Start.o
 .debug_ranges  0x000002b8       0x28 .\CortexM3\ARM_GCC_541\Debug\VCNL4030X01.a(I2C_1.o)
 .debug_ranges  0x000002e0       0x10 .\CortexM3\ARM_GCC_541\Debug\VCNL4030X01.a(I2C_1_INT.o)
 .debug_ranges  0x000002f0       0x28 .\CortexM3\ARM_GCC_541\Debug\VCNL4030X01.a(I2C_1_PM.o)
 .debug_ranges  0x00000318       0x70 .\CortexM3\ARM_GCC_541\Debug\VCNL4030X01.a(I2C_1_MASTER.o)
 .debug_ranges  0x00000388       0xd0 .\CortexM3\ARM_GCC_541\Debug\VCNL4030X01.a(CDC.o)
 .debug_ranges  0x00000458       0xd8 .\CortexM3\ARM_GCC_541\Debug\VCNL4030X01.a(CDC_cdc.o)
 .debug_ranges  0x00000530       0x88 .\CortexM3\ARM_GCC_541\Debug\VCNL4030X01.a(CDC_drv.o)
 .debug_ranges  0x000005b8       0x30 .\CortexM3\ARM_GCC_541\Debug\VCNL4030X01.a(CDC_episr.o)
 .debug_ranges  0x000005e8       0x30 .\CortexM3\ARM_GCC_541\Debug\VCNL4030X01.a(CDC_pm.o)
 .debug_ranges  0x00000618       0x70 .\CortexM3\ARM_GCC_541\Debug\VCNL4030X01.a(CDC_std.o)
 .debug_ranges  0x00000688       0x10 .\CortexM3\ARM_GCC_541\Debug\VCNL4030X01.a(CDC_vnd.o)
 .debug_ranges  0x00000698       0x38 .\CortexM3\ARM_GCC_541\Debug\VCNL4030X01.a(CDC_Dp.o)
 .debug_ranges  0x000006d0      0x290 .\CortexM3\ARM_GCC_541\Debug\VCNL4030X01.a(CyLib.o)
 .debug_ranges  0x00000960       0x88 .\CortexM3\ARM_GCC_541\Debug\VCNL4030X01.a(cyPm.o)
 .debug_ranges  0x000009e8       0x10 .\CortexM3\ARM_GCC_541\Debug\VCNL4030X01.a(CDC_cls.o)
 .debug_ranges  0x000009f8       0x78 .\CortexM3\ARM_GCC_541\Debug\VCNL4030X01.a(CyFlash.o)
 .debug_ranges  0x00000a70       0x70 .\CortexM3\ARM_GCC_541\Debug\VCNL4030X01.a(CySpc.o)

.comment        0x00000000       0x6e
 .comment       0x00000000       0x6e .\CortexM3\ARM_GCC_541\Debug\main.o
                                 0x6f (size before relaxing)
 .comment       0x0000006e       0x6f .\CortexM3\ARM_GCC_541\Debug\I2C_Functions.o
 .comment       0x0000006e       0x6f .\CortexM3\ARM_GCC_541\Debug\VCNL4030X01_PS.o
 .comment       0x0000006e       0x6f .\CortexM3\ARM_GCC_541\Debug\VCNL4030X01_ALS.o
 .comment       0x0000006e       0x6f .\CortexM3\ARM_GCC_541\Debug\VCNL4030X01_Application_Library.o
 .comment       0x0000006e       0x6f .\CortexM3\ARM_GCC_541\Debug\cyfitter_cfg.o
 .comment       0x0000006e       0x6f .\CortexM3\ARM_GCC_541\Debug\cymetadata.o
 .comment       0x0000006e       0x6f .\CortexM3\ARM_GCC_541\Debug\Cm3Start.o
 .comment       0x0000006e       0x6f .\CortexM3\ARM_GCC_541\Debug\VCNL4030X01.a(I2C_1.o)
 .comment       0x0000006e       0x6f .\CortexM3\ARM_GCC_541\Debug\VCNL4030X01.a(I2C_1_INT.o)
 .comment       0x0000006e       0x6f .\CortexM3\ARM_GCC_541\Debug\VCNL4030X01.a(I2C_1_PM.o)
 .comment       0x0000006e       0x6f .\CortexM3\ARM_GCC_541\Debug\VCNL4030X01.a(I2C_1_MASTER.o)
 .comment       0x0000006e       0x6f .\CortexM3\ARM_GCC_541\Debug\VCNL4030X01.a(CDC.o)
 .comment       0x0000006e       0x6f .\CortexM3\ARM_GCC_541\Debug\VCNL4030X01.a(CDC_cdc.o)
 .comment       0x0000006e       0x6f .\CortexM3\ARM_GCC_541\Debug\VCNL4030X01.a(CDC_drv.o)
 .comment       0x0000006e       0x6f .\CortexM3\ARM_GCC_541\Debug\VCNL4030X01.a(CDC_episr.o)
 .comment       0x0000006e       0x6f .\CortexM3\ARM_GCC_541\Debug\VCNL4030X01.a(CDC_pm.o)
 .comment       0x0000006e       0x6f .\CortexM3\ARM_GCC_541\Debug\VCNL4030X01.a(CDC_std.o)
 .comment       0x0000006e       0x6f .\CortexM3\ARM_GCC_541\Debug\VCNL4030X01.a(CDC_vnd.o)
 .comment       0x0000006e       0x6f .\CortexM3\ARM_GCC_541\Debug\VCNL4030X01.a(CDC_Dp.o)
 .comment       0x0000006e       0x6f .\CortexM3\ARM_GCC_541\Debug\VCNL4030X01.a(CyLib.o)
 .comment       0x0000006e       0x6f .\CortexM3\ARM_GCC_541\Debug\VCNL4030X01.a(cyPm.o)
 .comment       0x0000006e       0x6f .\CortexM3\ARM_GCC_541\Debug\VCNL4030X01.a(CDC_cls.o)
 .comment       0x0000006e       0x6f .\CortexM3\ARM_GCC_541\Debug\VCNL4030X01.a(CDC_descr.o)
 .comment       0x0000006e       0x6f .\CortexM3\ARM_GCC_541\Debug\VCNL4030X01.a(CyFlash.o)
 .comment       0x0000006e       0x6f .\CortexM3\ARM_GCC_541\Debug\VCNL4030X01.a(CySpc.o)

.debug_weaknames
 *(.debug_weaknames)

.debug_funcnames
 *(.debug_funcnames)

.debug_typenames
 *(.debug_typenames)

.debug_varnames
 *(.debug_varnames)

.note.gnu.arm.ident
 *(.note.gnu.arm.ident)

.ARM.attributes
                0x00000000       0x29
 *(.ARM.attributes)
 .ARM.attributes
                0x00000000       0x1d c:/program files (x86)/cypress/psoc creator/4.3/psoc creator/import/gnu/arm/5.4.1/bin/../lib/gcc/arm-none-eabi/5.4.1/armv7-m/crti.o
 .ARM.attributes
                0x0000001d       0x2d c:/program files (x86)/cypress/psoc creator/4.3/psoc creator/import/gnu/arm/5.4.1/bin/../lib/gcc/arm-none-eabi/5.4.1/armv7-m/crtbegin.o
 .ARM.attributes
                0x0000004a       0x1b c:/program files (x86)/cypress/psoc creator/4.3/psoc creator/import/gnu/arm/5.4.1/bin/../lib/gcc/arm-none-eabi/5.4.1/../../../../arm-none-eabi/lib/armv7-m/crt0.o
 .ARM.attributes
                0x00000065       0x33 .\CortexM3\ARM_GCC_541\Debug\main.o
 .ARM.attributes
                0x00000098       0x33 .\CortexM3\ARM_GCC_541\Debug\I2C_Functions.o
 .ARM.attributes
                0x000000cb       0x33 .\CortexM3\ARM_GCC_541\Debug\VCNL4030X01_PS.o
 .ARM.attributes
                0x000000fe       0x33 .\CortexM3\ARM_GCC_541\Debug\VCNL4030X01_ALS.o
 .ARM.attributes
                0x00000131       0x33 .\CortexM3\ARM_GCC_541\Debug\VCNL4030X01_Application_Library.o
 .ARM.attributes
                0x00000164       0x33 .\CortexM3\ARM_GCC_541\Debug\cyfitter_cfg.o
 .ARM.attributes
                0x00000197       0x33 .\CortexM3\ARM_GCC_541\Debug\cymetadata.o
 .ARM.attributes
                0x000001ca       0x33 .\CortexM3\ARM_GCC_541\Debug\Cm3Start.o
 .ARM.attributes
                0x000001fd       0x33 .\CortexM3\ARM_GCC_541\Debug\VCNL4030X01.a(I2C_1.o)
 .ARM.attributes
                0x00000230       0x33 .\CortexM3\ARM_GCC_541\Debug\VCNL4030X01.a(I2C_1_INT.o)
 .ARM.attributes
                0x00000263       0x33 .\CortexM3\ARM_GCC_541\Debug\VCNL4030X01.a(I2C_1_PM.o)
 .ARM.attributes
                0x00000296       0x33 .\CortexM3\ARM_GCC_541\Debug\VCNL4030X01.a(I2C_1_MASTER.o)
 .ARM.attributes
                0x000002c9       0x33 .\CortexM3\ARM_GCC_541\Debug\VCNL4030X01.a(CDC.o)
 .ARM.attributes
                0x000002fc       0x33 .\CortexM3\ARM_GCC_541\Debug\VCNL4030X01.a(CDC_cdc.o)
 .ARM.attributes
                0x0000032f       0x33 .\CortexM3\ARM_GCC_541\Debug\VCNL4030X01.a(CDC_drv.o)
 .ARM.attributes
                0x00000362       0x33 .\CortexM3\ARM_GCC_541\Debug\VCNL4030X01.a(CDC_episr.o)
 .ARM.attributes
                0x00000395       0x33 .\CortexM3\ARM_GCC_541\Debug\VCNL4030X01.a(CDC_pm.o)
 .ARM.attributes
                0x000003c8       0x33 .\CortexM3\ARM_GCC_541\Debug\VCNL4030X01.a(CDC_std.o)
 .ARM.attributes
                0x000003fb       0x33 .\CortexM3\ARM_GCC_541\Debug\VCNL4030X01.a(CDC_vnd.o)
 .ARM.attributes
                0x0000042e       0x33 .\CortexM3\ARM_GCC_541\Debug\VCNL4030X01.a(CDC_Dp.o)
 .ARM.attributes
                0x00000461       0x33 .\CortexM3\ARM_GCC_541\Debug\VCNL4030X01.a(CyLib.o)
 .ARM.attributes
                0x00000494       0x33 .\CortexM3\ARM_GCC_541\Debug\VCNL4030X01.a(cyPm.o)
 .ARM.attributes
                0x000004c7       0x21 .\CortexM3\ARM_GCC_541\Debug\VCNL4030X01.a(CyBootAsmGnu.o)
 .ARM.attributes
                0x000004e8       0x33 .\CortexM3\ARM_GCC_541\Debug\VCNL4030X01.a(CDC_cls.o)
 .ARM.attributes
                0x0000051b       0x33 .\CortexM3\ARM_GCC_541\Debug\VCNL4030X01.a(CDC_descr.o)
 .ARM.attributes
                0x0000054e       0x33 .\CortexM3\ARM_GCC_541\Debug\VCNL4030X01.a(CyFlash.o)
 .ARM.attributes
                0x00000581       0x33 .\CortexM3\ARM_GCC_541\Debug\VCNL4030X01.a(CySpc.o)
 .ARM.attributes
                0x000005b4       0x2d c:/program files (x86)/cypress/psoc creator/4.3/psoc creator/import/gnu/arm/5.4.1/bin/../lib/gcc/arm-none-eabi/5.4.1/../../../../arm-none-eabi/lib/armv7-m\libm.a(lib_a-w_pow.o)
 .ARM.attributes
                0x000005e1       0x2d c:/program files (x86)/cypress/psoc creator/4.3/psoc creator/import/gnu/arm/5.4.1/bin/../lib/gcc/arm-none-eabi/5.4.1/../../../../arm-none-eabi/lib/armv7-m\libm.a(lib_a-e_pow.o)
 .ARM.attributes
                0x0000060e       0x2d c:/program files (x86)/cypress/psoc creator/4.3/psoc creator/import/gnu/arm/5.4.1/bin/../lib/gcc/arm-none-eabi/5.4.1/../../../../arm-none-eabi/lib/armv7-m\libm.a(lib_a-e_sqrt.o)
 .ARM.attributes
                0x0000063b       0x2d c:/program files (x86)/cypress/psoc creator/4.3/psoc creator/import/gnu/arm/5.4.1/bin/../lib/gcc/arm-none-eabi/5.4.1/../../../../arm-none-eabi/lib/armv7-m\libm.a(lib_a-s_fabs.o)
 .ARM.attributes
                0x00000668       0x2d c:/program files (x86)/cypress/psoc creator/4.3/psoc creator/import/gnu/arm/5.4.1/bin/../lib/gcc/arm-none-eabi/5.4.1/../../../../arm-none-eabi/lib/armv7-m\libm.a(lib_a-s_finite.o)
 .ARM.attributes
                0x00000695       0x2d c:/program files (x86)/cypress/psoc creator/4.3/psoc creator/import/gnu/arm/5.4.1/bin/../lib/gcc/arm-none-eabi/5.4.1/../../../../arm-none-eabi/lib/armv7-m\libm.a(lib_a-s_lib_ver.o)
 .ARM.attributes
                0x000006c2       0x2d c:/program files (x86)/cypress/psoc creator/4.3/psoc creator/import/gnu/arm/5.4.1/bin/../lib/gcc/arm-none-eabi/5.4.1/../../../../arm-none-eabi/lib/armv7-m\libm.a(lib_a-s_matherr.o)
 .ARM.attributes
                0x000006ef       0x2d c:/program files (x86)/cypress/psoc creator/4.3/psoc creator/import/gnu/arm/5.4.1/bin/../lib/gcc/arm-none-eabi/5.4.1/../../../../arm-none-eabi/lib/armv7-m\libm.a(lib_a-s_nan.o)
 .ARM.attributes
                0x0000071c       0x2d c:/program files (x86)/cypress/psoc creator/4.3/psoc creator/import/gnu/arm/5.4.1/bin/../lib/gcc/arm-none-eabi/5.4.1/../../../../arm-none-eabi/lib/armv7-m\libm.a(lib_a-s_rint.o)
 .ARM.attributes
                0x00000749       0x2d c:/program files (x86)/cypress/psoc creator/4.3/psoc creator/import/gnu/arm/5.4.1/bin/../lib/gcc/arm-none-eabi/5.4.1/../../../../arm-none-eabi/lib/armv7-m\libm.a(lib_a-s_scalbn.o)
 .ARM.attributes
                0x00000776       0x2d c:/program files (x86)/cypress/psoc creator/4.3/psoc creator/import/gnu/arm/5.4.1/bin/../lib/gcc/arm-none-eabi/5.4.1/../../../../arm-none-eabi/lib/armv7-m\libm.a(lib_a-s_copysign.o)
 .ARM.attributes
                0x000007a3       0x1d c:/program files (x86)/cypress/psoc creator/4.3/psoc creator/import/gnu/arm/5.4.1/bin/../lib/gcc/arm-none-eabi/5.4.1/armv7-m\libgcc.a(_arm_addsubdf3.o)
 .ARM.attributes
                0x000007c0       0x1d c:/program files (x86)/cypress/psoc creator/4.3/psoc creator/import/gnu/arm/5.4.1/bin/../lib/gcc/arm-none-eabi/5.4.1/armv7-m\libgcc.a(_arm_muldivdf3.o)
 .ARM.attributes
                0x000007dd       0x1d c:/program files (x86)/cypress/psoc creator/4.3/psoc creator/import/gnu/arm/5.4.1/bin/../lib/gcc/arm-none-eabi/5.4.1/armv7-m\libgcc.a(_arm_cmpdf2.o)
 .ARM.attributes
                0x000007fa       0x1d c:/program files (x86)/cypress/psoc creator/4.3/psoc creator/import/gnu/arm/5.4.1/bin/../lib/gcc/arm-none-eabi/5.4.1/armv7-m\libgcc.a(_arm_unorddf2.o)
 .ARM.attributes
                0x00000817       0x1d c:/program files (x86)/cypress/psoc creator/4.3/psoc creator/import/gnu/arm/5.4.1/bin/../lib/gcc/arm-none-eabi/5.4.1/armv7-m\libgcc.a(_arm_truncdfsf2.o)
 .ARM.attributes
                0x00000834       0x1d c:/program files (x86)/cypress/psoc creator/4.3/psoc creator/import/gnu/arm/5.4.1/bin/../lib/gcc/arm-none-eabi/5.4.1/armv7-m\libgcc.a(_arm_addsubsf3.o)
 .ARM.attributes
                0x00000851       0x1d c:/program files (x86)/cypress/psoc creator/4.3/psoc creator/import/gnu/arm/5.4.1/bin/../lib/gcc/arm-none-eabi/5.4.1/armv7-m\libgcc.a(_arm_muldivsf3.o)
 .ARM.attributes
                0x0000086e       0x1d c:/program files (x86)/cypress/psoc creator/4.3/psoc creator/import/gnu/arm/5.4.1/bin/../lib/gcc/arm-none-eabi/5.4.1/armv7-m\libgcc.a(_arm_fixsfsi.o)
 .ARM.attributes
                0x0000088b       0x2d c:/program files (x86)/cypress/psoc creator/4.3/psoc creator/import/gnu/arm/5.4.1/bin/../lib/gcc/arm-none-eabi/5.4.1/../../../../arm-none-eabi/lib/armv7-m\libg_nano.a(lib_a-errno.o)
 .ARM.attributes
                0x000008b8       0x2d c:/program files (x86)/cypress/psoc creator/4.3/psoc creator/import/gnu/arm/5.4.1/bin/../lib/gcc/arm-none-eabi/5.4.1/../../../../arm-none-eabi/lib/armv7-m\libg_nano.a(lib_a-exit.o)
 .ARM.attributes
                0x000008e5       0x2d c:/program files (x86)/cypress/psoc creator/4.3/psoc creator/import/gnu/arm/5.4.1/bin/../lib/gcc/arm-none-eabi/5.4.1/../../../../arm-none-eabi/lib/armv7-m\libg_nano.a(lib_a-impure.o)
 .ARM.attributes
                0x00000912       0x2d c:/program files (x86)/cypress/psoc creator/4.3/psoc creator/import/gnu/arm/5.4.1/bin/../lib/gcc/arm-none-eabi/5.4.1/../../../../arm-none-eabi/lib/armv7-m\libg_nano.a(lib_a-init.o)
 .ARM.attributes
                0x0000093f       0x2d c:/program files (x86)/cypress/psoc creator/4.3/psoc creator/import/gnu/arm/5.4.1/bin/../lib/gcc/arm-none-eabi/5.4.1/../../../../arm-none-eabi/lib/armv7-m\libg_nano.a(lib_a-memcpy-stub.o)
 .ARM.attributes
                0x0000096c       0x2d c:/program files (x86)/cypress/psoc creator/4.3/psoc creator/import/gnu/arm/5.4.1/bin/../lib/gcc/arm-none-eabi/5.4.1/../../../../arm-none-eabi/lib/armv7-m\libg_nano.a(lib_a-memset.o)
 .ARM.attributes
                0x00000999       0x2d c:/program files (x86)/cypress/psoc creator/4.3/psoc creator/import/gnu/arm/5.4.1/bin/../lib/gcc/arm-none-eabi/5.4.1/../../../../arm-none-eabi/lib/armv7-m\libg_nano.a(lib_a-sprintf.o)
 .ARM.attributes
                0x000009c6       0x2d c:/program files (x86)/cypress/psoc creator/4.3/psoc creator/import/gnu/arm/5.4.1/bin/../lib/gcc/arm-none-eabi/5.4.1/../../../../arm-none-eabi/lib/armv7-m\libg_nano.a(lib_a-nano-svfprintf.o)
 .ARM.attributes
                0x000009f3       0x2d c:/program files (x86)/cypress/psoc creator/4.3/psoc creator/import/gnu/arm/5.4.1/bin/../lib/gcc/arm-none-eabi/5.4.1/../../../../arm-none-eabi/lib/armv7-m\libg_nano.a(lib_a-nano-vfprintf_i.o)
 .ARM.attributes
                0x00000a20       0x2d c:/program files (x86)/cypress/psoc creator/4.3/psoc creator/import/gnu/arm/5.4.1/bin/../lib/gcc/arm-none-eabi/5.4.1/../../../../arm-none-eabi/lib/armv7-m\libg_nano.a(lib_a-memchr-stub.o)
 .ARM.attributes
                0x00000a4d       0x2d c:/program files (x86)/cypress/psoc creator/4.3/psoc creator/import/gnu/arm/5.4.1/bin/../lib/gcc/arm-none-eabi/5.4.1/../../../../arm-none-eabi/lib/armv7-m\libg_nano.a(lib_a-memmove.o)
 .ARM.attributes
                0x00000a7a       0x2d c:/program files (x86)/cypress/psoc creator/4.3/psoc creator/import/gnu/arm/5.4.1/bin/../lib/gcc/arm-none-eabi/5.4.1/../../../../arm-none-eabi/lib/armv7-m\libg_nano.a(lib_a-nano-freer.o)
 .ARM.attributes
                0x00000aa7       0x2d c:/program files (x86)/cypress/psoc creator/4.3/psoc creator/import/gnu/arm/5.4.1/bin/../lib/gcc/arm-none-eabi/5.4.1/../../../../arm-none-eabi/lib/armv7-m\libg_nano.a(lib_a-nano-mallocr.o)
 .ARM.attributes
                0x00000ad4       0x2d c:/program files (x86)/cypress/psoc creator/4.3/psoc creator/import/gnu/arm/5.4.1/bin/../lib/gcc/arm-none-eabi/5.4.1/../../../../arm-none-eabi/lib/armv7-m\libg_nano.a(lib_a-nano-reallocr.o)
 .ARM.attributes
                0x00000b01       0x2d c:/program files (x86)/cypress/psoc creator/4.3/psoc creator/import/gnu/arm/5.4.1/bin/../lib/gcc/arm-none-eabi/5.4.1/../../../../arm-none-eabi/lib/armv7-m\libg_nano.a(lib_a-sbrkr.o)
 .ARM.attributes
                0x00000b2e       0x2d c:/program files (x86)/cypress/psoc creator/4.3/psoc creator/import/gnu/arm/5.4.1/bin/../lib/gcc/arm-none-eabi/5.4.1/../../../../arm-none-eabi/lib/armv7-m\libg_nano.a(lib_a-mlock.o)
 .ARM.attributes
                0x00000b5b       0x2d c:/program files (x86)/cypress/psoc creator/4.3/psoc creator/import/gnu/arm/5.4.1/bin/../lib/gcc/arm-none-eabi/5.4.1/../../../../arm-none-eabi/lib/armv7-m\libg_nano.a(lib_a-nano-msizer.o)
 .ARM.attributes
                0x00000b88       0x2d c:/program files (x86)/cypress/psoc creator/4.3/psoc creator/import/gnu/arm/5.4.1/bin/../lib/gcc/arm-none-eabi/5.4.1/../../../../arm-none-eabi/lib/armv7-m\libg_nano.a(lib_a-reent.o)
 .ARM.attributes
                0x00000bb5       0x2d c:/program files (x86)/cypress/psoc creator/4.3/psoc creator/import/gnu/arm/5.4.1/bin/../lib/gcc/arm-none-eabi/5.4.1/armv7-m/crtend.o
 .ARM.attributes
                0x00000be2       0x1d c:/program files (x86)/cypress/psoc creator/4.3/psoc creator/import/gnu/arm/5.4.1/bin/../lib/gcc/arm-none-eabi/5.4.1/armv7-m/crtn.o

/DISCARD/
 *(.note.GNU-stack)
OUTPUT(C:\Software\PSoC Cypress\VCNL4030X01\VCNL4030X01.cydsn\CortexM3\ARM_GCC_541\Debug\VCNL4030X01.elf elf32-littlearm)
